:100000000C94D2060C94F1060C94F1060C94F106B3
:100010000C94F1060C94F1060C948F080C94C5080E
:100020000C94F1060C94F1060C94F1060C94F10674
:100030000C94F1060C94F1060C94F1060C94320C1D
:100040000C94F1060C94F1060C94F1060C94F10654
:100050000C9472440C94943B0C94F1060C94F106AD
:100060000C94F1060C94693C0C94F1060C945D3CE4
:100070000C94F1060C94F1060C94F1060C94F10624
:100080000C94EA4F0C94F1060C94F1060C94F106D2
:100090000C94A73C0C94F1060C949B3C0C94F10638
:1000A0000C94F1060C94F1060C94F1060C94F106F4
:1000B0000C94F1060C94F1060C94F1060C94F106E4
:1000C0000C94F1060C94F1060C94F1060C94F106D4
:1000D0000C94F1060C94F1060C94F1060C94F106C4
:1000E0000C94F1060C942B440C9435440C9421444C
:1000F0000C94DB430C9466440C9457440C944B448E
:100100000C943F440C94F1060C94F1060C94F10607
:100110000C94F1060C94F1060C94F1060C94F10683
:100120000A0025303278002025362E3266204F6EA8
:100130002D426F61726400202573002530327800F3
:100140002025362E3266200020257300756E6B6EDA
:100150006F776E20636D640A00256300682020209D
:10016000202020202020202020202020202020208F
:1001700020202020202020202D2068656C700A0D72
:100180000076202020202020202020202020202039
:10019000202020202020202020202020202D2076FC
:1001A000657273696F6E0A0D007520202020202073
:1001B000202020202020202020202020202020203F
:1001C00020202020202D20757074696D650A0D0097
:1001D000616573205B6F6E7C6F66665D20202020FA
:1001E0002020202020202020202020202D20696E6B
:1001F000746567726574790A0D006164632020205C
:1002000020202020202020202020202020202020EE
:100210002020202020202D2073686F7720765F69B2
:100220006E2C2061312C20613220766F6C746167F6
:1002300065730A0D0063616C69205B5B765F696EB4
:100240007C61317C61325D20766F6C746167655DC5
:10025000202D2063616C6962726174650A0D00640F
:1002600065205B6D61736B5D2020202020202020A5
:1002700020202020202020202020202D20646562A6
:1002800075670A0D0068756D202020202020202031
:10029000202020202020202020202020202020205E
:1002A000202D2068756D69646974792073656E739B
:1002B0006F720A0D0068756D70205B6F6E7C6F66E3
:1002C000665D2020202020202020202020202020AB
:1002D000202D2068756D6964697479207065726D70
:1002E0002073656E736F72207077720A0D006964F7
:1002F000205B72657365745D202020202020202003
:10030000202020202020202020202D20696420680B
:10031000616E646C696E670A0D006D637520202044
:1003200020202020202020202020202020202020CD
:100330002020202020202D206D637520696E666F9F
:100340000A0D006E65205B666C7573685D20202069
:100350002020202020202020202020202020202D90
:10036000206E65696768626F72207461626C650AED
:100370000D006C6F67205B6175746F7C6F6E7C6FB6
:1003800066665D20202020202020202020202D2097
:100390006D6F7465732064617461206F6E205553B6
:1003A000420A0D006F7720202020202020202020CE
:1003B000202020202020202020202020202020203D
:1003C0002D206F6E652D776972652073656E736F72
:1003D00072730A0D007265205B6D61736B5D202086
:1003E000202020202020202020202020202020200D
:1003F000202D206D6F7465207265706F727420738C
:10040000657474696E670A0D007269205B696E74A9
:100410005D2020202020202020202020202020209F
:1004200020202020202D207265706F727420696E4C
:1004300074657276616C0A0D007273202020202092
:1004400020202020202020202020202020202020AC
:1004500020202020202D20726164696F2073746138
:1004600074730A0D00737320202020202020202088
:10047000202020202020202020202020202020207C
:10048000202D2073797374656D2073756D6D6172A5
:10049000790A0D0070777231205B6F6E7C6F666633
:1004A0005D2020202020202020202020202020200F
:1004B0002D2070696E31207077720A0D007265739D
:1004C0007420656570726F6D202020202020202010
:1004D0002020202020202020202D20726573746F82
:1004E000726520656570726F6D0A0D0070777273AA
:1004F000205B646565707C666F7263655F69646CC0
:10050000655D2020202020202D206D637520736CD8
:10051000656570206D6F64650A0D00626F6F7420F1
:1005200020202020202020202020202020202020CB
:10053000202020202020202D207265626F6F740AF9
:100540000D007570677220202020202020202020A0
:1005500020202020202020202020202020202D208E
:100560007265626F6F742076696120626F6F746C60
:100570006F616465720A0D0074657374205B6F6649
:10058000667C317C327C335D20202020202020209E
:10059000202020202D2074657374206D6F64657396
:1005A0000A0D00557074696D6520256420646179B9
:1005B000732C20253032643A253032643A253032AB
:1005C000640A00204E657665722D7573656420732C
:1005D0007461636B203E2025642062797465730A20
:1005E0000025352E3266200025372E33662025372C
:1005F0002E336600253032780025730A004E657769
:100600002064656275673D307825580A004375722D
:1006100072656E742064656275673D307825580A8E
:1006200000445F4F5045523D307825780A00445FC2
:1006300052583D307825780A00445F54583D307850
:1006400025780A00445F504B543D6E307825780A77
:1006500000445F4F573D307825780A00445F4C4591
:10066000443D307825780A00445F504F5745523D4D
:10067000307825780A00445F4556454E543D307821
:1006800025780A00445F50305F4C45443D30782562
:10069000780A00445F50315F4C45443D30782578FE
:1006A0000A00445F4145533D307825780A00445F95
:1006B0005057525F313D307825780A002563002578
:1006C00063002563004F4B0A002563007478206C9B
:1006D000656E20202020207268206D6973732020B1
:1006E00020207268207374616C652020207268205D
:1006F0006D6973630A00252D31306C7520252D310D
:10070000306C7520252D31306C7520252D31306CE5
:1007100075200A002563004D43553D2530366C7821
:100720000020467573653A2065653D253032782096
:1007300068663D25303278206C663D253032782061
:100740006C623D2530327800204F534343414C3D8D
:1007500025642000256300256300256300256300D0
:100760004E6577207265706F72743D307825580A37
:10077000005573696E67207265706F72743D3078D2
:1007800025580A00525F49443D0909307825780A06
:1007900000525F543D0909307825780A00525F54B1
:1007A000313D0909307825780A00525F545F4D4386
:1007B000553D09307825780A00525F565F4D435504
:1007C0003D09307825780A00525F50303D090930E4
:1007D0007825780A00525F50305F543D090930781F
:1007E00025780A00525F50313D0909307825780A92
:1007F00000525F50315F543D0909307825780A0076
:10080000525F555054494D453D09307825780A00CE
:10081000525F52483D0909307825780A00525F56E8
:100820005F494E3D0909307825780A00525F413111
:100830003D0909307825780A00525F41323D0909A7
:10084000307825780A002563004E65772072657040
:100850006F727420696E74657276616C3D252D64CB
:10086000207365630A0043757272656E7420726549
:10087000706F727420696E74657276616C3D252D9F
:1008800064207365630A0025630025630053797350
:1008900074656D2053756D6D6172790A0049443D30
:1008A000004E65696768626F72207461626C6520D2
:1008B00073697A653D25640A0052494D452061649B
:1008C00064723D252D642E252D640A005265706FDB
:1008D000727420496E74657276616C3D252D640AD0
:1008E000005265706F7274204D61736B3D307825D6
:1008F0002D780A00565F494E3D252D352E32660A69
:1009000000565F4D43553D252D352E32660A005564
:1009100053425F5057523D25730A00496E74722E40
:1009200020546F74616C3A2050303D252D6C64204A
:1009300050313D252D6C640A00496E74722E20538F
:1009400065633A20202050303D252D372E33662018
:1009500050313D252D372E33660A004C6F67206DD0
:100960006F64653D006175746F0A0025730A004865
:10097000554D5F5057525F414C574159533D257378
:100980000A0044656275673D3078252D780A00506D
:100990007772313D25730A002563002563005248B4
:1009A0003D252D342E31662000545F52483D252DC3
:1009B000342E316620002563005854414C5F545258
:1009C000494D3D2564004572726F72203020566F8C
:1009D0006C74004572726F72203020566F6C740018
:1009E0004572726F72203020566F6C740025352E60
:1009F0003266200025372E33662025372E336600D9
:100A000025730A005465737420312025730A00543D
:100A100065737420322025730A0054657374203383
:100A20002025730A005465737420342025730A004E
:100A300025730A0025730A0025730A002563002523
:100A40006300532025642E256420636C6F636B2044
:100A5000256C7520747820256C7520727820256CA3
:100A6000752072747820256C752072727820256C40
:100A700075207265786D697420256C752061636BD3
:100A8000747820256C75206E6F61636B74782025F7
:100A90006C752061636B727820256C752074696DAC
:100AA00065646F757420256C752062616461636B89
:100AB000727820256C7520746F6F6C6F6E672025BF
:100AC0006C7520746F6F73686F727420256C75205D
:100AD00062616473796E636820256C75206261645D
:100AE00063726320256C7520636F6E74656E746924
:100AF0006F6E64726F7020256C752073656E64690B
:100B00006E6764726F7020256C75206C6C74782031
:100B1000256C75206C6C727820256C750A00452058
:100B200025642E256420636C6F636B20256C752013
:100B300063707520256C75206C706D20256C752098
:100B400069727120256C7520676C656420256C7551
:100B500020796C656420256C7520726C6564202595
:100B60006C7520747820256C75206C697374656EC3
:100B700020256C752073656E736F727320256C75FC
:100B80002073657269616C20256C750A000A2A2A37
:100B90002A2A2A2A2A426F6F74696E672025732ACF
:100BA0002A2A2A2A2A2A0A0052616E646F6D204579
:100BB0005549363420616464726573732067656ECD
:100BC0006572617465640A004D414320616464721A
:100BD000657373200025783A000A00257320257379
:100BE0002C206368616E6E656C20257520706F77B0
:100BF0006572202575002C20636865636B20726127
:100C0000746520257520487A000A004F6E6C696E65
:100C1000650A00257325730A006C6F63616C686F49
:100C200073740041544D4547413132387266613129
:100C300000020000FFFE000001454550524F4D20CC
:100C4000697320636F72727570742C20726577728D
:100C50006974696E67207769746820646566617578
:100C60006C74732E0A006E616E00696E660000403F
:100C70007A10F35A00A0724E18090010A5D4E800AB
:100C800000E87648170000E40B54020000CA9A3BC3
:100C9000000000E1F5050000809698000000404249
:100CA0000F000000A08601000000102700000000D7
:100CB000E803000000006400000000000A000000DB
:100CC00000000100000000002C76D888DC674F0887
:100CD00023DFC1DFAE59E1B1B796E5E3E453C63A8D
:100CE000E651997696E8E6C28426EB898C9B62ED04
:100CF000407C6FFCEFBC9C9F40F2BAA56FA5F490BE
:100D0000055A2AF75C936B6CF9676DC11BFCE0E434
:100D10000D47FEF520E6B500D0ED902E030094358A
:100D200077050080841E080000204E0A000000C8DD
:100D30000C333333330F986E12831141EF8D21142E
:100D4000893BE65516CFFEE6DB18D1844B381BF7FE
:100D50007C1D901DA4BBE424203284725E2281009D
:100D6000C9F124ECA1E53D27494E46494E49545965
:100D70004E414E000020410000C84200401C462069
:100D8000BCBE4CCA1B0E5AAEC59D74CDCCCC3D0A20
:100D9000D7233C17B7D13877CC2B329595E6241F53
:100DA000B14F0A0011241FBECFEFD1E4DEBFCDBF8B
:100DB00016E0A0E0B2E0E8EFF3ED00E00BBF02C008
:100DC00007900D92AA30B107D9F71CE2AAE0B6E06D
:100DD00001C01D92A837B107E1F70E94125D0C9483
:100DE000FA690C940000E091C416F0E0EF71F07025
:100DF000E75EF84E80838091C4168F5F8093C4169F
:100E00008091B22388608093B2234FE554E0CA01F9
:100E100061E10E94352D80E090E008956F927F920D
:100E20008F929F92AF92BF92CF92DF92EF92FF92FA
:100E30000F931F93CF93DF934B01809110069091F6
:100E4000110681FD74980E94C1335C0186E196E031
:100E50000E94312E0AC0CE010296B4010E940C2BD2
:100E60000097E9F4CE010E94D72EEC01009799F784
:100E7000D5C0CE010296B4010E94032BD5018C91FE
:100E80008150888780E091E0A0E0B0E089879A8770
:100E9000AB87BC8786E196E0BE010E94A02ECE0102
:100EA0000D9660E074E646E258E09E010E94C23072
:100EB00084E00E94E5349D838C8383E00E94E534C6
:100EC0003C019F838E83F501C0808885C81ADD248C
:100ED000EE24FF24A6E0CC0CDD1CEE1CFF1CAA9522
:100EE000D1F769857A858B859C8520EC30E040E0E0
:100EF00050E00E94FA62DC01CB01892F9A2FAB2FC0
:100F0000BB27C80ED91EEA1EFB1EC986DA86EB86F1
:100F1000FC86D5018C9188878091100690911106EE
:100F200081FD08C080917F0480FD04C081FF6EC0F8
:100F30001D9B6CC0EDB7FEB772970FB6F894FEBF5D
:100F40000FBEEDBF0DB71EB70F5F1F4F80E092E0E1
:100F500092838183C5010196D80113969C938E9349
:100F60001297F401808114968C93149715961C9215
:100F70001597818116968C93169717961C92D5011A
:100F80008C91F801808711868C819D81938782875F
:100F900075866486BB27AF2D9E2D8D2D97878687FE
:100FA000C701B60124E630E040E050E00E94FA625A
:100FB000672F782F892F99270E944063DC01CB018E
:100FC000F801918B808B0E94D06620919B048DB795
:100FD0009EB742960FB6F8949EBF0FBE8DBF2223D8
:100FE000A9F000D000D0EDB7FEB731968FE39AE0BC
:100FF000ADB7BEB712969C938E931197228313823E
:101000000E94E2660F900F900F900F908091100653
:101010009091110681FF0BC0749A09C08CEA94E08C
:101020000E94BE2DEC01009709F023CFEFCFDF9196
:10103000CF911F910F91FF90EF90DF90CF90BF90D5
:10104000AF909F908F907F906F900895CF93DF9394
:10105000EC01809110069091110687FF2EC08DB78C
:101060009EB70C970FB6F8949EBF0FBE8DBFEDB71D
:10107000FEB731968CE392E0ADB7BEB712969C9363
:101080008E9311978A81828313828B818483158248
:101090008885868317828C819D81918780878E8148
:1010A0009F81938782870E94D0668DB79EB70C96EA
:1010B0000FB6F8949EBF0FBE8DBF86E196E0BE01CD
:1010C0000E946B2E8CEA94E0BE010E94E92DDF9114
:1010D000CF91089587EE93E08115910511F0019766
:1010E000F1F70895882369F06D987598ED9A8091CD
:1010F0006A00886080936A008091680081608093B4
:1011000068006E98769AEE9A80916A008062809369
:101110006A008091680081608093680008951F9242
:101120000F920FB60F9211248F939F93AF93BF939B
:101130008091680080FF20C080919223909193233A
:10114000A0919423B09195230196A11DB11D809388
:10115000922390939323A0939423B093952380910B
:1011600010069091110690FF07C0749882E090E0FD
:101170009093A9048093A804BF91AF919F918F9100
:101180000F900FBE0F901F9018951F920F920FB6E1
:101190000F9211248F939F93AF93BF938091680018
:1011A00080FF20C08091962390919723A09198234F
:1011B000B09199230196A11DB11D80939623909320
:1011C0009723A0939823B093992380911006909130
:1011D000110691FF07C0739882E090E09093A904F4
:1011E0008093A804BF91AF919F918F910F900FBEF4
:1011F0000F901F90189580937C0080917B00877FD3
:1012000080937B0080917C00806C80937C0085E0E3
:1012100080937A0080917A00806880937A00809130
:101220007B0087FFFCCF80917B0085FFFCCF809106
:101230007A00806480937A0080917A0086FDFCCFEA
:10124000109279001092780084E090E060E070E005
:1012500020917A00206420937A0020917A0026FD64
:10126000FCCF2091780030917900620F731F0197B5
:1012700079F710927C0080917A008F7780937A00C2
:10128000769567957695679580E090E00E94E56198
:10129000462F572F682F792FCB01BA01089580E090
:1012A0000E94FB082091A4043091A5044091A6045B
:1012B0005091A7040E94976221EE3AE744E95EE369
:1012C0000E941561462F572F682F792FCB01BA0145
:1012D000089580E1809351018093510190915101D3
:1012E00095FF03C08F5F8F31B9F76BE4869FB00124
:1012F0001124882777FD8095982F0E94E76120E0D0
:1013000030E64FE954E40E941561462F572F682FAD
:10131000792FCB01BA0120E030E04AE754E40E9483
:101320007D61462F572F682F792FCB01BA01089581
:101330008091830483FF4DC080917B0088608093FF
:101340007B0089EC80937C0085E080937A0080911B
:101350007A00806880937A0080917B0087FFFCCFC1
:1013600080917B0085FFFCCF80917A008064809320
:101370007A0080917A0086FDFCCF80917A008064AB
:1013800080937A0080917A0086FDFCCF609178008E
:101390007091790080E090E00E94E56127ED33EAEA
:1013A00040E95FE30E94976226E636E648E853E4A8
:1013B0000E941461DC01CB018093C0169093C1168A
:1013C000A093C216B093C31680917A008F77809352
:1013D0007A000895CF92DF92EF92FF921F93CF93FE
:1013E000DF93CDB7DEB729970FB6F894DEBF0FBEF7
:1013F000CDBF6C0110920A068FEF898325EDE22E96
:1014000026E1F22E10E03FC0183009F440C0CE01B2
:101410000196BE016E5F7F4F0E94A83689818F3F83
:1014200011F08E3F19F480930A0631C0CE01029666
:10143000C114D10479F40E94C1368093AF23DE0138
:101440001296E7EAF3E288E09D9191938150E1F7EB
:1014500011E01DC00E94C136F7018083DE011296A3
:1014600020E030E0C70108974D91FC01E20FF31F27
:1014700040832F5F3F4F28303105B1F71F5F89E070
:1014800090E0E80EF91E8981882309F0BDCF812FF5
:1014900029960FB6F894DEBF0FBECDBFDF91CF9176
:1014A0001F91FF90EF90DF90CF90089500D080E2E1
:1014B00091E0EDB7FEB7928381830E94E2660F90C0
:1014C0000F9008952F923F924F925F926F927F926A
:1014D0008F929F92AF92BF92CF92DF92EF92FF9244
:1014E0000F931F93CF93DF9300D000D0CDB7DEB71B
:1014F0008C01009741F489E290E06BE270E04AE2EF
:1015000050E027E00AC08130910549F489E290E07B
:101510006BE270E04AE250E026E00E947D35C801AF
:101520000E94EA09ABE08A2EA6E09A2E800E911E58
:10153000D4018C930115110599F065EDA62E66E195
:10154000B62E00E010E07BE3672E71E0772EE0E43A
:101550004E2EE1E05E2EF8E42F2EF1E03F2E10C17A
:1015600087EA93E20E94E437FC01BF01882777FDF8
:101570008095982F0E94E761F82EE92E07EA13E282
:10158000AA24BB2452E2C52E51E0D52ED8018D915C
:101590008D0100D000D0EDB7FEB73196ADB7BEB724
:1015A0001296DC92CE921197828313826B837C8396
:1015B0000E94E2660894A11CB11C0F900F900F903E
:1015C0000F906B817C81B8E0AB16B104F9F600D0C6
:1015D00000D000D00DB71EB70F5F1F4F87E291E01C
:1015E000EDB7FEB7928381839701862F972FA32FA4
:1015F000BE2DBC01CD0120E030E048EC52E40E9459
:101600007D61DC01CB01F80182839383A483B583E0
:101610000E94E2662DB73EB72A5F3F4F0FB6F8949F
:101620003EBF0FBE2DBF8091AF23882319F08BE6FC
:1016300092E002C084E792E000D000D027E331E0DE
:10164000ADB7BEB712963C932E93119714969C9308
:101650008E9313970E94E2660F900F900F900F9059
:101660000E94560A94C0C80133E0880F991F3A952A
:10167000E1F7800F911F8353994E0E94E437FC01DC
:10168000BF01882777FD8095982F0E94E7616C0144
:1016900020E030E048EFE42E4FEFF42EEA0CFB1C84
:1016A00000D000D0ADB7BEB71196EDB7FEB77282CD
:1016B0006182F701E20FF31F808112968C931297DB
:1016C00013961C9229833A836B837C830E94E26683
:1016D00029813A812F5F3F4F0F900F900F900F900D
:1016E0006B817C8128303105D9F600D000D000D044
:1016F000EDB6FEB60894E11CF11CADB7BEB712966C
:101700005C924E921197862F972FAC2DBD2DBC0168
:10171000CD0120E030E048EC52E40E947D61DC0124
:10172000CB01F70182839383A483B5830E94E26691
:101730002DB73EB72A5F3F4F0FB6F8943EBF0FBE9E
:101740002DBFD5018C91882319F08BE692E002C061
:1017500084E792E000D000D0EDB7FEB7328221825C
:10176000948383830E94E2660F900F900F900F90F6
:101770000E94560A0F5F1F4F29E030E0A20EB31EF1
:10178000D4018C9190E0081719070CF46CCF0F90DE
:101790000F900F900F90DF91CF911F910F91FF90BD
:1017A000EF90DF90CF90BF90AF909F908F907F9001
:1017B0006F905F904F903F902F900895CF93DF935D
:1017C00000D0CDB7DEB78091A82389838091AE2366
:1017D0008A83CE0101960E941E2B0F900F90DF91FD
:1017E000CF910895CF93DF93EC018091A7238F3F92
:1017F000B1F58091A8238F3F91F58091A9238F3F68
:1018000071F58091AA238F3F51F58091AB238F3FD3
:1018100031F58091AC238F3F11F58091AD238F3F3F
:10182000F1F48091AE238F3FD1F489E290E06BE236
:1018300070E04AE250E027E00E947D3580E090E0D1
:101840000E94EA09C55FD94F888387EA93E260E086
:1018500070E049E050E00E9428680E94DE0BDF91B2
:10186000CF9108951F920F920FB60F920BB60F9261
:1018700011242F933F934F935F936F937F938F9395
:101880009F93AF93BF93EF93FF938091B2238260B6
:101890008093B22380917F0486FD2B9A87FD2B9A3B
:1018A0008091A8049091A9041816190614F4749A4A
:1018B000739A809110069091110685FF02C074986A
:1018C00073988091AA049091AB0401979093AB0414
:1018D0008093AA04009709F068C080911406909143
:1018E00015069C012F5F3F4F309315062093140679
:1018F00040913D1F50913E1F60913F1F7091401FCE
:101900004F5F5F4F6F4F7F4F40933D1F50933E1F80
:1019100060933F1F7093401F20E130E03093AB0491
:101920002093AA0420917F0420FD02C01D9B05C0C6
:1019300010920E0610920D0606C021E030E03093A2
:101940000E0620930D06209181043091820421150A
:101950003105A1F00296B9010E941963009771F454
:101960007798809110069091110693FF07C07498A4
:1019700084E090E09093A9048093A8042115310598
:1019800081F08091140690911506B9010E941963A7
:10199000009739F487E494E062E140E050E00E946F
:1019A000352D80917F0486FD2B9880ED94E060E0DA
:1019B00040E050E00E94352DFF91EF91BF91AF9133
:1019C0009F918F917F916F915F914F913F912F9157
:1019D0000F900BBE0F900FBE0F901F901895809127
:1019E000C4169091511F891B08950E94EF0C882303
:1019F00079F0E091511FF0E0EF71F070E75EF84E82
:101A0000808190E02091511F2F5F2093511F0895F6
:101A10008FEF9FEF0895CF93DF93EC0110921306A1
:101A20001092120688819981009731F022E08F3957
:101A3000920709F0B7C009C00E94EF0C882341F457
:101A40008FE992E099838883B1C0613109F0AEC01B
:101A5000F89478940E94F50C90E090931F06809380
:101A60001E068D3009F47CC08F3F31F38231910521
:101A700069F18F37910521F08830910509F053C045
:101A80008091200690912106181619060CF060C06E
:101A90006091722C7091732C88E090E00E94A46693
:101AA0006091722C7091732C80E290E00E94A46689
:101AB0006091722C7091732C88E090E00E94A46673
:101AC000809120069091210601973EC06091722C72
:101AD0007091732C8DE090E00E94A4661092230612
:101AE0001092220614C08E5A904EFC0180816091A3
:101AF000722C7091732C90E00E94A4668091220653
:101B0000909123060196909323068093220680915C
:101B100022069091230620912006309121068217FB
:101B200093070CF315C06091722C7091732C0E9476
:101B3000A466809120069091210620911E06FC014A
:101B4000EE5AF04E20830196909321068093200652
:101B500080912006909121068F33910509F06CCF7A
:101B60001092511F1092C416809120069091210668
:101B7000FC01EE5AF04E10829093130680931206E9
:101B800010922106109220068091B0239091B123EB
:101B9000009709F451CF60911C0640E050E00E948C
:101BA000352D4ACF1982188283E001C081E0DF9190
:101BB000CF910895789480910D0690910E0600972C
:101BC00031F080917F049091800490FF03C083B72F
:101BD000817F03C083B7817F866083BFF89483B71A
:101BE000816083BF7894889583B78E7F83BF789414
:101BF0000895CF93DF93EC0188819981009721F0BC
:101C000027E0883C920789F40E94DA0D8091BA0D92
:101C10009091BB0D65E840E050E00E94352D88ECC6
:101C200097E09983888381E003C01982188283E05A
:101C3000DF91CF910895FF920F931F93CF93DF937E
:101C4000729A80917F0483FD06C0C0E5D0E00E94B7
:101C50006A082197E1F78EE40E946238882309F030
:101C60008BC0C0E5D0E00E946A082197E1F78FE4BD
:101C70000E9462380E94CA38C82F82958695869540
:101C800083708130A9F44091451F5091461F6091A7
:101C9000471F7091481F4F5F5F4F6F4F7F4F4093BB
:101CA000451F5093461F6093471F7093481F16C0EF
:101CB0008230A0F04091491F50914A1F60914B1F04
:101CC00070914C1F4F5F5F4F6F4F7F4F4093491F85
:101CD00050934A1F60934B1F70934C1F0E94CA3849
:101CE0001C2F1F7300E0080F111D0E94CA38F82E28
:101CF0000E94D438DF2D90E0C92FC80FD11DD69592
:101D0000C795D695C7950E94B13880917F0483FF0F
:101D10007298B80180E090E00E94E56120E134E033
:101D200048EC5BE30E949762DC01CB01809339179A
:101D300090933A17A0933B17B0933C17BE0180E0F5
:101D400090E00E94E56124EA3CEF44E25CE30E94FB
:101D5000976220E030E040E252E40E941461DC012E
:101D6000CB018093B3239093B423A093B523B09376
:101D7000B62380E090E015C08091411F9091421FF2
:101D8000A091431FB091441F0196A11DB11D8093E6
:101D9000411F9093421FA093431FB093441F81E0C3
:101DA00090E0DF91CF911F910F91FF90089572986D
:101DB000729A8EE40E94623880EA0E94B93880E00C
:101DC0000E94B93880E00E94B9388FE40E946238DE
:101DD0000E94CA3882958695869583708130A9F4D1
:101DE0004091451F5091461F6091471F7091481FB9
:101DF0004F5F5F4F6F4F7F4F4093451F5093461F7C
:101E00006093471F7093481F16C08230A0F0409126
:101E1000491F50914A1F60914B1F70914C1F4F5F9B
:101E20005F4F6F4F7F4F4093491F50934A1F6093FE
:101E30004B1F70934C1F00D000D0EDB7FEB731960A
:101E400025E732E0ADB7BEB712963C932E931197BB
:101E5000828313820E94D0660F900F900F900F9094
:101E60008EE40E94623880E80E94B93880E00E94C7
:101E7000B93880E00E94B9380E94B13880E090E023
:101E8000089500D08CE491E0ADB7BEB712969C9354
:101E90008E9311970E94E26620919B040F900F9001
:101EA0002223A9F000D000D0EDB7FEB7319689E526
:101EB00091E0ADB7BEB712969C938E931197228393
:101EC00013820E94E2660F900F900F900F9008957A
:101ED00000D08CE591E0EDB7FEB7928381830E943C
:101EE000E26681E891E0EDB7FEB7928381830E94BC
:101EF000E26689EA91E0EDB7FEB7928381830E94A2
:101F0000E26680ED91E0EDB7FEB7928381830E9497
:101F1000E2668AEF91E0EDB7FEB7928381830E947B
:101F2000E26685E392E0EDB7FEB7928381830E947B
:101F3000E2668FE592E0EDB7FEB7928381830E945F
:101F4000E26685E892E0EDB7FEB7928381830E9456
:101F5000E26685EB92E0EDB7FEB7928381830E9443
:101F6000E2668EEE92E0EDB7FEB7928381830E9427
:101F7000E2668AE193E0EDB7FEB7928381830E9427
:101F8000E26683E493E0EDB7FEB7928381830E941B
:101F9000E26682E793E0EDB7FEB7928381830E9409
:101FA000E26684EA93E0EDB7FEB7928381830E94F4
:101FB000E26685ED93E0EDB7FEB7928381830E94E0
:101FC000E26689E094E0EDB7FEB7928381830E94D8
:101FD000E26689E394E0EDB7FEB7928381830E94C5
:101FE000E26685E694E0EDB7FEB7928381830E94B6
:101FF000E26684E994E0EDB7FEB7928381830E94A4
:10200000E2668DEB94E0EDB7FEB7928381830E9488
:10201000E2668CEE94E0EDB7FEB7928381830E9476
:10202000E2668BE195E0EDB7FEB7928381830E9473
:10203000E26682E495E0EDB7FEB7928381830E9469
:10204000E26688E795E0EDB7FEB7928381830E9450
:10205000E2660F900F90089585E892E00E9409676C
:1020600008954F925F926F927F928F929F92AF925C
:10207000BF92CF92DF92EF92FF920F931F93CF9375
:10208000DF9300D000D0CDB7DEB760913D1F7091D7
:102090003E1F80913F1F9091401F80903D1F909068
:1020A0003E1FA0903F1FB090401F40903D1F50909A
:1020B0003E1F60903F1F7090401F20913D1F309148
:1020C0003E1F40913F1F5091401F29833A834B830D
:1020D0005C834DB75EB74A5050400FB6F8945EBF70
:1020E0000FBE4DBF0DB71EB70F5F1F4F23EA35E080
:1020F000EDB7FEB732832183A0E8CA2EA1E5DA2E20
:10210000A1E0EA2EF12CA70196010E944063F8019C
:1021100033832283C501B401A70196010E94406365
:10212000B0E1CB2EBEE0DB2EE12CF12CA701960115
:102130000E944063332727FD3095F80135832483BF
:10214000C301B201A70196010E9440632CE3C22E95
:10215000D12CE12CF12CA70196010E94406333277A
:1021600027FD3095F8013783268369817A818B8139
:102170009C81A70196010E944063772767FD7095B7
:10218000F801718760870E94E2662DB73EB7265F2F
:102190003F4F0FB6F8943EBF0FBE2DBF0F900F906C
:1021A0000F900F90DF91CF911F910F91FF90EF90C3
:1021B000DF90CF90BF90AF909F908F907F906F9067
:1021C0005F904F900895E8E7FCE28081918122E4DE
:1021D00082349207B9F000D000D083EC95E0ADB71F
:1021E000BEB712969C938E931197E857FC421496B3
:1021F000FC93EE9313970E94E2660F900F900F905E
:102200000F9008953A96B1E4E53FFB07F0F2089588
:10221000EF92FF920F931F93CF93DF930E944F098A
:10222000DC01CB0100D000D000D021EE35E0EDB7CD
:10223000FEB73283218383839483A583B6830E9470
:10224000E2668DB79EB706960FB6F8949EBF0FBE96
:102250008DBF81E00E94FB082091A0043091A10471
:102260004091A2045091A3040E9497628B01D82F41
:10227000C92F82E00E94FB08AB01BC01EDB7FEB79D
:102280003A970FB6F894FEBF0FBEEDBFEDB6FEB69F
:102290000894E11CF11C28EE35E0328321839E0175
:1022A000802F912FA32FB22FF70182839383A483D2
:1022B000B583CB01BA0120919C0430919D044091DB
:1022C0009E0450919F040E949762DC01CB01F701AC
:1022D00086839783A087B1870E94E2668DB79EB7F9
:1022E0000A960FB6F8949EBF0FBE8DBF0E94560A85
:1022F000DF91CF911F910F91FF90EF900895EF9292
:10230000FF920F931F93CF93DF93882389F087EA7F
:1023100093E26FEF70E049E050E00E945A6687EA6E
:1023200093E260E070E049E050E00E94286822C03B
:1023300007EA13E2C0E0D0E034EFE32E35E0F32EFD
:10234000D8018D918D0100D000D0EDB7FEB7319648
:10235000ADB7BEB71296FC92EE92119782831382AC
:102360000E94E26621960F900F900F900F90C83058
:10237000D10531F70E94560ADF91CF911F910F913D
:10238000FF90EF900895CF92DF92EF92FF926091CD
:10239000990470919A0480E090E00E944C6666EA8D
:1023A00072E00E946166009709F07BC083E19AE0C9
:1023B000909384048093830483E894E06DE070E05C
:1023C00042E050E00E9428688CE390E09093820401
:1023D0008093810481E894E06BE070E042E050E09B
:1023E0000E9428688AE090E09093800480937F04A4
:1023F0008FE794E069E070E042E050E00E942868D6
:10240000109211061092100680E196E06BE170E0E8
:1024100042E050E00E9428680F2EF2E2CF2EFFEF3C
:10242000DF2EFCECEF2EFBE3FF2EF02DC092A0047C
:10243000D092A104E092A204F092A30480EA94E076
:1024400063E170E044E050E00E942868C0929C0480
:10245000D0929D04E0929E04F0929F048CE994E057
:102460006FE070E044E050E00E9428688DEE97E451
:10247000AAE8BCE38093A4049093A504A093A604C7
:10248000B093A70484EA94E067E170E044E050E090
:102490000E94286881E00E947F1180E090E00E9405
:1024A000F20BFF90EF90DF90CF9008952F923F9224
:1024B0004F925F926F927F928F929F92AF92BF9254
:1024C000CF92DF92EF92FF920F931F93CF93DF9300
:1024D00000D0CDB7DEB79A838983DC018D919C91C2
:1024E0001197009711F00C948622609199047091D5
:1024F0009A0482E59FE10E944C6682E59FE160E4D8
:1025000070E00E946A66009759F46091722C709195
:10251000732C8AE090E00E94A46681E00C948C22E7
:102520008130910549F42090521F332444245524CE
:10253000662477244301BEC18230910599F430911D
:10254000521F2091531F932F80E0820F911D1C0179
:10255000892F880F880B482E582E682E782E882EAB
:10256000982EA8C18330910509F09CC02091521F7C
:102570008090531FB090541F30E040E050E060E086
:1025800070E080E090E000E10E94555C922EA32E66
:10259000142FF52EE62EC72E282ED92E282D30E00A
:1025A00040E050E060E070E080E090E008E00E94F1
:1025B000555C290DB1E0291508F0B0E03A0DE1E0D5
:1025C0003A1508F0E0E0B30FF1E0B31708F0F0E0DF
:1025D000EF2B410F31E0411708F030E0E40FF1E05C
:1025E000E41708F0F0E03F2B5F0D41E05F1508F0C5
:1025F00040E0A32FA50F31E0A51708F030E0432BF2
:102600006E0D31E06E1508F030E0F42FF60F41E06A
:10261000F61708F040E0342B7C0D41E07C1508F003
:1026200040E0532F570F31E0571708F030E0432BAD
:10263000820D31E0821508F030E0480F61E0481764
:1026400008F060E0362BD90ED30EB20E81E0B21640
:1026500008F080E0182F1B0F71E01B1708F070E0E6
:102660007E0F61E07E1708F060E06A0F31E06A17C4
:1026700008F030E03F0F21E03F1708F020E0250F81
:1026800091E0251708F090E0940F81E0941708F08E
:1026900080E02B2C312E472E562E632E722E892E43
:1026A000982EFDC08430910509F0FBC02091521F87
:1026B0008090531FA090541FB090551F30E040E011
:1026C00050E060E070E080E090E008E10E94555C3E
:1026D000722E932E142FF52EE62EC72E282ED92ECD
:1026E000282D30E040E050E060E070E080E090E0D5
:1026F00000E10E94555C270DF1E0271508F0F0E09D
:10270000390DE1E0391508F0E0E0F30FA1E0F3172F
:1027100008F0A0E0EA2B410F31E0411708F030E06B
:10272000E40FA1E0E41708F0A0E03A2B5F0D41E0D0
:102730005F1508F040E0B32FB50F31E0B51708F092
:1027400030E0432B6E0D31E06E1508F030E0A42F21
:10275000A60F41E0A61708F040E0342B7C0D41E0C5
:102760007C1508F040E0532F570F31E0571708F061
:1027700030E0432B820D31E0821508F030E0480F45
:1027800061E0481708F060E0362BD90ED30E222EF8
:102790002B0C81E0221608F080E0B82EBF0E81E0FD
:1027A000BF1608F080E0982E9E0E81E09E1608F07D
:1027B00080E0C82ECB0E11E0CB1608F010E01A0F07
:1027C00081E01A1708F080E0F82EF50E81E0F5168A
:1027D00008F080E0E82EE40E81E0E41608F080E0E6
:1027E000D80E2A2D30E040E050E060E070E080E05C
:1027F00090E008E00E94555C220DE1E0221508F00F
:10280000E0E03B0DF1E03B1508F0F0E0E30FA1E064
:10281000E31708F0A0E0FA2B490D31E0491508F064
:1028200030E0F40FA1E0F41708F0A0E03A2B5C0DC3
:1028300041E05C1508F040E0A32FA50F31E0A5179B
:1028400008F030E0432B610F31E0611708F030E011
:10285000542F560F41E0561708F040E0342B7F0DFF
:1028600041E07F1508F040E0632F670F31E0671704
:1028700008F030E0432B8E0D31E08E1508F030E08B
:10288000480F71E0481708F070E0372BD90E222E60
:102890003E2E4F2E5A2E652E762E842E932E9D0C74
:1028A00009C08AE0282E3324442455246624772442
:1028B000882499240E94560AB2E72B1689F43B1605
:1028C00079F4E5E64E1661F4552051F4662041F4A2
:1028D000772031F4882021F4992011F40C94B41C51
:1028E0009101A201B301C401B2E7AB2E12E7B12EF0
:1028F00005E6C02EDD24EE24FF2400E010E00E9457
:10290000CF5C823008F0BFC1F7E72F1689F48FE65D
:10291000381671F4442061F4552051F4662041F4D6
:10292000772031F4882021F4992011F40C94961D1D
:102930009101A201B301C401F7E7AF2EAFE6BA2EB1
:10294000CC24DD24EE24FF2400E010E00E94CF5CC4
:10295000823008F0A3C094E6291689F4A1E63A165D
:1029600071F4442061F4552051F4662041F477203D
:1029700031F4882021F4992011F40C94F321910171
:10298000A201B301C40104E6A02EE1E6BE2ECC24D0
:10299000DD24EE24FF2400E010E00E94CF5C8230B2
:1029A00008F046C0B5E72B1679F4332069F44420CB
:1029B00059F4552049F4662039F4772029F4882009
:1029C00019F4992009F432C6E6E72E1679F433207B
:1029D00069F4442059F4552049F4662039F47720ED
:1029E00029F4882019F4992009F42FC6F8E62F1647
:1029F00011F00C948422332011F00C948422442092
:102A000011F00C948422552011F00C94842266203D
:102A100011F00C948422772011F00C9484228820E9
:102A200011F00C948422992011F00C948422DBC5BF
:102A300084E6281681F499E6391669F4442059F49D
:102A4000552049F4662039F4772029F4882019F4B8
:102A5000992009F4CBC5A5E62A1689F4BEE63B16F3
:102A600071F4442061F4552051F4662041F477203C
:102A700031F4882021F4992011F40C94F81DE5E636
:102A80002E1611F00C948422F4E63F1611F00C94EB
:102A90008422442011F00C948422E0C083E728169D
:102AA00089F492E7391671F4442061F4552051F409
:102AB000662041F4772031F4882021F4992011F424
:102AC0000C9434209101A201B301C401B3E7AB2EF1
:102AD00012E7B12ECC24DD24EE24FF2400E010E028
:102AE0000E94CF5C823008F04BC0A5E62A1681F424
:102AF0003B1471F4442061F4552051F4662041F4F4
:102B0000772031F4882021F4992011F40C94BA1E16
:102B1000B9E62B1689F4E2E73E1671F4442061F41D
:102B2000552051F4662041F4772031F4882021F4B7
:102B3000992011F40C94DB1FF3E32F1611F00C9481
:102B4000842281E7381611F00C948422442011F07D
:102B50000C948422552011F00C948422662011F0EC
:102B60000C948422772011F00C948422882011F098
:102B70000C948422992011F00C9484220C94F3215B
:102B800093E6291691F4A4E63A1679F4B1E64B16C9
:102B900061F4552051F4662041F4772031F4882007
:102BA00021F4992011F40C94F3219101A201B301B5
:102BB000C401E3E6AE2EF4E6BF2EA1E6CA2EDD2464
:102BC000EE24FF2400E010E00E94CF5C823018F574
:102BD000E3E72E1611F00C9484223E1611F00C94AB
:102BE0008422442011F00C948422552011F00C947E
:102BF0008422662011F00C948422772011F00C942A
:102C00008422882011F00C948422992011F00C94D5
:102C100084220C944320F3E72F1689F485E63816B6
:102C200071F491E6491659F4552049F4662039F4B7
:102C3000772029F4882019F4992009F415C5A2E613
:102C40002A1611F00C948422B5E63B1611F00C9470
:102C50008422E4E64E1611F00C948422552011F0E3
:102C60000C948422662011F00C948422772011F0B9
:102C70000C948422882011F00C948422992011F065
:102C80000C948422B3C3F0E72F1691F48CE6381627
:102C900079F495E6491661F4A8E65A1649F46620D7
:102CA00039F4772029F4882019F4992009F49BC479
:102CB0009101A201B301C401A0E7AA2EBCE6BB2E7C
:102CC00015E6C12E08E6D02EEE24FF2400E010E029
:102CD0000E94CF5C823008F0F8C0B0E32B1689F474
:102CE000E1E33E1671F4F1E74F1659F4552049F42B
:102CF000662039F4772029F4882019F4992009F402
:102D000033C69101A201B301C40100E3A02EE1E3A7
:102D1000BE2EF1E7CF2EDD24EE24FF2400E010E0EC
:102D20000E94CF5C823008F04DC087E6281689F4F7
:102D30009FE6391671F4ACE64A1659F4552049F469
:102D4000662039F4772029F4882019F4992009F4B1
:102D5000AEC5B5E72B1689F4E3E63E1671F4FDE641
:102D60004F1659F4552049F4662039F4772029F498
:102D7000882019F4992009F45AC68DE6281611F016
:102D80000C94842295E7391611F00C948422A8E65D
:102D90004A1611F00C948422552011F00C948422D0
:102DA000662011F00C948422772011F00C94842278
:102DB000882011F00C948422992011F00C94842224
:102DC0000C940222B0E72B1689F4E5E63E1671F466
:102DD000F2E74F1659F4552049F4662039F477206C
:102DE00029F4882019F4992009F4C4C79101A2019B
:102DF000B301C401A0E7AA2EB5E6BB2E12E7C12E8F
:102E0000DD24EE24FF2400E010E00E94CF5C82303D
:102E100018F581E3281611F00C948422381611F06D
:102E20000C94842291E7491611F00C9484225520C9
:102E300011F00C948422662011F00C9484227720E7
:102E400011F00C948422882011F00C948422992093
:102E500011F00C948422EBC5A4E72A1689F4BFE68E
:102E60003B1671F44B1661F4E2E65E1649F46620F7
:102E700039F4772029F4882019F4992009F424C41E
:102E8000F9E62F1611F00C9484228CE6381611F016
:102E90000C94842291E6491611F00C948422A3E646
:102EA0005A1611F00C948422662011F00C9484229E
:102EB000772011F00C948422882011F00C94842245
:102EC000992011F00C94842225C1B3E72B1691F4BC
:102ED000E2E73E1679F4F7E74F1661F480E75816FB
:102EE00049F4662039F4772029F4882019F49920D0
:102EF00009F408C79101A201B301C40113E7A12E8F
:102F000002E7B02EE7E7CE2EF0E7DF2EEE24FF2417
:102F100000E010E00E94CF5C823008F04EC02D141B
:102F200091F49DE6391679F4A5E74A1661F4B8E6FE
:102F30005B1649F4662039F4772029F4882019F4C7
:102F4000992009F421C6E1E32E1691F4F2E73F1629
:102F500079F487E7481661F490E7591649F466203A
:102F600039F4772029F4882019F4992009F4AAC0AB
:102F7000A1E62A1611F00C948422BDE63B1611F04E
:102F80000C948422E5E74E1611F00C948422F8E6A6
:102F90005F1611F00C948422662011F00C948422A8
:102FA000772011F00C948422882011F00C94842254
:102FB000992011F00C948422CEC584E7281689F458
:102FC00093E7391671F4A5E64A1659F4581649F4F0
:102FD000662039F4772029F4882019F4992009F41F
:102FE00076C39101A201B301C401E4E7AE2EF3E779
:102FF000BF2EA5E6CA2EB4E7DB2EEE24FF2400E0A8
:1030000010E00E94CF5C823010F52D1411F00C946A
:1030100084223B1411F00C9484224C1411F00C9473
:103020008422B2E75B1611F00C948422662011F022
:103030000C948422772011F00C948422882011F0C3
:103040000C948422992011F00C94842258C6E2E753
:103050002E1691F4F7E63F1679F480E7481661F4EE
:1030600095E7591649F4662039F4772029F4882029
:1030700019F4992009F4EAC3ACE62A1611F00C946D
:103080008422B1E63B1611F00C948422E4E74E163C
:1030900011F00C948422F8E75F1611F00C9484224E
:1030A000662011F00C948422772011F00C94842275
:1030B000882011F00C948422992011F00C94842221
:1030C0000C944A226091990470919A0480E090E0F7
:1030D0000E944C668C016DEA72E00E946166009766
:1030E00019F477980C948622C80160EB72E00E9474
:1030F0006166009719F4779A0C948622779903C039
:103100008DEA92E002C080EB92E000D000D029EF7F
:1031100035E01FC46091990470919A0480E090E0BA
:103120000E944C668C0167EC72E00E946166009719
:1031300009F043C06091990470919A0480E090E096
:103140000E944C668C01009711F40C9486226AEC64
:1031500072E00E946166009729F482E29FEFACEC76
:10316000BBE318C0C8010E943F656B017C0120E0F1
:1031700030E040E050E00E9479618823D1F081E0A6
:103180000E94FB089B01AC01C701B6010E947D6152
:10319000DC01CB018093A0049093A104A093A2042E
:1031A000B093A30480EA94E063E170E044E050E06F
:1031B000ADC200D086EC99E09FC0C80160ED72E01E
:1031C0000E946166009709F047C060919904709170
:1031D0009A0480E090E00E944C668C01009711F404
:1031E0000C9486226AEC72E00E946166009729F4D2
:1031F00082E29FEFACECBBE318C0C8010E943F65C0
:103200006B017C0120E030E040E050E00E947961F9
:103210008823C1F082E00E94FB089B01AC01C7013A
:10322000B6010E947D61DC01CB0180939C049093E8
:103230009D04A0939E04B0939F048CE994E06FE0FA
:1032400070E0B4CF00D083ED99E0ADB7BEB7129671
:103250009C938E93119754C0C80163ED72E00E9455
:103260006166009709F052C06091990470919A04C8
:1032700080E090E00E944C668C01009711F40C9461
:1032800086226AEC72E00E946166009729F48DEE56
:1032900097E4AAE8BCE320C0C8010E943F656B0127
:1032A0007C0120E030E040E050E00E94796188231A
:1032B00001F180E00E94FB084B015C01C701B601EF
:1032C00021EE3AE744E95EE30E941461A50194010E
:1032D0000E947D61DC01CB018093A4049093A5043E
:1032E000A093A604B093A70484EA94E067E170E099
:1032F0005DCF00D080EE99E0EDB7FEB79283818379
:103300000E94E2660F900F900C9486220E944F0953
:10331000AB01BC0100D000D000D08DEE99E0ADB77C
:10332000BEB712969C938E931197EDB7FEB7438369
:103330005483658376830E94E2668DB79EB70696B6
:103340000FB6F8949EBF0FBE8DBF81E00E94FB08B0
:103350002091A0043091A1044091A2045091A304B3
:103360000E9497626B01182F092F82E00E94FB08D0
:10337000AB01BC01ADB7BEB71A970FB6F894BEBF8C
:103380000FBEADBFEDB6FEB60894E11CF11C84EF94
:1033900099E012969C938E93119798018C2D9D2DF8
:1033A000A32FB22FF70182839383A483B583CB012C
:1033B000BA0120919C0430919D0440919E0450914B
:1033C0009F040E949762DC01CB01F70186839783FB
:1033D000A087B1870E94E2668DB79EB70A960FB6A6
:1033E000F8949EBF0FBE8DBF0C948122609199040A
:1033F00070919A0480E090E00E944C66009771F111
:1034000060E070E040E150E00E94FE63AB01BC016F
:1034100080911006909111068417950799F15093A9
:1034200011064093100680E196E06BE170E042E007
:1034300050E00E942868809110069091110600D0FB
:1034400000D02DEF35E0ADB7BEB712963C932E936A
:10345000119714969C938E9313970EC0809110062B
:103460009091110600D000D02DE036E0EDB7FEB708
:1034700032832183948383830E94E2660F900F90AE
:103480000F900F900E94560A00D000D081E296E083
:10349000ADB7BEB712969C938E93119781E090E0E2
:1034A00014969C938E9313970E94E2668EE296E0A8
:1034B000EDB7FEB79283818382E090E094838383AB
:1034C0000E94E26689E396E0ADB7BEB712969C9380
:1034D0008E93119784E090E014969C938E931397AB
:1034E0000E94E26684E496E0EDB7FEB792838183A2
:1034F00088E090E0948383830E94E26681E596E011
:10350000ADB7BEB712969C938E93119780E190E071
:1035100014969C938E9313970E94E2668CE596E036
:10352000EDB7FEB79283818380E290E0948383833A
:103530000E94E26688E696E0ADB7BEB712969C930D
:103540008E93119780E490E014969C938E9313973A
:103550000E94E26686E796E0EDB7FEB7928381832C
:1035600080E890E0948383830E94E26684E896E09A
:10357000ADB7BEB712969C938E93119780E091E001
:1035800014969C938E9313970E94E26683E996E0CB
:10359000EDB7FEB79283818380E092E094838383CA
:1035A0000E94E26682EA96E0ADB7BEB712969C939F
:1035B0008E93119780E094E014969C938E931397CA
:1035C0000E94E2668EEA96E0EDB7FEB792838183B1
:1035D00080E098E0948383830E94E2660F900F90CE
:1035E0000F900F9093C70E94680F90C76091990445
:1035F00070919A0480E090E00E944C666AEC72E060
:103600000E946166009711F481E001C080E00E9491
:103610007F1120919B04222309F478C700D000D0A9
:10362000EDB7FEB731968CEB96E0A5C20E94311043
:1036300020919B04222309F469C700D000D0EDB784
:10364000FEB731968FEB96E096C20E942C10209127
:103650009B04222309F45AC700D000D0EDB7FEB76F
:10366000319682EC96E087C26091990470919A0439
:1036700080E090E00E944C668C016DEA72E00E944E
:103680006166009731F480917F049091800484609A
:1036900033C0C80160EB72E00E9461669C018091BA
:1036A0007F04909180042115310511F48B7F24C093
:1036B00082FF03C08DEA92E002C080EB92E000D06E
:1036C00000D020E03AE08FC20C9400001FC7609148
:1036D000990470919A0480E090E00E944C668C01FD
:1036E00068ED72E00E946166009799F4219A8091DA
:1036F0007F049091800480619093800480937F0484
:103700008FE794E069E070E042E050E00E942868B2
:10371000FDC6C8016AED72E00E946166009739F447
:10372000229A80917F04909180048062E5CFC80145
:103730006CED72E00E946166009739F4239A8091E3
:103740007F04909180048064D7CFC8016EED72E051
:103750000E946166009739F4239A80917F049091CA
:1037600080048068C9CFC80160EB72E00E94616686
:103770009C0180917F04909180042115310539F4DA
:103780008F709093800480937F042B9AB9CF84FF2D
:1037900003C08DEA92E002C080EB92E000D000D03E
:1037A00024E03AE0ADB7BEB712963C932E93119742
:1037B00014969C938E9313970E94E26680917F04E7
:1037C0000F900F900F900F9085FF03C08DEA92E04D
:1037D00002C080EB92E000D000D02FE03AE0EDB7DD
:1037E000FEB732832183948383830E94E2668091B3
:1037F0007F040F900F900F900F9086FF03C08DEA0B
:1038000092E002C080EB92E000D000D02AE13AE0E2
:10381000ADB7BEB712963C932E93119714969C9316
:103820008E9313970E94E26680917F040F900F9011
:103830000F900F9087FF03C08DEA92E002C080EBEB
:1038400092E000D000D025E23AE0CDC100D085EC76
:1038500096E0ADB7BEB712969C938E9311970E94D7
:10386000E26620919B040F900F902223A9F000D0D4
:1038700000D0EDB7FEB7319689EC96E0ADB7BEB794
:1038800012969C938E931197228313820E94E26674
:103890000F900F900F900F9088E10FB6F8948093DF
:1038A0006000109260000FBE0C94007C2FC66091E7
:1038B000990470919A0480E090E00E944C667C012B
:1038C0006DEA72E00E946166009749F40E94A43E8E
:1038D00080917F049091800481608D7F0DCFC7011E
:1038E00060EB72E00E946166009741F40E94953F90
:1038F00080917F04909180048C7FFECE00EE12E0D8
:10390000C701B8010E946166009749F40E94953F83
:1039100080917F04909180048E7F8260EDCE8091B3
:103920007F0481FF0BC000D000D080E39AE0EDB7A8
:10393000FEB792838183148303834ECE80FF03C03E
:103940008DEA92E002C080EB92E000D000D024E348
:103950003AE0ADB7BEB712963C932E9311971496EA
:103960009C938E93139738CE00D08CEC96E0EDB7F5
:10397000FEB7928381830E94E2668DB79EB740971F
:103980000FB6F8949EBF0FBE8DBFEDB7FEB7319650
:1039900086EF96E0ADB7BEB712969C938E931197C3
:1039A00080914D1F90914E1FA0914F1FB091501FBD
:1039B00082839383A483B5838091411F9091421F9A
:1039C000A091431FB091441F86839783A087B1873E
:1039D0008091451F9091461FA091471FB091481FAD
:1039E00082879387A487B5878091491F90914A1F4A
:1039F000A0914B1FB0914C1F86879787A08BB18BEE
:103A00000E94E26620919B04EDB7FEB772960FB656
:103A1000F894FEBF0FBEEDBF222309F477C500D096
:103A200000D0EDB7FEB7319684E197E0A4C0F894DA
:103A300009E081E090E0FC0100935700C895F02C6C
:103A400020E030E0F90100935700C895E02C78940D
:103A5000F89423E030E0F90100935700C895102D49
:103A600082E090E0FC0100935700C895002D789407
:103A700000D000D000D027E137E0EDB7FEB73283A9
:103A800021838091151790911617A0911717B09167
:103A9000181783839483A583B6830E94E26600D0BF
:103AA00000D0EDB7FEB7319681E297E0ADB7BEB773
:103AB00012969C938E93119702831382148315821E
:103AC000E6821782F08611860E94E266EDB7FEB7A5
:103AD0003A960FB6F894FEBF0FBEEDBF0E94E310FA
:103AE0002091660000D000D0EDB7FEB7319688E493
:103AF00097E0ADB7BEB712969C938E931197228331
:103B000013820E94E2660F900F900F900F900E9418
:103B1000560A20919B04222309F4F8C400D000D057
:103B2000EDB7FEB7319684E597E025C080E090E0E0
:103B30000E94620A81E090E00E94620A20919B0448
:103B4000222309F4E3C400D000D0EDB7FEB73196CC
:103B500087E597E010C00E94D70E0E94560A209178
:103B60009B04222309F4D2C400D000D0EDB7FEB7E5
:103B700031968AE597E0ADB7BEB712969C938E93C7
:103B800011972283138228CD6091990470919A0431
:103B900080E090E00E944C668C016DEA72E00E9429
:103BA0006166009731F480917F0490918004886071
:103BB000A3CDC80160EB72E00E9461669C01809118
:103BC0007F04909180042115310511F4877F94CDF5
:103BD00083FF03C08DEA92E002C080EB92E000D048
:103BE00000D028E33AE0EDB7FEB732832183F2CC70
:103BF0006091990470919A0480E090E00E944C6674
:103C000065EE72E00E946166009731F5F89486E1F6
:103C100096E00E94312E0CC0C8010D960E944931D9
:103C20008CEA94E0B8010E94E92DC8010E94D72EC9
:103C30008C01009789F704C086E196E00E945E2E11
:103C400086E196E00E94B92E0097B1F786E196E0F2
:103C50000E942D2E789446C086E196E00E94312E77
:103C60007C010BEE12E03BC08DB79EB70C970FB6F0
:103C7000F8949EBF0FBE8DBFEDB7FEB73196ADB7BE
:103C8000BEB712961C930E931197D70112968C9182
:103C900012978283138213968C91139784831582D3
:103CA00018968C9118978683178214968D919C9103
:103CB00015979187808716968D919C91179793877A
:103CC00082870E94D066EDB7FEB73C960FB6F89497
:103CD000FEBF0FBEEDBFC7010E94D72E7C01E114CD
:103CE000F10411F620919B04222309F40FC400D0A3
:103CF00000D0EDB7FEB731968DE597E03CCF0E943E
:103D0000C31104C46091990470919A0480E090E01A
:103D10000E944C668C016FEB72E00E946166009716
:103D200031F480917F04909180049E7FE5CCC8019E
:103D300064EB72E00E9461669C0180917F04909127
:103D400080042115310511F49160D6CC90FF03C099
:103D500084EB92E002C08FEB92E000D000D022E131
:103D600033E0EDB7FEB732832183948383830E94CF
:103D7000D06634CC6091990470919A0480E090E010
:103D80000E944C66009731F160E070E040E150E045
:103D90000E94FE63DC01CB01909384048093830432
:103DA00000D000D04DB75EB74F5F5F4F20E637E0E1
:103DB000EDB7FEB732832183FA01938382830E9499
:103DC000E2660F900F900F900F9083E894E06DE003
:103DD00070E09ACC00D000D081E797E0ADB7BEB7D5
:103DE00012969C938E9311978091830490918404F2
:103DF00014969C938E9313970E94E2660F900F90F7
:103E00000F900F900E94560A00D000D084E897E0EF
:103E1000EDB7FEB79283818381E090E09483838342
:103E20000E94E26681E997E0ADB7BEB712969C9317
:103E30008E93119782E090E014969C938E93139743
:103E40000E94E2668DE997E0EDB7FEB79283818329
:103E500084E090E0948383830E94E2668AEA97E09C
:103E6000ADB7BEB712969C938E93119788E090E001
:103E700014969C938E9313970E94E26689EB97E0C9
:103E8000EDB7FEB79283818380E190E094838383D2
:103E90000E94E26688EC97E0ADB7BEB712969C939D
:103EA0008E93119780E290E014969C938E931397D3
:103EB0000E94E26685ED97E0EDB7FEB792838183BD
:103EC00080E490E0948383830E94E26684EE97E02E
:103ED000ADB7BEB712969C938E93119780E890E091
:103EE00014969C938E9313970E94E26681EF97E05D
:103EF000EDB7FEB79283818380E091E09483838362
:103F00000E94E26680E098E0ADB7BEB712969C933F
:103F10008E93119780E092E014969C938E93139762
:103F20000E94E26680E198E0EDB7FEB7928381835C
:103F300080E094E0948383830E94E2668DE198E0C0
:103F4000ADB7BEB712969C938E93119780E098E020
:103F500014969C938E9313970E94E2668CE298E0ED
:103F6000EDB7FEB79283818380E090E194838383F1
:103F70000E94E26689E398E0ADB7BEB712969C93C3
:103F80008E93119780E090E214969C938E931397F2
:103F90000E94E26620919B040F900F900F900F906B
:103FA000222309F4B3C200D000D0EDB7FEB731969A
:103FB00086E498E0E0CD6091990470919A0480E0E5
:103FC00090E00E944C66009751F160E070E04AE09A
:103FD00050E00E94FE63DC01CB0190938204809349
:103FE000810400D000D04DB75EB74F5F5F4F29E42A
:103FF00038E0EDB7FEB732832183FA0193838283E1
:104000000E94E2660F900F900F900F9081E894E06D
:104010006BE070E042E050E00E94286818C000D0D9
:1040200000D086E698E0ADB7BEB712969C938E930B
:104030001197809181049091820414969C938E93A1
:1040400013970E94E2660F900F900F900F902091AF
:104050009B04222309F45AC200D000D0EDB7FEB76A
:10406000319687E898E087CD0E94823120919B04A9
:10407000222309F44BC200D000D0EDB7FEB7319631
:104080008AE898E078CD00D08DE898E0EDB7FEB7EB
:10409000928381830E94E2660F900F900E942C1001
:1040A00000D08DE998E0ADB7BEB712969C938E9381
:1040B00011970E94E2660F900F9080E00E947F119E
:1040C0000E94311000D000D081EA98E0EDB7FEB731
:1040D0009283818380E490E0948383830E94E266EC
:1040E00000D0EDB7FEB7319689EB98E0ADB7BEB71B
:1040F00012969C938E9311978091B723828313829B
:104100008091B823848315820E94E2660F900F90FD
:104110008CEC98E0EDB7FEB79283818380918104A7
:1041200090918204948383830E94E26681EE98E0FA
:10413000ADB7BEB712969C938E931197809183046E
:104140009091840414969C938E9313970E94E26638
:104150000F900F900F900F900E944F09AB01BC0180
:1041600000D000D000D084EF98E0EDB7FEB7928386
:10417000818343835483658376830E94E266EDB72F
:10418000FEB736960FB6F894FEBF0FBEEDBF0E9485
:1041900098090E946909AB01BC0100D000D000D091
:1041A00081E099E0ADB7BEB712969C938E931197BC
:1041B000EDB7FEB743835483658376830E94E2663E
:1041C0008DB79EB706960FB6F8949EBF0FBE8DBFF3
:1041D0001D9B03C084EC92E002C080EB92E000D013
:1041E00000D02FE039E0ADB7BEB712963C932E93C6
:1041F000119714969C938E9313970E94E266809178
:10420000922390919323A0919423B0919523409170
:10421000962350919723609198237091992300D011
:1042200000D000D00DB71EB70F5F1F4F2BE139E054
:10423000EDB7FEB732832183F80182839383A48391
:10424000B58346835783608771870E94E266EDB726
:10425000FEB7319689E399E0ADB7BEB712969C934D
:104260008E93119780919F239091A023A091A123D9
:10427000B091A22382839383A483B5838091A323E7
:104280009091A423A091A523B091A6238683978320
:10429000A087B1870E94E266EDB7FEB738960FB6E9
:1042A000F894FEBF0FBEEDBF8BE599E0928381834A
:1042B0000E94E26680917F040F900F9081FF0EC0F4
:1042C00000D085E699E0ADB7BEB712969C938E9369
:1042D00011970E94E2660F900F9017C080FF03C0F5
:1042E0008DEA92E002C080EB92E000D000D02BE695
:1042F00039E0EDB7FEB732832183948383830E9434
:10430000E2660F900F900F900F9080917F0483FFD3
:1043100003C08DEA92E002C080EB92E000D000D0B2
:104320002FE639E0ADB7BEB712963C932E931197A6
:1043300014969C938E9313970E94E26680911006C8
:104340009091110622E839E0EDB7FEB73283218360
:10435000948383830E94E2660F900F900F900F90DA
:10436000779903C08DEA92E002C080EB92E000D022
:1043700000D02FE839E0ADB7BEB712963C932E932C
:10438000119714969C938E9313970E94E2668091E6
:104390007F04909180040F900F900F900F9090FFEA
:1043A00003C084EB92E002C08FEB92E000D000D01B
:1043B00022E133E0EDB7FEB7328321839483838318
:1043C0000E94D06620919B040F900F900F900F9049
:1043D000222309F49BC000D000D0EDB7FEB7319680
:1043E00088E999E0C8CB0E94081120919B04222300
:1043F00009F48CC000D000D0EDB7FEB731968BE940
:1044000099E0B9CB0E941B0E00D000D000D08EE9FD
:1044100099E0EDB7FEB7928381838091391790912F
:104420003A17A0913B17B0913C1783839483A583DF
:10443000B6830E94E26689EA99E0ADB7BEB71296EC
:104440009C938E9311978091B3239091B423A09164
:10445000B523B091B623EDB7FEB783839483A583CC
:10446000B6830E94E2668DB79EB706960FB6F894A3
:104470009EBF0FBE8DBF0E94560A20919B0422232F
:1044800009F444C000D000D0EDB7FEB7319686EBFA
:1044900099E071CB6091990470919A0480E090E06A
:1044A0000E944C666BE173E00E9461660097A1F484
:1044B0006091990470919A0480E090E00E944C66AB
:1044C000009721F10E944365803100F590915201DF
:1044D000982B909352011AC08091520100D000D0C5
:1044E00029EB39E0EDB7FEB73283218390E08F707E
:1044F0009070948383830E94E2660F900F900F90D8
:104500000F900E94560A02C00E94410FA981BA81F1
:1045100011961C921E9283E00F900F90DF91CF9125
:104520001F910F91FF90EF90DF90CF90BF90AF90D1
:104530009F908F907F906F905F904F903F902F90C3
:104540000895F89491E2E0E0F0E0909357008491B0
:10455000E2E0F0E0909357004491E4E0F0E09093C3
:104560005700E49190E0A0E0B0E0DC0199278827B3
:1045700050E060E070E0762F652F542F4427840FC1
:10458000951FA61FB71F8E0F911DA11DB11D8093F2
:10459000151790931617A0931717B09318177894C0
:1045A0000895CF93DF9300D000D000D0CDB7DEB711
:1045B000CE0101966DE070E042E050E00E940A6892
:1045C00089819A812FEF8F3F920749F483E894E025
:1045D0006DE070E042E050E00E94286804C09093D3
:1045E000840480938304CE0101966BE070E042E086
:1045F00050E00E940A6889819A812FEF8F3F9207CD
:1046000079F48CE390E0909382048093810481E8B4
:1046100094E06BE070E042E050E00E94286804C043
:104620009093820480938104CE01019669E070E04A
:1046300042E050E00E940A6889819A812FEF8F3F03
:10464000920779F48AE090E09093800480937F044D
:104650008FE794E069E070E042E050E00E94286853
:1046600004C09093800480937F04CE0101966BE197
:1046700070E042E050E00E940A6889819A812FEF41
:104680008F3F920769F4109211061092100680E194
:1046900096E06BE170E042E050E00E94286804C0C0
:1046A000909311068093100687EA93E260E070E031
:1046B00049E050E00E940A680E94DE0BCE0103969A
:1046C00063E170E044E050E00E940A688B819C81C5
:1046D000AD81BE818F3F2FEF92072FEFA2072FEF03
:1046E000B20749F480EA94E063E170E044E050E00E
:1046F0000E94286808C080EA94E063E170E044E02A
:1047000050E00E940A68CE0103966FE070E044E03A
:1047100050E00E940A688B819C81AD81BE818F3FF1
:104720002FEF92072FEFA2072FEFB20749F48CE982
:1047300094E06FE070E044E050E00E94286808C018
:104740008CE994E06FE070E044E050E00E940A6879
:10475000CE01039667E170E044E050E00E940A68F1
:104760008B819C81AD81BE818F3F2FEF92072FEF10
:10477000A2072FEFB20749F484EA94E067E170E002
:1047800044E050E00E94286808C084EA94E067E1B1
:1047900070E044E050E00E940A6826960FB6F89454
:1047A000DEBF0FBECDBFDF91CF9108956C9A6B9A9B
:1047B0006A9A6F9A729A749A739A779A809880B369
:1047C000897F80BB87E080937E00549A0E94A1225B
:1047D0000E94D12281E00E94720880E090E00E9455
:1047E000F20B0E945C3880917F0486FD239A089525
:1047F000CF93DF93EC0188819981009731F027E016
:104800008B3B920709F073C069C00E94D623809148
:104810007F0480FD02C00E94953F809170008C7FD4
:10482000809370008091B60080628093B6001092F1
:10483000B20082E08093B1008091B60090E0877072
:1048400090700097C9F7809170008160809370002C
:1048500080E090E063EF76E00E94673D0E942C10BC
:1048600080E00E947F110E94FE41809318060E9402
:1048700057408093190600D000D000D0EDB7FEB7A6
:10488000319620E233E0ADB7BEB712963C932E933B
:1048900011978283138280911806848315820E9467
:1048A000D06610921B0610921A068DB79EB7069618
:1048B0000FB6F8949EBF0FBE8DBF85E794E090932E
:1048C000B1238093B02383E290E090931D06809300
:1048D0001C068BEB97E0998388830DC0633259F4F3
:1048E0008AE196E060E070E00E945612E6CF1982FD
:1048F000188283E001C081E0DF91CF910895853671
:10490000910564F1209110063091110620FF10C02E
:1049100000D000D022E333E0EDB7FEB7328321832D
:10492000948383830E94D0660F900F900F900F9016
:1049300080914D1F90914E1FA0914F1FB091501F1D
:104940000196A11DB11D80934D1F90934E1FA09302
:104950004F1FB093501F81E090E0089580E090E0F9
:1049600008954F925F926F927F928F929F92AF9233
:10497000BF92CF92DF92EF92FF920F931F93CF934C
:10498000DF93CDB7DEB7CB57D0400FB6F894DEBF7C
:104990000FBECDBF2C01633851F484E296E0EC9653
:1049A0006FAFEC970E946F2BEC966FADEC97D20136
:1049B0008D919C911197B6E0833C9B07E9F0E6E06E
:1049C000843C9E0718F4009761F0FEC5F7E0883834
:1049D0009F0709F4D2C527E08F38920709F0F4C584
:1049E000E5C584E296E061E870E044EB54E00E94A3
:1049F000542B83EC96E0D5C5623109F0EAC50E94DC
:104A00009809809183049091840492FF02C00E94CF
:104A10001B0E809183049091840493FF0CC00E942C
:104A20004F09DC01CB0180939A2390939B23A093A1
:104A30009C23B0939D238091830480FF60C000D0AD
:104A400000D000D0EDB7FEB7319672E0C72ED12C62
:104A5000CC0EDD1EADB7BEB71296DC92CE9211978A
:104A600088E790E09383828386E493E09583848350
:104A70000E9437678C0187EAA82E83E2B82EEDB733
:104A8000FEB736960FB6F894FEBF0FBEEDBFEE240C
:104A9000FF2498E7892E912C2AE4622E23E0722EBF
:104AA000D5012D915D01EDB7FEB738970FB6F8949B
:104AB000FEBF0FBEEDBF3196C601800F911FADB78F
:104AC000BEB712969C938E931197938282827582C1
:104AD0006482268317820E943767080F191F089483
:104AE000E11CF11CEDB7FEB738960FB6F894FEBF87
:104AF0000FBEEDBFF8E0EF16F10491F602C000E042
:104B000010E08091830490918404009781F12DB787
:104B10003EB7285030400FB6F8943EBF0FBE2DBFB1
:104B2000EDB7FEB73196CE010296800F911FADB75B
:104B3000BEB712969C938E93119788E790E093836B
:104B400082838FE493E09583848380910D06909116
:104B50000E06978386830E943767080F191FEDB7EB
:104B6000FEB738960FB6F894FEBF0FBEEDBF80912A
:104B7000830481FF51C089E290E06BE270E04AE279
:104B800050E027E00E947D3587EA93E20E94E437F7
:104B90002DB73EB72A5030400FB6F8943EBF0FBE37
:104BA0002DBFEDB6FEB60894E11CF11C9E012E5FF0
:104BB0003F4F200F311FADB7BEB712963C932E93D7
:104BC000119728E730E0F7013383228326E533E0AD
:104BD000358324839C01B901882777FD8095982F20
:104BE0000E94E76120E030E048EC52E40E947D61E1
:104BF000DC01CB01F70186839783A087B1870E94F0
:104C00003767080F191F2DB73EB7265F3F4F0FB606
:104C1000F8943EBF0FBE2DBF8091830482FF57C022
:104C200089E290E06BE270E04AE250E026E00E9408
:104C30007D3581E090E00E94EA0980930C068DECBE
:104C400096E10E94E4374DB75EB74A5050400FB628
:104C5000F8945EBF0FBE4DBFEDB6FEB60894E11CE2
:104C6000F11C9E012E5F3F4F200F311FADB7BEB725
:104C700012963C932E93119728E730E0F701338387
:104C8000228320E633E0358324839C01B901882701
:104C900077FD8095982F0E94E76120E030E048EC96
:104CA00052E40E947D61DC01CB01F701868397838A
:104CB000A087B1870E943767080F191F2DB73EB72D
:104CC000265F3F4F0FB6F8943EBF0FBE2DBF8091B9
:104CD000830483FF36C04DB75EB74A5050400FB6CD
:104CE000F8945EBF0FBE4DBFEDB7FEB73196CE0153
:104CF0000296800F911FADB7BEB712969C938E930C
:104D0000119788E790E0938382838BE693E0958305
:104D100084838091C0169091C116A091C216B09163
:104D2000C31686839783A087B1870E943767080FD1
:104D3000191FEDB7FEB73A960FB6F894FEBF0FBE37
:104D4000EDBF8091830484FF32C00E946909AB01EA
:104D5000BC012DB73EB72A5030400FB6F8943EBF85
:104D60000FBE2DBFEDB7FEB73196CE010296800F74
:104D7000911FADB7BEB712969C938E93119788E79B
:104D800090E09383828389E793E0958384834683CD
:104D90005783608771870E943767080F191FEDB727
:104DA000FEB73A960FB6F894FEBF0FBEEDBF8091E6
:104DB000830485FF38C0F894409192235091932347
:104DC000609194237091952378942DB73EB72A5023
:104DD00030400FB6F8943EBF0FBE2DBFEDB7FEB703
:104DE0003196CE010296800F911FADB7BEB71296D5
:104DF0009C938E93119788E790E09383828387E852
:104E000093E09583848346835783608771870E94EC
:104E10003767080F191FEDB7FEB73A960FB6F8942B
:104E2000FEBF0FBEEDBF8091830486FF8DC08091D1
:104E3000810490918204009709F486C0F8948090D0
:104E4000922390909323A0909423B09095237894EC
:104E50008091C5169091C616A091C716B091C8163C
:104E6000A5019401281B390B4A0B5B0BCA01B90140
:104E70000E94E561E62EC72EF82ED92E609181049E
:104E80007091820480E090E00E94E5619B01AC019A
:104E90008E2D9C2DAF2DBD2DBC01CD010E947D61BD
:104EA000E82EC92E4DB75EB74A5050400FB6F89461
:104EB0005EBF0FBE4DBFEDB7FEB73196CE01029675
:104EC000800F911FADB7BEB712969C938E9311972A
:104ED00088E790E09383828380E993E095838483DD
:104EE000862F972FAE2DBC2D86839783A087B18701
:104EF000EC966FAFEC97EB967FAFEB970E9437671E
:104F0000080F191FEC966FADEC97EB967FADEB9702
:104F1000862F972FAE2DBC2D80939F239093A02397
:104F2000A093A123B093A2238092C5169092C61697
:104F3000A092C716B092C816EDB7FEB73A960FB654
:104F4000F894FEBF0FBEEDBF8091830487FF3EC083
:104F5000F8944091962350919723609198237091F3
:104F6000992378942DB73EB72A5030400FB6F89465
:104F70003EBF0FBE2DBFEDB7FEB73196CE010296F4
:104F8000800F911FADB7BEB712969C938E93119769
:104F900088E790E0938382838DE993E0958384830F
:104FA00046835783608771870E943767080F191FF0
:104FB000EDB7FEB73A960FB6F894FEBF0FBEEDBF41
:104FC000C8010E947F24009709F013CD80918304CB
:104FD0009091840490FF8DC080918104909182040F
:104FE000009709F486C0F8948090962390909723B8
:104FF000A0909823B090992378948091C9169091AD
:10500000CA16A091CB16B091CC16A5019401281B0D
:10501000390B4A0B5B0BCA01B9010E94E561E62E10
:10502000C72EF82ED92E609181047091820480E001
:1050300090E00E94E5619B01AC018E2D9C2DAF2D6F
:10504000BD2DBC01CD010E947D61E82EC92E4DB75A
:105050005EB74A5050400FB6F8945EBF0FBE4DBFCA
:10506000EDB7FEB73196CE010296800F911FADB716
:10507000BEB712969C938E93119788E790E0938326
:10508000828386EA93E095838483862F972FAE2DC3
:10509000BC2D86839783A087B187EC966FAFEC9782
:1050A000EB967FAFEB970E943767080F191FEC96BE
:1050B0006FADEC97EB967FADEB97862F972FAE2DCC
:1050C000BC2D8093A3239093A423A093A523B093F6
:1050D000A6238092C9169092CA16A092CB16B092BF
:1050E000CC16EDB7FEB73A960FB6F894FEBF0FBEDA
:1050F000EDBF809183049091840491FF3CC0409166
:105100003D1F50913E1F60913F1F7091401F2DB772
:105110003EB72A5030400FB6F8943EBF0FBE2DBFA9
:10512000EDB7FEB73196CE010296800F911FADB755
:10513000BEB712969C938E93119788E790E0938365
:10514000828383EB93E095838483468357836087D0
:1051500071870E943767080F191FEDB7FEB73A969F
:105160000FB6F894FEBF0FBEEDBFC8010E947F24AA
:10517000009709F03ECC809183049091840492FFC3
:105180003CC02DB73EB72A5030400FB6F8943EBF12
:105190000FBE2DBFEDB7FEB73196CE010296800F40
:1051A000911FADB7BEB712969C938E93119788E767
:1051B00090E0938382838CEB93E09583848380914A
:1051C000391790913A17A0913B17B0913C178683FD
:1051D0009783A087B1870E943767080F191FEDB723
:1051E000FEB73A960FB6F894FEBF0FBEEDBFC801EA
:1051F0000E947F24009709F0FCCB8091830490915A
:10520000840493FF3CC02DB73EB72A5030400FB600
:10521000F8943EBF0FBE2DBFEDB7FEB73196CE015D
:105220000296800F911FADB7BEB712969C938E93D6
:10523000119788E790E09383828387EC93E09583CE
:10524000848380919A2390919B23A0919C23B09179
:105250009D2386839783A087B1870E943767080FB5
:10526000191FEDB7FEB73A960FB6F894FEBF0FBE02
:10527000EDBFC8010E947F24009709F0BACB80914E
:1052800083049091840494FF4CC081E00E94FB0849
:10529000AB01BC012DB73EB72A5030400FB6F89491
:1052A0003EBF0FBE2DBFEDB6FEB60894E11CF11C4B
:1052B000CE010296800F911FADB7BEB712969C9398
:1052C0008E93119788E790E0F7019383828384EDB2
:1052D00093E095838483CB01BA012091A00430919F
:1052E000A1044091A2045091A3040E949762DC01A2
:1052F000CB01F70186839783A087B1870E94376728
:10530000080F191F2DB73EB7265F3F4F0FB6F89411
:105310003EBF0FBE2DBFC8010E947F24009709F039
:1053200068CB809183049091840495FF4BC082E008
:105330000E94FB08AB01BC018DB79EB70A970FB660
:10534000F8949EBF0FBE8DBFEDB6FEB60894E11C6B
:10535000F11CCE010296800F911FADB7BEB7129619
:105360009C938E93119788E790E0F7019383828353
:1053700081EE93E095838483CB01BA0120919C0454
:1053800030919D0440919E0450919F040E94976229
:10539000DC01CB01F70186839783A087B1870E9448
:1053A0003767080F191F2DB73EB7265F3F4F0FB65F
:1053B000F8943EBF0FBE2DBFC8010E947F24009706
:1053C00009F017CB779A809110069091110693FD02
:1053D000749A809110069091110682FD08C0809108
:1053E0007F0480FD04C081FF31C01D9B2FC000D011
:1053F00000D08EEE93E0ADB7BEB712969C938E931D
:105400001197CE01029614969C938E9313970E9447
:10541000D06620919B040F900F900F900F90222345
:10542000A9F000D000D0EDB7FEB731968CE39AE03A
:10543000ADB7BEB712969C938E93119722831382B9
:105440000E94E2660F900F900F900F9080912F06B0
:105450008983FE01E00FF11F128280911006909166
:10546000110680FF12C000D000D085EF93E0EDB7A9
:10547000FEB792838183C8010296948383830E943E
:10548000D0660F900F900F900F9062E0C62ED12C37
:10549000C00ED11ECE010196B6010E9489348091C2
:1054A0007F0482FF49C085E894E0BE016F5F7F4FB3
:1054B000A60122E93FE10E94DE388091100690911A
:1054C000110692FF39C042E9E42E4FE1F42E00E0CC
:1054D00010E056E0A52E54E0B52ED7018D917D0148
:1054E00000D000D0EDB7FEB73196ADB7BEB712967B
:1054F000BC92AE921197828313820E94D0660F5F96
:105500001F4F0F900F900F900F900031110529F74A
:105510008AE090E00E94026700D000D08BE094E027
:10552000EDB7FEB792838183D482C3820E94D06696
:105530000F900F900F900F90809110069091110690
:1055400082FD73980E94A43E84E296E00E94722B32
:1055500080910D0690910E06009711F00E94953FE4
:1055600080912F068F5F80932F0680911006909177
:10557000110682FF3ECA739A3CCA80E396E00E94FD
:10558000F42F009731F10E94A43E80917F0487FDA3
:105590002B9880E396E060E470E00E94C92F8FE8CA
:1055A00097E0D20111969C938E9313C080E396E00E
:1055B0000E94F42F009769F00E94953F80917F042C
:1055C00087FF17CA2B9A15CAF2011182108283E055
:1055D00001C081E0C558DF4F0FB6F894DEBF0FBEA3
:1055E000CDBFDF91CF911F910F91FF90EF90DF9092
:1055F000CF90BF90AF909F908F907F906F905F9073
:105600004F9008950895FC01DB018C9180831196E1
:105610008C91119781830895FC01DB0190818C911D
:10562000981741F421E030E0918111968C91119707
:10563000981711F020E030E0C9010895BC0187EB14
:1056400093E20E94032B0895DC011996ED91FC91E1
:105650001A970280F381E02D309709F0099508959B
:105660000F931F93CF93DF9300D0CDB7DEB78C019C
:1056700088E10E94F834BC01CE0101960E94032B00
:10568000D8011996ED91FC911A970190F081E02DC7
:10569000C801BE016F5F7F4F09950F900F90DF919A
:1056A000CF911F910F910895EF92FF920F931F9347
:1056B000CF93DF93EC018B017A014AEB54E00E9417
:1056C000802BFA86E986C8016EEB74E00E94DE2B1F
:1056D000DF91CF911F910F91FF90EF9008950E945D
:1056E000992B0895CF93DF93EC0188E167EB73E288
:1056F0000E94EE34CE010E949C2BDF91CF91089541
:10570000EF92FF920F931F93CF93DF93EC018B01E6
:105710007A010E94BA2BF886EF82C80162EC74E02D
:105720000E94DE2BDF91CF911F910F91FF90EF90A0
:1057300008950E94C32B08950E940D450895DC0131
:105740001796ED91FC9118970190F081E02D099545
:105750000895DC011796ED91FC9118970280F38172
:10576000E02D309709F00995089588EB9DE00E949F
:105770002D2E0895FC017383628388EB9DE0BF01A9
:105780000E94A02E0895BC0188EB9DE00E946B2E24
:105790000895CF93DF93EC0188EB9DE00E94312EBA
:1057A00008C0FC01228133812C173D0721F00E94A3
:1057B000D72E0097B1F7DF91CF9108950F931F93E4
:1057C000CF93DF938B010E94C92BEC01009731F03E
:1057D0001D830C83C8010E9450478E83DF91CF91B7
:1057E0001F910F9108951F93CF93DF93EC01162F14
:1057F000888580FF1DC0EC81FD813097C9F0D09372
:10580000BB0DC093BA0D82E08887CE01069609953C
:10581000992787FD909502978230910510F01338F3
:1058200029F4CE01BE010E941C2C02C081E08887B1
:10583000DF91CF911F910895CF92DF92EF92FF9267
:105840000F931F93CF93DF93EC017B01C090BA0DB0
:10585000D090BB0D0091BC0D1091BD0DF80103C09F
:105860000190F081E02DEC17FD0719F03097C1F79A
:1058700046C0209709F443C08885882309F118861B
:105880000BC0C017D10729F0C80167E8AE010E941C
:10589000F32BF801008111810115110591F7EC81BD
:1058A000FD81309769F0CE15DF0551F0D093BB0D27
:1058B000C093BA0DCE01069663E840E050E009952A
:1058C000E091BC0DF091BD0DCE17DF0791F48881FA
:1058D00099819093BD0D8093BC0D0DC08081918105
:1058E0008C179D0729F4888199819183808303C057
:1058F000FC01309799F7D092BB0DC092BA0DDF91A1
:10590000CF911F910F91FF90EF90DF90CF9008956E
:105910001F93CF93DF931092BE0DC091BC0DD09119
:10592000BD0D11E00EC08985882341F018871986C6
:10593000CE0162E840E050E00E94F32B0990D8814C
:10594000C02D209781F7DF91CF911F91089580910D
:10595000BF0D982F9F5F9093BF0D08956091BA0D72
:105960007091BB0D0E941C2C08958AE88093BF0D96
:105970001092C00D1092C10D1092BD0D1092BC0D71
:105980001092BB0D1092BA0D08958091BE0D882320
:1059900011F00E94882C7091C10D772309F455C035
:1059A0002091C00D30E0F901EE0FFF1FEE0FFF1F39
:1059B000E20FF31FEE53F24F60816093620E41815C
:1059C00052815093640E4093630E8381948190932F
:1059D000660E8093650E2F5F3F4F2F7130702093BE
:1059E000C00D71507093C10D009741F58091BC0DB1
:1059F0009091BD0D18C08091BE0D882311F00E94BA
:105A0000882C4091630E5091640E8091670E9091A6
:105A1000680E6091620E0E94F32BE091670EF09188
:105A2000680E808191819093680E8093670E8091BB
:105A3000670E9091680E0097F1F607C0613819F46F
:105A400021E0FC0120870E94F32B8091BE0D209164
:105A5000C10D90E0820F911D08958091BE0D20919F
:105A6000C10D90E0820F911D08959C017091C10DB0
:105A70007032D9F08091C00D870F8F718093690EBD
:105A800090E0FC01EE0FFF1FEE0FFF1FE80FF91F64
:105A9000EE53F24F608352834183348323837F5FCD
:105AA0007093C10D80E090E0089581E090E008954A
:105AB000CF93DF93C091BA0DD091BB0D0E94F32B11
:105AC000D093BB0DC093BA0DDF91CF910895FC0127
:105AD000AB019091BC0D8091BD0DA92FB82F03C0D3
:105AE0000D90BC91A02DAE17BF0791F01097C1F794
:105AF000309771F090838183F093BD0DE093BC0DDE
:105B000081E0808717821682CF0161E80E94582DBC
:105B10000895FC01009741F080858150823020F487
:105B200081E081878093BE0D089521E030E0FC0183
:105B30008085882311F420E030E0C9010895CF93D7
:105B4000DF93EC014A815B818C819D8160E070E094
:105B50000E945A662A813B8188819981289FA001F1
:105B6000299F500D389F500D11248E819F8160E038
:105B700070E00E945A66DF91CF910895DC01129681
:105B80002D913C91139780E090E01DC01496ED910B
:105B9000FC911597E80FF91F4081442399F421E007
:105BA00020832D913C911197829FA001839F500DDE
:105BB000929F500D112416968D919C911797840FEA
:105BC000951F089501968217930701F780E090E0F2
:105BD0000895FC0146815781A281B38120E030E025
:105BE00019C04617570781F4A481B581A20FB31FCE
:105BF0008C91181614F481508C930480F581E02D5B
:105C0000E20FF31F8081089580819181480F591F11
:105C10002F5F3F4F2A173B0721F78FEF0895FC01B5
:105C20004681578164177507A8F0A081B1818281F0
:105C30009381A89F9001A99F300DB89F300D11242A
:105C4000240F351F81E090E06217730728F080E091
:105C500090E0089580E090E00895FC0111821082A8
:105C60000895FC01808191810895FB01208131819B
:105C7000FC01318320830895FC018081918100978C
:105C800011F40895C901FC012081318121153105EC
:105C9000C9F70895DC01ED91FC911197309729F433
:105CA0000BC0DF010190F081E02D80819181009790
:105CB000C1F711961C921E92CF010895DC01ED915F
:105CC000FC911197309729F08081918111969C93D6
:105CD0008E93CF010895CF93DF93EC01E881F98192
:105CE0003097B9F0A0E0B0E002C0DF01FC01808194
:105CF0009181E617F70759F4109719F4998388836F
:105D000003C011969C938E931182108202C000975B
:105D100061F7DF91CF9108950F931F93CF93DF9396
:105D20008C01EB010E946B2EF80180819181998397
:105D30008883D183C083DF91CF911F910F91089504
:105D40000F931F93CF93DF938C01EB010E946B2E77
:105D500019821882C8010E943C2E009711F4F801A4
:105D600001C0FC01D183C083DF91CF911F910F91BE
:105D70000895DC01ED91FC91119780E090E004C062
:105D800001960190F081E02D3097D1F70895FB0145
:105D9000BA01309719F40E948C2E08958081918168
:105DA000DA0111969C938E93518340830895009756
:105DB00021F0FC0180819181089580E090E00895B8
:105DC00080916A0E90916B0E009729F410926D0EDF
:105DD00010926C0E08950E94153CBC01E0916A0E71
:105DE000F0916B0E4281538180819181480F591F40
:105DF000461B570B0CC08281938120813181820F19
:105E0000931F861B970B8417950708F4AC01048039
:105E1000F581E02D309779F7460F571F50936D0E9F
:105E200040936C0E089580ED94E00E94892D0895B2
:105E3000EF92FF920F931F93CF93DF937C01FC01AE
:105E400080819181009729F08A35910509F06DC014
:105E50000BC010926B0E10926A0E8AE590E0F7016B
:105E60009183808381E065C0673859F5A0916A0EFF
:105E7000B0916B0E04C014960D90BC91A02D10979C
:105E800041F316968D919C9117978417950799F376
:105E9000A0936A0EB0936B0E0DC086819781841714
:105EA000950739F48481958115969C938E93149768
:105EB000FD01DF011496ED91FC911597309769F77C
:105EC000CCCF623851F6C0916A0ED0916B0E00E0D3
:105ED00010E028C0CE010E94354B0097F1F08E8172
:105EE0009F8168E8AE010E94352D0097A1F41F82C2
:105EF0001E828C819D810115110521F0F801958389
:105F0000848304C090936B0E80936A0E1D821C8262
:105F10000E94E02ED8CF0E94132F9C818D818E018C
:105F2000C92FD82F2097B1F698CFF7011182108290
:105F300083E0DF91CF911F910F91FF90EF90089533
:105F4000CF93DF93EC010E94132F8E819F813091BC
:105F50006A0E20916B0E009759F0E32FF22F06C0C6
:105F6000EC17FD0789F00480F581E02D3097C1F72B
:105F70008091BA0D9091BB0D9F838E833C832D83BE
:105F8000D0936B0EC0936A0E0E94E02EDF91CF91EA
:105F90000895CF93DF93EC010E94154BCE010E9430
:105FA000A02FDF91CF910895CF93DF93EC010E9452
:105FB000214BCE010E94A02FDF91CF910895CF9366
:105FC000DF93EC010E942B4BCE010E94A02FDF91AA
:105FD000CF910895FC0180819181860F971F918355
:105FE00080830E94E02E089521E030E0FC0186814C
:105FF0009781009711F020E030E0C9010895FC017D
:106000002281338180819181280F391FC901089530
:10601000FC0180819181089581E090E020916A0ED9
:1060200030916B0E2115310511F480E090E0089558
:1060300080916A0E90916B0E009729F080916C0E02
:1060400090916D0E089580E090E00895CF93DF93D6
:10605000EC01E0916A0EF0916B0E8E179F0741F4F0
:106060008C819D8190936B0E80936A0E14C0FC010D
:10607000309731F0848195818C179D07C1F707C057
:106080001D821C821F821E82DF91CF9108958C8118
:106090009D81958384830E94E02EF2CFEF92FF9240
:1060A0000F931F93CF93DF937C018A01FC018081C2
:1060B0009181009729F08B34910509F049C01AC0ED
:1060C0008FE69EE00E94312EEC0109C06C817D813B
:1060D000CE0102960E94C92F0990D881C02D209729
:1060E000A9F781E080936E0E8BE490E0F701918335
:1060F000808333C0683889F58FE69EE00E94312E98
:10610000EC0123C0CE01029608171907D9F48FE6D7
:106110009EE0BE010E946B2E0091BA0D1091BB0D46
:106120008A859B859093BB0D8093BA0DEC85FD8588
:10613000309719F08E859F8509951093BB0D0093BC
:10614000BA0DD2CF0990D881C02D2097D9F6CCCFE7
:10615000F7011182108283E001C081E0DF91CF91CD
:106160001F910F91FF90EF90089510926E0E8FE6A1
:106170009EE00E942D2E89EE94E060E070E00E9487
:10618000672D08950F931F93CF93DF93EC01009138
:10619000BA0D1091BB0D1B870A875D874C873F871F
:1061A0002E8780916E0E882379F089EE94E090938B
:1061B000BB0D8093BA0DCE0102960E94C92F109399
:1061C000BB0D0093BA0D02C07D836C838FE69EE009
:1061D000BE010E946B2E8FE69EE0BE010E94A02EA3
:1061E000DF91CF911F910F9108950F931F93CF933C
:1061F000DF93EC0180916E0E882391F00091BA0D2F
:106200001091BB0D89EE94E09093BB0D8093BA0D75
:10621000CE0102960E94D42F1093BB0D0093BA0DAD
:106220008FE69EE0BE010E946B2E8FE69EE0BE01CF
:106230000E94A02EDF91CF911F910F9108950F938F
:106240001F93CF93DF93EC0180916E0E882391F022
:106250000091BA0D1091BB0D89EE94E09093BB0DA7
:106260008093BA0DCE0102960E94DF2F1093BB0DD2
:106270000093BA0D8FE69EE0BE010E946B2E8FE662
:106280009EE0BE010E94A02EDF91CF911F910F9141
:106290000895CF93DF93EC0180916E0E882329F04F
:1062A000CE0102960E94263004C01F821E821986EB
:1062B00018868FE69EE0BE010E946B2EDF91CF9183
:1062C0000895CF93DF93EC0180916E0E882329F01F
:1062D000CE0102960E94F42F12C08FE69EE00E942B
:1062E000312E06C08C179D0741F0FC018081918101
:1062F0000097C1F781E090E002C080E090E0DF917C
:10630000CF910895CF93DF93D091B723C091B82355
:106310000E94413CAB01BC018DB79EB782559040B5
:106320000FB6F8949EBF0FBE8DBFEDB7FEB7319686
:1063300082E49AE0ADB7BEB712969C938E93119704
:10634000D2831382C4831582468357836087718703
:106350008091AA259091AB25A091AC25B091AD2557
:1063600082879387A487B5878091AE259091AF25CA
:10637000A091B025B091B12586879787A08BB18B6E
:106380008091B2259091B325A091B425B091B52507
:10639000828B938BA48BB58B8091B6259091B7257A
:1063A000A091B825B091B925868B978BA08FB18F1E
:1063B0008091BA259091BB25A091BC25B091BD25B7
:1063C000828F938FA48FB58F8091BE259091BF252A
:1063D000A091C025B091C125868F978FA0A3B1A3AE
:1063E0008091C2259091C325A091C425B091C52567
:1063F00082A393A3A4A3B5A38091C6259091C7259A
:10640000A091C825B091C92586A397A3A0A7B1A73D
:106410008091CA259091CB25A091CC25B091CD2516
:1064200082A793A7A4A7B5A78091CE259091CF2549
:10643000A091D025B091D12586A797A7A0ABB1ABED
:106440008091D2259091D325A091D425B091D525C6
:1064500082AB93ABA4ABB5AB8091D6259091D725F9
:10646000A091D825B091D92586AB97ABA0AFB1AF9D
:106470008091DA259091DB25A091DC25B091DD2576
:1064800082AF93AFA4AFB5AFEDB7FEB7FF968091E3
:10649000DE259091DF25A091E025B091E125808354
:1064A0009183A283B383EDB7FEB7ED5BFF4F80917D
:1064B000E2259091E325A091E425B091E525808324
:1064C0009183A283B383EDB7FEB7E95BFF4F809161
:1064D000E6259091E725A091E825B091E9258083F4
:1064E0009183A283B383EDB7FEB7E55BFF4F809145
:1064F000EA259091EB25A091EC25B091ED258083C4
:106500009183A283B383EDB7FEB7E15BFF4F809128
:10651000EE259091EF25A091F025B091F125808393
:106520009183A283B3830E94E266D091B723C09186
:10653000B8238DB79EB78E5A9F4F0FB6F8949EBF63
:106540000FBE8DBF0E94413CAB01BC01ADB7BEB7D1
:10655000D2970FB6F894BEBF0FBEADBFEDB7FEB772
:1065600031968EE19BE012969C938E931197D28385
:106570001382C48315824683578360877187809115
:10658000F2259091F325A091F425B091F52582870D
:106590009387A487B5878091F6259091F725A091E0
:1065A000F825B091F92586879787A08BB18B8091CC
:1065B000FA259091FB25A091FC25B091FD25828BB9
:1065C000938BA48BB58B8091FE259091FF25A09194
:1065D0000026B0910126868B978BA08FB18F80917A
:1065E000022690910326A0910426B0910526828F61
:1065F000938FA48FB58F8091062690910726A09146
:106600000826B0910926868F978FA0A3B1A3809109
:106610000A2690910B26A0910C26B0910D2682A3FC
:1066200093A3A4A3B5A380910E2690910F26A091C9
:106630001026B091112686A397A3A0A7B1A7809199
:106640001A2690911B26A0911C26B0911D2682A788
:1066500093A7A4A7B5A780911E2690911F26A0916D
:106660002026B091212686A797A7A0ABB1AB0E94A8
:10667000E2668DB79EB7C2960FB6F8949EBF0FBE66
:106680008DBFDF91CF91089580E38093750E0895BB
:10669000CF93DF936091750E70E0C0E3D0E0C61B2E
:1066A000D70B6858714FAE010E945166CE01DF9141
:1066B000CF910895CF92DF92EF92FF920F931F93A5
:1066C000CF93DF937C01C090730ED090740E6091D5
:1066D000750E70E08601005D1F4F061B170B013819
:1066E0001105D8F4C0E3D0E0C61BD70B6858714F32
:1066F000AE010E945166C7018C0F9D1F6091760EFE
:106700007091770E2091710E3091720E620F731F8F
:10671000A6010E945166C80102C080E090E0DF91AE
:10672000CF911F910F91FF90EF90DF90CF90089540
:106730009091750E980F9093750E08954091730E79
:106740005091740E9C014817590798F08091710E72
:106750009091720E820F931F9093720E8093710E20
:10676000421B530B5093740E4093730E81E090E0E4
:10677000089580E090E008959093740E8093730ED6
:1067800008958091710E9091720E8855914F0895E1
:106790008091750E90E08858914F089581E090E0C7
:1067A0002091760E3091770E4EE0283A340711F49E
:1067B00080E090E008950E94CE33009769F088EA67
:1067C0009EE06091760E7091770E4091730E50911D
:1067D000740E0E94516608954091710E5091720E90
:1067E00041155105C1F08091730E9091740EC096C1
:1067F000A8EABEE020E330E007C0FD01E40FF51F8A
:1068000060816D932F5F3F4F28173907B4F31092C3
:10681000720E1092710E08958091760E9091770EFF
:1068200008958091730E9091740E08959091750E55
:1068300080E3891B089520E38091750E281B8091C9
:10684000730E9091740E820F911D08951F93CF9334
:10685000DF93EC011091750E812F90E08C179D074E
:106860006CF00E941B348C0F9D1F8138910530F411
:106870001C1B1093750E81E090E002C080E090E058
:10688000DF91CF911F910895CF93DF93E1ECF3E275
:106890001192119283E2E13FF807D1F7C0E0D0E016
:1068A000CE01880F991F87549C4D68EB74E00E94BD
:1068B000032B2196C430D10599F7DF91CF9108952C
:1068C0001092720E1092710E1092740E1092730E3E
:1068D00080E38093750E88EA9EE09093770E809314
:1068E000760E0E94443408950F931F93CF93DF9345
:1068F000EC018B010E946034D093770EC093760E2A
:106900001093740E0093730EDF91CF911F910F912E
:106910000895EF92FF920F931F93CF93DF9300D0D0
:10692000CDB7DEB78C0169837A830E9460346981B8
:10693000E62E7A81F72E81E8E816F10418F030E8A7
:10694000E32EF12C8091760E9091770EB801A7017D
:106950000E945166F092740EE092730EC7010F9080
:106960000F90DF91CF911F910F91FF90EF900895BD
:10697000FC01A1ECB3E280E30D9001928150E1F7BC
:10698000FB01A9EBB3E288E00D9001928150E1F7A1
:106990000895A1ECB3E2FC0180E301900D928150D7
:1069A000E1F7A9EBB3E2FB0188E001900D92815081
:1069B000E1F70895E82FF0E0EE0FFF1FEF53FC4DD5
:1069C0007183608381E090E00895E82FF0E0EE0F9E
:1069D000FF1FEF53FC4D80819181089590E0880F57
:1069E000991F87579C4D0E94032B81E090E00895EA
:1069F00090E0880F991F87579C4D08958115910548
:106A000011F00197F1F70895E091F423F091F52347
:106A100090818091F32389230895E091F123F091EF
:106A2000F22380819091F323892B8083E091F623D8
:106A3000F091F72380819091F323892B808308952F
:106A4000E091F123F091F22390818091F3238095DE
:106A500089238083E091F623F091F7239081809140
:106A6000F32380958923808308951F93CF93DF9329
:106A7000E091F123F091F22390818091F3238095AE
:106A800089238083E091F623F091F7238081909110
:106A9000F323892B80838FEB93E00E94FE341FB792
:106AA000F894E091F623F091F72390818091F323FD
:106AB00080958923808383E890E00E94FE34E091F2
:106AC000F423F091F523D081C091F3231FBF789474
:106AD0008BE393E00E94FE34E091F423F091F523E0
:106AE00080819091F323892319F08D2F8C2301C08D
:106AF00081E0DF91CF911F9108955093F723409348
:106B0000F6237093F2236093F1239093F5238093FF
:106B1000F42381E090E002C0880F991F2A95E2F7E4
:106B20008093F3230E9435350895CF93DF93C82FC8
:106B3000DFB7F894E091F623F091F72380819091EC
:106B4000F323892B808383E090E00E94FE34CC23E2
:106B500051F0E091F623F091F72390818091F32397
:106B600080958923808387E190E00E94FE34E09144
:106B7000F423F091F52380819091F323892309F484
:106B8000C0E089E590E00E94FE34E091F623F091A8
:106B9000F72390818091F323809589238083DFBF41
:106BA0008BE390E00E94FE348C2FDF91CF9108950B
:106BB000CF93DF93C82FD8E08C2F81700E9495353A
:106BC000C6958111C068D150B9F78C2FDF91CF9154
:106BD00008958FEF0E94D8350895DF92EF92FF92CB
:106BE0000F931F93CF93DF93182FEB010E9435353E
:106BF000882381F580EF0E94D835EE2400E498E0E8
:106C0000D92E81E00E949535F82E81E00E949535BD
:106C1000882319F0FF2069F020C0FF2051F40117EC
:106C200028F0888180FF05C0101719F0E02EFF249E
:106C3000F3948F2D0E949535888186958883FF2057
:106C400011F0806888830150DA94D9F621960023E8
:106C5000B1F605C0EE24EA9402C08EEFE82E8E2D28
:106C6000DF91CF911F910F91FF90EF90DF900895EA
:106C70000F931F93CF93DF93182FEB010E943535AD
:106C8000209751F085E50E94D83508E089910E944F
:106C9000D8350150D9F703C08CEC0E94D835812F2C
:106CA0000E94D835DF91CF911F910F9108950F93D6
:106CB0001F93CF93DF93E82FDB01EA01B9014C91D9
:106CC00050E011969C91119780E0482B592BE031B0
:106CD00081F4CA018E7F33E0880F991F3A95E1F75E
:106CE00016962C9116974CE050E0421B5109480F24
:106CF000591F57FF06C081E08883509541955F4F2B
:106D000001C01882E83299F414968C91149790E09F
:106D10009C01207630702036310549F086FF02C094
:106D20004E7F05C085FF02C04C7F01C0487FCA016D
:106D300024E0969587952A95E1F7FB0180834F70B3
:106D4000F801408380E0DF91CF911F910F9108956A
:106D50000F931F93CF93DF93EC018B018881B801D0
:106D60000E94ED35888381508D3F30F4F801808199
:106D7000883211F0803191F7DF91CF911F910F91FF
:106D80000895CF93DF93EC010E94353584EBBE016B
:106D90000E94383681E00E949535C82F0E94353513
:106DA00081E0CC2309F480E0DF91CF9108951F9317
:106DB000CF93DF93182FEB010E9435350E940435E5
:106DC000882349F084E4BE010E943836113029F04E
:106DD0000E940D3502C082E001C080E0DF91CF91BA
:106DE0001F9108956F927F928F929F92BF92CF9240
:106DF000DF92EF92FF920F931F93CF93DF93CDB764
:106E0000DEB729970FB6F894DEBF0FBECDBF7C0169
:106E10004B013A0169010E9435358EEBB7010E94A2
:106E200038368E010F5F1F4FE9E0BE2E0E94E93514
:106E3000F80181938F01BA94C9F7CE01019669E0F8
:106E400070E00E94CF4F882361F4F7018081BE017A
:106E50006F5F7F4FA401930186010E94573680E047
:106E600001C083E029960FB6F894DEBF0FBECDBFF8
:106E7000DF91CF911F910F91FF90EF90DF90CF9016
:106E8000BF909F908F907F906F9008958F929F9268
:106E9000AF92BF92CF92DF92EF92FF920F931F9328
:106EA000CF93DF93CDB7DEB729970FB6F894DEBF47
:106EB0000FBECDBFD82E5B014A0179018EEB60E099
:106EC00070E00E9438368E010F5F1F4FF9E0CF2E21
:106ED0000E94E935F80181938F01CA94C9F7CE0168
:106EE000019669E070E00E94CF4F882359F48D2D00
:106EF000BE016F5F7F4FA501940187010E94573645
:106F000080E001C083E029960FB6F894DEBF0FBE83
:106F1000CDBFDF91CF911F910F91FF90EF90DF9048
:106F2000CF90BF90AF909F908F900895EF92FF9277
:106F30001F93CF93DF93CDB7DEB728970FB6F894A2
:106F4000DEBF0FBECDBF182F262FDE011196E3EF57
:106F5000F4E088E001900D928150E1F7E42EFF24E7
:106F6000E7FCF09441E752E0E49EC001E59E900DFD
:106F7000F49E900D112464E670E00E942D63CB0115
:106F800034E6239F90011124820F931FFE01319656
:106F900040E0219130E0E216F30611F4019603C0BF
:106FA0004F5F4830B1F7112319F0909581959F4FAD
:106FB00028960FB6F894DEBF0FBECDBFDF91CF91FC
:106FC0001F91FF90EF9008950F931F93CF93DF933E
:106FD000CDB7DEB72B970FB6F894DEBF0FBECDBF8F
:106FE000182F092F885F612F792F0E94D7368823A9
:106FF00009F048C066E471E48FE090E00E944F38E9
:10700000812F902FBE016D5F7F4FAE014E5F5F4FAE
:107010009E012F5F3F4F0E94F236882399F5DE01D3
:107020001496E3EFF4E088E001900D928150E1F7CF
:10703000E9814E2F50E021E732E0429FC001439F9B
:10704000900D529F900D112464E670E00E942D6314
:10705000CB013A8124E6329F90011124820F931FC5
:10706000DE01149620E03D91E31711F4019603C070
:107070002F5F2830C1F72B81222331F09095819525
:107080009F4F02C084E391E22B960FB6F894DEBFC7
:107090000FBECDBFDF91CF911F910F910895DC01FD
:1070A000CB0181159105A105B10529F081509040D2
:1070B000A040B040D9F708951092B90080E28093C3
:1070C000B800089594EA9093BC009091BC0097FF9B
:1070D000FCCF9091B900987F983011F0903199F4DD
:1070E0008093BB0084E88093BC008091BC0087FF44
:1070F000FCCF9091B900987F983139F081E09034BD
:1071000029F480E0089581E0089580E0089544EA3C
:1071100034E824E94093BC009091BC0097FFFCCF79
:107120009091B900987F983011F0903199F7809341
:10713000BB003093BC009091BC0097FFFCCF9091B6
:10714000B900987F903211F0983539F42093BC0043
:107150009091BC0094FDFCCFDDCF08950E94623871
:10716000089584E98093BC008091BC0084FDFCCF2D
:1071700008958093BB0084E88093BC008091BC009C
:1071800087FFFCCF9091B900987F81E0983209F495
:1071900080E0089584EC8093BC008091BC0087FF60
:1071A000FCCF8091BB00089584E88093BC0080915F
:1071B000BC0087FFFCCF8091BB000895FC0180E1FB
:1071C000919190933F018150D9F780913C018F7D3F
:1071D00080933C0180913C01877F80933C01FB01BF
:1071E00080E1919190933E018150D9F780913C01CB
:1071F000806880933C0180913D0180FFFCCF40512D
:10720000504080913C01806280933C0180913C0120
:10721000877F80933C0112C0FB0180E191919093A4
:107220003E018150D9F780913C01806880933C01F8
:1072300080913D0180FFFCCF40515040141615064F
:107240005CF3F90180E190913E0191938150D9F76F
:1072500081E090E00895E6E4F1E080812081908172
:107260003081829586958695837022952F70822B2A
:10727000832B92959F70892B0895DF92EF92FF9256
:107280000F931F93CF93DF9300D0CDB7DEB780E08D
:107290006CE046E00E94D93C89E18093C4001092E2
:1072A000C50082E08093C00080E00E947B3D0E9488
:1072B000053C84B784B784B784B784B7E8E7FCE2B9
:1072C00022E432E4318320833A968DB79EB70A9741
:1072D000E817F907B8F300D000D08DE89BE0ADB710
:1072E000BEB712969C938E9311978BEF94E01496F1
:1072F0009C938E9313970E94E2660F900F900F90CD
:107300000F900E94004C0E94B52C80ED94E060E04C
:1073100070E00E94672D0E94B530E0914605F09123
:10732000470509950E942B3990E00E943D4CCE0103
:1073300001960E94373B882359F000D088EA9BE0F1
:10734000EDB7FEB7928381830E94E2660F900F90A3
:10735000CE0101960E941E2B0E94413B8C010E948F
:10736000463BBC01C801AE014F5F5F4F0E947540B4
:107370000E94A43A0E945A400E944B3B0E94F64150
:1073800000D088EC9BE0ADB7BEB712969C938E936D
:1073900011970E94E26600D0EDB7FEB7319605ED79
:1073A0001BE0ADB7BEB712961C930E9311978A815E
:1073B000828313820E94E266EDB7FEB73196ADB7C5
:1073C000BEB712961C930E93119789818283138204
:1073D0000E94E2660F900F9089ED9BE0EDB7FEB73B
:1073E000928381830E94E2660F900F900E94434C2B
:1073F000E091C905F091CA050995E091B005F091B9
:10740000B1050995E0917205F09173050995009118
:10741000AE051091AF05E090C705F090C8050E9439
:107420005740D82E0E94FE412DB73EB72A5030401B
:107430000FB6F8943EBF0FBE2DBFEDB7FEB7319625
:107440002BED3BE0ADB7BEB712963C932E93119750
:1074500013830283F582E482D682178280871186A5
:107460000E94E266E091D305F091D4052DB73EB7B6
:10747000265F3F4F0FB6F8943EBF0FBE2DBF30972B
:10748000D1F00995BC0100D000D086EF9BE0ADB7EC
:10749000BEB712969C938E93119780E890E00E945D
:1074A0001963EDB7FEB7748363830E94E2660F90A1
:1074B0000F900F900F9000D089E09CE0ADB7BEB761
:1074C00012969C938E9311970E94E2660F900F90F4
:1074D00082EF95E060E070E00E94672D83E194E028
:1074E0000E94F94A00D08BE09CE0EDB7FEB7928392
:1074F00081830E94E2660F900F900F900F90DF91B2
:10750000CF911F910F91FF90EF90DF90089500D0E1
:1075100000D000D0EDB7FEB7319623E13CE0ADB727
:10752000BEB712963C932E931197938382837583F3
:1075300064830E94E2668DB79EB706960FB6F894F4
:107540009EBF0FBE8DBF08950F931F93CF93DF9300
:10755000CDB7DEB7A0970FB6F894DEBF0FBECDBF94
:1075600082E290E00E942268082F282F2B502031C1
:1075700008F0982F9095891709F46DC000D089E321
:107580009CE0ADB7BEB712969C938E9311970E9464
:10759000E2668E010F5F1F4F0F900F90D80180E0C1
:1075A00090E0FC01EF5CF34FE491ED93019688309D
:1075B0009105B9F7F894CE0101966EE370E048E0CA
:1075C00050E00E942868D80180E090E0FC01ED5D69
:1075D000F34FE491ED9301968E309105B9F7CE010A
:1075E000019660E370E04EE050E00E94286880E081
:1075F00090E0FC01E75EF34FE491D801ED938D013B
:1076000001968A309105A9F7CE01019666E270E0F5
:107610004AE050E00E94286880E290E06DEC7BEA4E
:107620000E9440688EE190E060E070E00E94406857
:107630008DE190E060E00E94326884E290E060E0DA
:1076400070E00E9440680AE182E290E06AE175EE33
:107650000E9440687894802FA0960FB6F894DEBF01
:107660000FBECDBFDF91CF911F910F910895F89478
:107670006EE370E042E050E00E940A68789480E097
:10768000089580E290E00E94226808958EE190E0E3
:107690000E94226808958DE190E00E941A68089582
:1076A0004091062450910724609108247091092488
:1076B00090E0A0E0B0E0480F591F6A1F7B1F409385
:1076C0000624509307246093082470930924409162
:1076D0000224509103246091042470910524480FE2
:1076E000591F6A1F7B1F4093022450930324609309
:1076F0000424709305242091A6252223A1F0409113
:10770000FE235091FF236091002470910124480FC3
:10771000591F6A1F7B1F4093FE235093FF236093E2
:1077200000247093012408951F920F920FB60F92B8
:107730000BB60F9211242F933F934F935F936F9348
:107740007F938F939F93AF93BF93EF93FF9380911A
:107750002C0F90912D0F019690932D0F80932C0F4D
:1077600080912B0F8F5F80932B0F8038A9F410929C
:107770002B0F8091062490910724A0910824B091AA
:1077800009240196A11DB11D80930624909307241E
:10779000A0930824B09309248091A6258823E1F0C2
:1077A00080912A0F8F5F80932A0F8038A9F410925E
:1077B0002A0F8091FE239091FF23A0910024B09185
:1077C00001240196A11DB11D8093FE239093FF23F8
:1077D000A0930024B09301240E940C30009711F074
:1077E0000E94132FFF91EF91BF91AF919F918F91C5
:1077F0007F916F915F914F913F912F910F900BBEB1
:107800000F900FBE0F901F901895F8941092B6002D
:1078100016BC83EF87BD82E084BD94E095BD95B32F
:1078200095BB80936E007894089580912C0F909171
:107830002D0F20912C0F30912D0F82179307A9F750
:10784000089507C022E330E0000021503040E1F706
:1078500001970097B9F708950F931F93CF93DF9384
:107860008C010E94153CEC010E94153C8C1B9D0B69
:1078700080179107C8F3DF91CF911F910F91089561
:1078800008950F931F9300910624109107242091CF
:107890000824309109248091062490910724A09116
:1078A0000824B0910924081719072A073B0759F73C
:1078B000B801C9011F910F9108951F920F920FB641
:1078C0000F921124109211050F900FBE0F901F9070
:1078D00018951F920F920FB60F920BB60F921124AC
:1078E0002F933F934F935F936F937F938F939F93C8
:1078F000AF93BF93EF93FF93E0910705F0910805D5
:107900008081E0911205F0911305309709F00995F7
:10791000FF91EF91BF91AF919F918F917F916F9167
:107920005F914F913F912F910F900BBE0F900FBE23
:107930000F901F9018951F920F920FB60F9211245F
:1079400010921E050F900FBE0F901F9018951F925A
:107950000F920FB60F920BB60F9211242F933F93F5
:107960004F935F936F937F938F939F93AF93BF9347
:10797000EF93FF93E0911405F09115058081E0915C
:107980001F05F0912005309709F00995FF91EF91BF
:10799000BF91AF919F918F917F916F915F914F9127
:1079A0003F912F910F900BBE0F900FBE0F901F9025
:1079B000189590E02DE030E0829FF001839FF00D5C
:1079C000929FF00D1124E95FFA4FA281B3811C92BE
:1079D000A481B5816C93A681B78188ED8C93A08535
:1079E000B1854C93128614861386089590E02DE09D
:1079F00030E0829FF001839FF00D929FF00D1124E3
:107A0000E95FFA4F81E08287A081B1816C933A9659
:107A100080818823E9F70895CF93C82F8A3031F405
:107A200080916E0F6DE00E94F63C02C08D3029F00F
:107A300080916E0F6C2F0E94F63C80E090E0CF9119
:107A400008951F93CF93DF93182FEB010CC08A305A
:107A500021F4812F6DE00E94F63C69916D3019F0A0
:107A6000812F0E94F63C8881882389F7DF91CF918E
:107A70001F9108950F931F93CF93DF93CDB7DEB778
:107A80009E01265F3F4F0EE21FE0C80160E470E0F8
:107A9000488559850E9474678F81B8010E94213DF5
:107AA000DF91CF911F910F9108951F93CF93DF9393
:107AB000182FEB0104C0812F0E94F63C2196FE0195
:107AC00064916623C1F7DF91CF911F91089590E0F3
:107AD0002DE030E0829FF001839FF00D929FF00D2A
:107AE0001124E95FFA4F748763870895682F80E057
:107AF0000E94F63C089580936E0F81E295E090938A
:107B0000732C8093722C089584B7877F84BF88E19B
:107B10000FB6F89480936000109260000FBE089535
:107B20002FE088E190E00FB6F894A895809360006C
:107B30000FBE209360000895A895089588E10FB6C0
:107B4000F89480936000109260000FBE0895F8943E
:107B500028E088E190E00FB6F894A8958093600043
:107B60000FBE20936000FFCF8091112480911124DB
:107B700090E008958091390181FD10C081E491E089
:107B80006FE140E00E949543813059F021E030E000
:107B9000813111F020E030E0C901089580E090E0EB
:107BA000089581E090E0089581E491E06FE140E084
:107BB0000E9495430895E9E3F1E0808180818D7F03
:107BC00080838DE090E00197F1F782E491E06FE12E
:107BD00040E023E00E949F4383E090E00197F1F7AB
:107BE00008959091390191FD0AC0282F803108F045
:107BF0002FE085E491E06FE040E00E949F4308950C
:107C00008091390181FD13C081E491E06FE140E092
:107C10000E949543982F8151823038F09F3129F08E
:107C2000913019F081E0923019F480E0089581E0FC
:107C300008950E94003E8823E1F30895CF93DF93D7
:107C4000C82F883049F0863039F0893029F08631E4
:107C500019F0893109F045C08091390181FD44C096
:107C60000E94193E0E94D43DD82FC817B9F1C830E0
:107C700019F40E94DB3D2BC0C93141F48631A9F4CF
:107C800082E491E06FE140E029E009C0C63169F487
:107C9000893159F482E491E06FE140E026E00E94EE
:107CA0009F43E3E0F0E03197F1F782E491E06FE188
:107CB00040E02C2F0E949F43D83029F489E691E0C0
:107CC0000197F1F704C0E3E0F0E03197F1F70E948B
:107CD000D43D8C1719F083E490E008C080E490E074
:107CE00005C082E490E002C084E490E0DF91CF918F
:107CF0000895809194009091950090933F268093F1
:107D00003E2621E020932B268091390181FF15C06A
:107D10002093A525809194009091950090933B2607
:107D200080933A2620932926809139018D7F809374
:107D300039018091A5258823E1F786E10E941E3E46
:107D400081E08093A62508958091A625882351F48B
:107D50008091700F882321F081E08093F20F02C0A0
:107D60000E94793E81E090E008950E94193E1092B1
:107D7000A6250E94DB3D8091390182608093390104
:107D8000809129268823E9F18091940090919500B3
:107D900020913A2630913B2682179307A0F48091D8
:107DA000062690910726A0910826B09109268C57A7
:107DB000914EAF4FBF4F8093062690930726A09316
:107DC0000826B09309268091940090919500821B1B
:107DD000930BA0E0B0E040910626509107266091F9
:107DE000082670910926840F951FA61FB71F809340
:107DF000062690930726A0930826B0930926109292
:107E0000292680912B268823E9F180919400909176
:107E1000950020913E2630913F2682179307A0F4CB
:107E200080910E2690910F26A0911026B0911126D8
:107E30008C57914EAF4FBF4F80930E2690930F26D5
:107E4000A0931026B09311268091940090919500F4
:107E5000821B930BA0E0B0E040910E2650910F26BC
:107E60006091102670911126840F951FA61FB71FD1
:107E700080930E2690930F26A0931026B093112680
:107E800010922B2608958091F20F882321F00E94F2
:107E9000793E1092F20F8091F30F882321F00E9417
:107EA000B53E1092F30F1092700F08950F931F9329
:107EB000CF93DF93F82FE92FAB0181E08093700F10
:107EC0000091EA251091EB252091EC253091ED25CC
:107ED0000F5F1F4F2F4F3F4F0093EA251093EB2565
:107EE0002093EC253093ED25862F8E5F87FF0CC005
:107EF0008091A3259091A42501969093A425809329
:107F0000A325CFEFDFEF09C021E73FE0C9016F2FC5
:107F10007E2F0E945166C0E0D0E00E94433FCE0118
:107F2000DF91CF911F910F9108958091A62588230D
:107F300099F08091700F882321F40E94003E8823DD
:107F400031F481E08093F30F81E090E008950E9486
:107F5000B53E80E090E0089580E090E008951F93A2
:107F6000CF93DF930F92CDB7DEB78FB78983809120
:107F7000700F882331F5F8948091A625882351F05D
:107F80008091390181FD1BC00E94003E8823B9F019
:107F900080E003C00E94A43E81E0909147019E30A2
:107FA00010F010E001C01FEF882311F00E94953FF0
:107FB00016FF05C089818FBF81E090E004C08981F0
:107FC0008FBF80E090E00F90DF91CF911F910895D7
:107FD00080936F0F08950E94D43D8250813130F418
:107FE000E82FF0E0E65AFA4F8081089581E0089585
:107FF00008958FEF80934E018CE691E060EF44E0AE
:1080000022E00E949F438CE290E06EE041E025E098
:108010000E949F4380E880936F0180914601809386
:108020006D0184E491E060E245E021E00E949F431D
:108030000895CF93DF93CDEFD3E0CE010197F1F711
:108040000E948B4310921A2410929C2410921E2599
:108050001092192410921824E9E3F1E080818E7FB8
:10806000808380818D7F80838DE090E00197F1F7A0
:1080700080818160808382E491E06FE140E023E0D1
:108080000E949F432197F1F780915D0180915E01ED
:108090000E94F93F8CE395E060E070E00E94672D5C
:1080A0000E94793E81E090E0DF91CF910895809128
:1080B000F40F0895CF93DF930F92CDB7DEB7898386
:1080C0000E94193E29812093F40F88E491E06FE12A
:1080D00040E00E949F430F90DF91CF9108950E944E
:1080E0005A4086E00E941E3E0895FA018093620184
:1080F0009093630160936001709361013097C1F0C8
:10810000808180936B01818180936A018281809359
:1081100069018381809368018481809367018581EF
:1081200080936601868180936501878180936401D5
:1081300008958CE395E00E94892D81E080931124BD
:10814000809112249091132401969093132480938C
:10815000122481E090E00895CF93DF935091192489
:10816000252F30E0F901EE0FFF1F3695322F222721
:1081700037952795E20FF31FE65EFB4D40814423C0
:1081800009F4F4C02091390121FDF0C02091A62509
:10819000222309F4EBC047FF23C0852F90E0FC01A8
:1081A000EE0FFF1F9695982F882797958795E80FD4
:1081B000F91FE65EFB4D10828091DA259091DB2558
:1081C000A091DC25B091DD250196A11DB11D809304
:1081D000DA259093DB25A093DC25B093DD25C6C07E
:1081E000433018F5852F90E0FC01EE0FFF1F9695A8
:1081F000982F882797958795E80FF91FE65EFB4D26
:1082000010828091D6259091D725A091D825B09144
:10821000D9250196A11DB11D8093D6259093D72510
:10822000A093D825B093D925A1C0C42FD0E0229720
:108230006C177D0718F5852F90E0FC01EE0FFF1FEE
:108240009695982F882797958795E80FF91FE65EF2
:10825000FB4D10828091D2259091D325A091D425F9
:10826000B091D5250196A11DB11D8093D225909383
:10827000D325A093D425B093D52578C0252F30E001
:10828000B901660F771F3695322F2227379527952C
:10829000620F731F655E7B4D50E00E945166209116
:1082A0001924822F90E0FC01EE0FFF1F9695982F66
:1082B000882797958795E80FF91FE656FB4D808133
:1082C00080930A24822F90E0FC01EE0FFF1F969509
:1082D000982F882797958795E80FF91FE65EFB4D45
:1082E00010822F5F20931924233010F0109219244C
:1082F0008091192490E0FC01EE0FFF1F9695982FB6
:10830000882797958795E80FF91FE65EFB4D8081DA
:10831000882311F00E9499406091470160930B24DB
:1083200080911024882311F0681710F460931024B2
:1083300084E070E00E94DA3460910A2483E070E007
:108340000E94DA348091EE259091EF25A091F025DE
:10835000B091F1250196A11DB11D8093EE2590935A
:10836000EF25A093F025B093F12502C0C0E0D0E046
:10837000CE01DF91CF910895CF93DF93EC018881F7
:108380009981009729F024E08B3F920739F505C0C9
:108390008BEF94E09983888325C0623819F5109299
:1083A00011240E9460340E94C13360E870E00E9492
:1083B000AC401816190644F40E94BC33E091CD0578
:1083C000F091CE050995E4CF80910E2490910F2471
:1083D000019690930F2480930E24DACF198218828D
:1083E00083E001C081E0DF91CF91089591E0909307
:1083F000700F0E94F13D0E94433F08958091390122
:1084000081FD07C085E491E06FE040E00E94954364
:10841000089580E108950F931F93CF93DF93C82FA2
:1084200021E02093700FD091A6258091390181FF22
:1084300016C0809194009091950090933B26809374
:108440003A26209329262093A525809139018D7FF6
:10845000809339018091A5258823E1F7D0E00E941F
:10846000193E8091A625882309F441C080912B26CE
:108470008823E9F1809194009091950020913E2607
:1084800030913F2682179307A0F480910E26909199
:108490000F26A0911026B09111268C57914EAF4F08
:1084A000BF4F80930E2690930F26A0931026B09373
:1084B00011268091940090919500821B930BA0E06F
:1084C000B0E040910E2650910F26609110267091D9
:1084D0001126840F951FA61FB71F80930E26909319
:1084E0000F26A0931026B093112610922B2689E117
:1084F0000E941E3E86E00E94E534009751F00E94E3
:10850000FE41082F86E00E94E53481500E94F13D33
:1085100002C000E010E0809194009091950090934B
:108520003D2680933C2681E080932A26F894809112
:108530003901826080933901809139018D7F809368
:1085400039016C2F6E5F81E79FE00E94D0437894E1
:108550008091A0259091A12501969093A1258093CB
:10856000A0250E94193E82E491E060EE45E00E9461
:108570009543C82F86E00E94E534009719F0802FBC
:108580000E94F13DDD2319F00E94793E02C00E9455
:10859000B53E80912A268823E9F18091940090913C
:1085A000950020913C2630913D2682179307A0F438
:1085B00080910A2690910B26A0910C26B0910D2651
:1085C0008C57914EAF4FBF4F80930A2690930B2646
:1085D000A0930C26B0930D26809194009091950065
:1085E000821B930BA0E0B0E040910A2650910B262D
:1085F00060910C2670910D26840F951FA61FB71F42
:1086000080930A2690930B26A0930C26B0930D26F8
:1086100010922A268091A625882361F080919400EB
:108620009091950090933F2680933E2681E0809321
:108630002B2607C082E491E06FE140E023E00E9436
:108640009F430E94433FC130E1F0C330A9F48091C1
:10865000E2259091E325A091E425B091E5250196CE
:10866000A11DB11D8093E2259093E325A093E425FD
:10867000B093E525C2E00AC0C53029F0C73031F417
:1086800004C0C0E003C0C3E001C0C1E08C2F90E093
:10869000DF91CF911F910F910895CF93DF93EB015D
:1086A0000E94563F009729F4CE010E940B4200978A
:1086B00051F02091A3253091A4252F5F3F4F309397
:1086C000A4252093A325DF91CF910895CF93DF9325
:1086D0008091A625882321F40E94A43EC1E001C018
:1086E000C0E00E94D43D863111F0813119F4D0915F
:1086F000470109C086E491E06FE140E00E949543A4
:10870000D82FDD0FD80FCC2311F00E94953F8D2F6D
:10871000DF91CF9108951092F60F1092F50FEFE6CA
:10872000F0E08081806280830895FC01808186234F
:1087300090E002C0959587954A95E2F70895F894E0
:10874000FC019081862F8095892330E002C0220FA2
:10875000331F4A95E2F72623282B20837894089527
:10876000CF93DF93EC012196E0917B01DC01EC9348
:108770002E2FA0E8B1E03D9139932150E1F7E1506F
:10878000F0E0E058FE4F2181FC01E058FF4F2083CC
:108790008F579F4F21E0FC012083DF91CF910895F7
:1087A000FC0160938001A1E8B1E0615881918D9353
:1087B0006A17E1F708951F920F920FB60F920BB64A
:1087C0000F9211242F933F934F935F936F937F9357
:1087D0008F939F93AF93BF93EF93FF938091470144
:1087E00080930B242091182430E0C901880F991F31
:1087F0003695322F222737952795820F931F865E55
:108800009B4D0E94B043809118248F5F8093182461
:10881000833010F0109218240E949940FF91EF913C
:10882000BF91AF919F918F917F916F915F914F9188
:108830003F912F910F900BBE0F900FBE0F901F9086
:1088400018951F920F920FB60F9211240F900FBE22
:108850000F901F9018951F920F920FB60F92112430
:108860000F900FBE0F901F9018951F920F920FB68A
:108870000F9211240F900FBE0F901F9018951F920A
:108880000F920FB60F9211241092A5250F900FBED4
:108890000F901F9018951F920F920FB60F921124F0
:1088A0001092A5250F900FBE0F901F9018951F9244
:1088B0000F920FB60F9211248F9381E080931124B1
:1088C0008F910F900FBE0F901F9018951F920F92CF
:1088D0000FB60F9211241092A5250F900FBE0F9086
:1088E0001F9018951F920F920FB60F9211248F931D
:1088F0009F938091F50F9091F60F01969093F60F4C
:108900008093F50F9F918F910F900FBE0F901F9046
:1089100018950F931F93CF93DF938091AE2590917D
:10892000AF25A091B025B091B1250196A11DB11D33
:108930008093AE259093AF25A093B025B093B12539
:108940000E9421478C0187EF9FE00E94312E08C0D2
:10895000EA81FB81309709F00995CE010E94D72E5C
:10896000EC010097A9F70115110519F0C8010E9443
:108970009F2BDF91CF911F910F9108950E94434C3F
:108980000E9460340E943A458EEA95E09093A925B2
:108990008093A8250E941E4782E090E060E074E08A
:1089A00040E05EE12FEF31E00E94DF460895CF9274
:1089B000DF92EF92FF920F931F93CF93DF936C019F
:1089C0008B017A0187EF9FE00E94312E09C0EC8174
:1089D000FD81309711F0C8010995CE010E94D72E74
:1089E000EC010097A1F7C601B801A7010E94A92BCD
:1089F000DF91CF911F910F91FF90EF90DF90CF907B
:108A00000895BC0187EF9FE00E94A02E0895BC014D
:108A100087EF9FE00E946B2E0895CF93DF93EC01C8
:108A20008091AA259091AB25A091AC25B091AD2560
:108A30000196A11DB11D8093AA259093AB25A0930B
:108A4000AC25B093AD25CE010E943447009769F064
:108A50000E94DB33E091B205F091B30587ED94E419
:108A6000BE01099581E090E002C080E090E0DF91D6
:108A7000CF91089589EF9FE00E942D2E08950F93C6
:108A8000CF93DF93EC017B836A8318865F834E83E9
:108A900089EF9FE0BE010E94A02EE091FB0FF091B4
:108AA000FC0F309749F04C815D818A819B816885FC
:108AB00020E030E001E00995DF91CF910F9108951A
:108AC000BC0189EF9FE00E946B2E08950F93DC019B
:108AD00018961C921897E091FB0FF091FC0F3097BD
:108AE00059F012968D919C91139760E040E050E010
:108AF00020E030E000E009950F9108950F93DC012C
:108B0000AB0114962D913C91159781E018968C93AA
:108B1000189715967C936E931497E091FB0FF09144
:108B2000FC0F309739F012968D919C91139761E06C
:108B300000E009950F9108950F93DC01E091FB0F80
:108B4000F091FC0F309769F014962D913C91159798
:108B500012968D919C91139718966C91A90101E042
:108B600009950F910895E091FD0FF091FE0F309758
:108B700009F0099508959093FE0F8093FD0F0895D5
:108B80009093FC0F8093FB0F089589EF9FE00E9464
:108B9000312E0895EF92FF920F931F93CF93DF939F
:108BA0008C01EB017A0189EF9FE00E94312E15C004
:108BB000DC0112962D913C9113972C173D0759F427
:108BC0001696ED91FC911797309749F0B801AE01D8
:108BD0009701099504C00E94D72E009749F7DF91AD
:108BE000CF911F910F91FF90EF9008950895AF924C
:108BF000BF92CF92DF92EF92FF920F931F93CF938A
:108C0000DF9300D0CDB7DEB75B010E94C133FC011A
:108C1000E080F180FA82E982FCE0EF16F10418F4BA
:108C200000E010E02DC000D000D086E795E0EDB761
:108C3000FEB792838183F482E3820E94D0660F9014
:108C40000F900F900F901FC00E94C133F801EE0FDC
:108C5000FF1FEE0FFF1FE80FF91FC280D3800E9495
:108C6000C1330F5F1F4FF801EE0FFF1FEE0FFF1F05
:108C7000E80FF91F40815181C501B6010E94CA4524
:108C80000E151F0509F70F900F90DF91CF911F91DF
:108C90000F91FF90EF90DF90CF90BF90AF9008952D
:108CA000CF93DF93CAE1D0E1609130107091311021
:108CB000CE0143E756E420E030E00E94C2300E943B
:108CC000404C60913010709131100E941963BC01CA
:108CD000CE01409747E956E420E030E00E94C230E0
:108CE000DF91CF91089580913010909131102091B3
:108CF0002E1030912F10880F991F2817390708F46C
:108D0000C90190933110809330100E94504608950D
:108D10000F93013051F480912A1090912B10909371
:108D20003110809330100E9450460F910895CF93D8
:108D3000DF930E9460340E94C133EC0119821882D3
:108D40000E94C54520C012962D913C911397FC01BD
:108D5000EE0FFF1FEE0FFF1FEC0FFD1F338322836B
:108D600014962D913C9115970196FC01EE0FFF1F73
:108D7000EE0FFF1FEC0FFD1F318320839983888343
:108D8000CD010E94D72EDC0188819981109729F0AE
:108D900018962C9118972223B1F6880F991F880FE7
:108DA000991F02960E94BC3388819981009721F017
:108DB0008FEF9FE00E94722BDF91CF910895EF9289
:108DC000FF920F931F93CF93DF93FC018B017A01E6
:108DD000E9018FEF9FE0BF0143E955E00E94542B6A
:108DE00010932B1000932A10F0922D10E0922C106B
:108DF000D0932F10C0932E1088E896E40E94C045AF
:108E0000DF91CF911F910F91FF90EF900895CF9335
:108E1000DF93CAE1D0E1CE010E944931CE014097F3
:108E20000E944931CE014B970E946F2BDF91CF9169
:108E30000895809130109091311008950E94B52BC3
:108E40000895CF93DF93E0919705F09198050995E8
:108E5000EC01009729F06A817B8181E00E94DA347D
:108E6000CE01DF91CF9108950F931F93CF93DF939E
:108E7000EC01E0919905F0919A0509958C016A81C0
:108E80007B8181E00E94DA3481E090E001151105D8
:108E900011F480E090E0DF91CF911F910F91089540
:108EA000E0919B05F0919C05099508959C0180E057
:108EB00090E005C0F90131974081840F911D2E5F2C
:108EC0003F4FF901329740814423A1F70895FC01F7
:108ED000308120E0818190E0822B932B02C0880FAB
:108EE000991F6A95E2F7892F9927FA01E356FA4FFD
:108EF000208130E08223932328E030E0241B350BCF
:108F000002C0969587952A95E2F708956F927F9211
:108F10008F929F92AF92BF92CF92DF92EF92FF9289
:108F20000F931F93CF93DF935C013B018A0169018B
:108F30002830310544F4CB01BA01A9010E946747EA
:108F4000F50180834EC0790173E0F594E7947A953A
:108F5000E1F74115510521F04501C0E0D0E005C021
:108F6000F301D50180E090E021C0C3018C0F9D1F6B
:108F7000B80148E050E00E946747F40181934F0137
:108F80002196CE15DF058CF3C701F7FE02C080E005
:108F900090E0A601477050704115510511F1E501AF
:108FA000C80FD91F860D971DB80118C021912D93A8
:108FB00001968E159F05D4F3C701F7FE02C080E02D
:108FC00090E0A601477050704115510551F0E50140
:108FD000C80FD91F860D971D60E070E00E9467479B
:108FE0008883DF91CF911F910F91FF90EF90DF90D9
:108FF000CF90BF90AF909F908F907F906F9008958B
:109000008F929F92AF92BF92CF92DF92EF92FF9298
:109010000F931F93CF93DF9300D000D0CDB7DEB76F
:109020000E94C1338C0182E090E00E949E33009741
:1090300009F45FC0F801918180E02081820F911DC9
:109040000E94C92B7C01009709F455C00E94C133CE
:109050004C01F7018681482F46954695469550E08C
:1090600090E08770907021E030E0009711F420E0EC
:1090700030E0CA01820F931F0E949E330097C9F10E
:10908000F70104811581CC24DD242EC0F801A180D4
:10909000BB24B601A3E075956795AA95E1F7680D25
:1090A000791DA60147705070883168F0CE01039693
:1090B00095010E948647F8018081BE016D5F7F4F58
:1090C0000E94EE340DC01A821982CE0101969501DC
:1090D0000E94864769817A81F80180810E94DA3492
:1090E000CA0CDB1C0E5F1F4FF8018081882371F6CC
:1090F00002C0EE24FF24C7010F900F900F900F9035
:10910000DF91CF911F910F91FF90EF90DF90CF9063
:10911000BF90AF909F908F900895FC0150E080E148
:1091200090E0861B970B821B930B02C0440F551FC8
:109130008A95E2F78081852B80838181842B8183CE
:1091400008956F927F928F929F92AF92BF92CF922B
:10915000DF92EF92FF920F931F93CF93DF933C0127
:109160006B015A0179012830310524F4C301FA0159
:10917000408159C08901B3E015950795BA95E1F78B
:109180006115710521F04A01C0E0D0E005C0FA0187
:10919000D30180E090E023C0F40141914F01C3016D
:1091A0008C0F9D1FB60128E030E00E948D4821966B
:1091B000C017D1078CF3980117FF02C020E030E000
:1091C000D701A770B070109781F1F501E20FF31F7E
:1091D000408150E0C6018A1B9B0B089619C0219163
:1091E0002D93019680179107D4F3980117FF02C0C1
:1091F00020E030E0D701A770B0701097B1F0F50112
:10920000E20FF31F408150E088E090E08A1B9B0B47
:1092100002C0559547958A95E2F7C301820F931FC7
:1092200060E070E09D010E948D48DF91CF911F9119
:109230000F91FF90EF90DF90CF90BF90AF909F90F5
:109240008F907F906F9008956F927F928F929F92F0
:10925000AF92BF92CF92DF92EF92FF920F931F9344
:10926000CF93DF9300D0CDB7DEB77C01DC0116963B
:109270008C911697282F26952695269530E090E01C
:109280008770907001E010E0009711F400E010E0AA
:10929000020F131FC80102960E942634009709F49A
:1092A00051C00E94C833FC01D70112968C911297CD
:1092B000808313968C9181830E94C83332E0632EA1
:1092C000712C680E791EC30160E070E0A8010E9455
:1092D0005A66F701E480F580CC24DD242CC0D70148
:1092E0001196AC901197BB24860193E015950795D4
:1092F0009A95E1F7060D171D27E0822E912C8C2000
:109300009D20883130F00E94F834AC01C801B401CE
:1093100009C00E94E5349A838983C801B401AE0173
:109320004F5F5F4F95010E94A148CA0CDB1CE2E031
:10933000F0E0EE0EFF1ED7018C91882381F681E0CC
:1093400090E002C080E090E00F900F90DF91CF910D
:109350001F910F91FF90EF90DF90CF90BF90AF9053
:109360009F908F907F906F900895E091CB05F09142
:10937000CC0509950895E0917405F091750509955E
:109380000895E091CF05F091D00509950895E091F9
:10939000D105F091D2050995089580E090E00895F7
:1093A0000895E0915605F09157050995089580E0DC
:1093B00090E008950F931F93CF93DF93CDB7DEB75F
:1093C000E0970FB6F894DEBF0FBECDBF0E941134F8
:1093D0008C010E94C133602FAE014F5F5F4F0E942E
:1093E000D051882309F446C088A99801281B310967
:1093F000C9010E949E330097E9F12E81222379F161
:109400008A859B853BEA8D3C930721F03FEF8F3F98
:10941000930781F5223069F088E090E00197E1E060
:10942000F0E0EC0FFD1FE80FF91F23852F3F21F01F
:1094300007C082E090E0F2CF181619067CF30FC047
:1094400089E1BE01645F7F4F0E94EE3489E10E9492
:10945000F83467EB73E20E940C2B009759F088E117
:10946000BE016A5E7F4F0E94EE34E091B405F09138
:10947000B5050995E0960FB6F894DEBF0FBECDBFD7
:10948000DF91CF911F910F910895AF92BF92CF922C
:10949000DF92EF92FF920F931F93CF93DF93CDB79D
:1094A000DEB7E0970FB6F894DEBF0FBECDBF5C010C
:1094B0006B01FE01319680E3DF011D928A95E9F789
:1094C00081E089838CE00E94E5348C831D821F82B9
:1094D0008091341089878F5F8093341003E0088770
:1094E0008DEC9BEA9B878A8789E10E94F83468EBC0
:1094F00074E00E940C2B009731F082E08E838FEF96
:109500008C878D8709C089E10E94F834BC01CE01A7
:109510000C960E94032B0E838DEC9BEA9D8B8C8B0B
:10952000CE01469667EB73E20E94032B0E94C13383
:109530009FA78EA70E94113488ABCE0101960E948E
:10954000E150082F90E00E942634009749F10E94D4
:10955000C833BC01CE010196402F0E94FF500091FC
:109560004C0510914D050E94C8337C010E941B34AC
:10957000BC01C701F8010995A114B10489F0009755
:1095800021F08130910561F404C0C60160E070E013
:1095900003C0C60164E070E041E050E0F5010995C8
:1095A000E0960FB6F894DEBF0FBECDBFDF91CF912E
:1095B0001F910F91FF90EF90DF90CF90BF90AF90F1
:1095C00008950E94404C80933410E0915605F0912C
:1095D000570509950895009731F0E0915605F091EF
:1095E000570509950895E0915805F0915905099599
:1095F0000895CF93DF93EC0104C060E070E00E9417
:10960000672D899199910097C1F7DF91CF910895C6
:10961000CF93DF93EC0102C00E94AE2C8991999107
:109620000097D1F7DF91CF910895CF93DF93EC01AD
:109630007B836A830E94153C99838883DF91CF9155
:109640000895FC018081918122813381820F931FD3
:10965000918380830895CF93DF93EC010E94153CA2
:1096600099838883DF91CF910895CF93DF93EC01A5
:109670000E94153C28813981AC01421B530B9A0191
:109680002F5F3F4F81E090E04A815B814217530793
:1096900010F080E090E0DF91CF910895CF93DF93B9
:1096A000FC01C281D38180819181C80FD91F0E94A2
:1096B000153C9E01281B390BC901DF91CF910895FC
:1096C000CF93DF93E0E3F6E2C2EFD5E2A4E2B6E2A5
:1096D0001192119219921992199219921D9286E281
:1096E000E834F807A9F7DF91CF9108950F931F93FE
:1096F000CF93DF93FC01EC5DF94D20818C01000FCD
:10970000111F000F111F222311F12091940030919D
:109710009500E801CE50DA4DFC01EE0FFF1FE05D31
:10972000F94D80819181A901481B590BCA01A0E024
:10973000B0E0488159816A817B81840F951FA61F03
:10974000B71F88839983AA83BB8331832083F80161
:10975000EE50FA4D6081718182819381DF91CF91CA
:109760001F910F91089560E070E080E090E008950F
:10977000FC01EE0FFF1FEE0FFF1FEE50FA4D40836E
:109780005183628373830895EF92FF920F931F9327
:10979000CF93DF93B4E2EB2EB6E2FB2EE2EFF5E2DD
:1097A000C0E3D6E220E030E0D7018D917D0188232F
:1097B000C9F0009194001091950088819981A801C9
:1097C000481B590B60E070E080819181A281B381D8
:1097D000840F951FA61FB71F80839183A283B38335
:1097E000198308832F5F3F4F349622962C30310522
:1097F000D9F6DF91CF911F910F91FF90EF900895CF
:109800000E94635008950F931F93FC0180913510BF
:109810009091361033832283158304837183608390
:10982000F0933610E0933510009719F4CB010E94A5
:109830007D5080E090E01F910F9108958091351048
:10984000909136100097C1F010923610109235109A
:10985000DC0114966D917C9115971296ED91FC9117
:1098600013970995E0913510F0913610309721F05B
:10987000808191810E947D5008950E94F363089534
:109880000E94EE63089585ED95E00E949F2D8DED79
:1098900095E00E949F2D0895CF93DF930E94CE33D1
:1098A0000097A9F08DED95E00E94BE2DEC01009788
:1098B00029F10E941134998388830E940C349B8380
:1098C0008A83CE0104960E9448338CAB17C085ED85
:1098D00095E00E94BE2DEC01009771F002960E9467
:1098E0005A3399838883BE016E547F4FCE018E57C1
:1098F0009F4F0E94B83402C0C0E0D0E0CE01DF919B
:10990000CF910895BC016E547F4F8E579F4F0E9498
:10991000B8340895CF93DF93EC0185ED95E0BE0157
:109920000E940F2E009719F085ED95E009C08DED8E
:1099300095E0BE010E940F2E009729F08DED95E075
:10994000BE010E94E92DDF91CF910895CF93DF935F
:10995000EC0185ED95E0BE010E940F2E009779F095
:1099600068817981CE0102960E948934BE016E54CD
:109970007F4FCE018E579F4F0E94C9341CC08DED82
:1099800095E0BE010E940F2E0097A9F00E9460345E
:10999000688179818A819B810E9489348CA990E0B9
:1099A0000E9426340E94C8334CA9BE016C5F7F4FD1
:1099B00050E00E945166DF91CF910895CF93DF93DD
:1099C000EC0185ED95E0BE010E940F2E009719F085
:1099D000CE0102960CC08DED95E0BE010E940F2EC7
:1099E000009719F08A819B8102C080E090E0DF91AE
:1099F000CF910895FC0180819181089570E06F5BA3
:109A00007F4F660F771F680F791FCB010895E62FF0
:109A1000F0E0EF5BFF4FEE0FFF1FE80FF91F8081B3
:109A200091810895089580E996E10E94F42F0097AE
:109A300021F080E996E10E94DF2F0895E0917B16E6
:109A4000F0917C16309711F00995089580E0089503
:109A5000EF92FF920F931F93CF93DF937C018A01C4
:109A6000FC0180819181009731F0F3E08C309F07F9
:109A700009F0FFC02BC080E0E82FF0E0EE0FFF1FE1
:109A8000EE0FFF1FE258F94E118210828F5F843073
:109A900098F380937D168091BA0D9091BB0DEEE7FF
:109AA000F6E1918B808B0E94A72C8093482680E959
:109AB00096E160E470E00E94C92F0E9445538CE05B
:109AC00093E0F7019183808381E0D7C0623009F48D
:109AD000B2C0633030F4662309F482C0613079F794
:109AE00095C0673819F0683851F73AC01092981647
:109AF000CEE7D6E113C08A819B818017910741F49C
:109B0000888199810E947B54198218821B821A8253
:109B10002496809198168F5F80939816809198165E
:109B2000843048F3E8E5FBE2848D958D801791073A
:109B300019F4158E148E118EB0962BE2E83DF207C3
:109B400098F3EEEEFBE2818592858017910711F480
:109B5000158214823D968CE2E037F807A0F3AFCF70
:109B6000E6E140395E0709F0AACFCA010E94F42F4E
:109B7000009709F4A4CF109298162DC0F0E035E0BC
:109B8000EE0FFF1F3A95E1F7E85AF44D818D8823D7
:109B9000E9F080E996E10E94DF2F8091981690E02D
:109BA00025E0880F991F2A95E1F7885A944D9093E4
:109BB000572B8093562B82E00E94AF548091492608
:109BC00090914A26009711F00E941E4D80919816A0
:109BD0008F5F80939816E0919816E43078F26FCFFB
:109BE0004115510509F46BCF5093572B4093562BD9
:109BF00083E00E94AF548091492690914A260097B5
:109C000011F00E941E4D0E94134D59CF4115510570
:109C100009F455CF5093532B4093522B85E00E946B
:109C2000AF548091492690914A26009709F447CF76
:109C30000E941E4D44CF8091492690914A2600975C
:109C400009F43DCF80915A26863031F480917226F6
:109C500081FF02C00E94134D81E00E94AF548091A9
:109C6000492690914A26009709F429CF0E944B4F2C
:109C700026CFF7011182108283E0DF91CF911F91EF
:109C80000F91FF90EF90089590937C1680937B1630
:109C900008959C014091BA0D5091BB0D60E0EEE734
:109CA000F6E114C0808191818217930769F4828163
:109CB00093818417950741F460939916118210825D
:109CC000C9010E947B54089534966F5F643050F34D
:109CD00060939916089540E0EEE7F6E116C0542F20
:109CE0005F5F208131812115310569F440939A1617
:109CF000918380832091BA0D3091BB0D33832283F1
:109D00000E94955408953496452F443040F3409373
:109D10009A160895FC018091BA0D9091BB0D958F14
:109D2000848F778F668F0895FC018091BA0D909192
:109D3000BB0D92878187748763870895CF93DF93E4
:109D4000EA010E940754009749F02091BA0D309122
:109D5000BB0DFC0132872187D487C387DF91CF9168
:109D600008950F931F93CF93DF9300D000D0CDB70A
:109D7000DEB78C01AB018FEF89838A838B838C8361
:109D8000CE010196B8010E949E4E009719F0FC0189
:109D9000158304830F900F900F900F90DF91CF9158
:109DA0001F910F91089582EF95E062E040E050E04E
:109DB0000E94582D10924A26109249260895AC010F
:109DC00082EF95E061E00E94352D0895AC0182EFAD
:109DD00095E060E00E94352D08950F931F93CF9377
:109DE000DF938A010E947B53EC01009759F0809128
:109DF000BA0D9091BB0D9D8F8C8F1F8F0E8FCE0152
:109E00000E94E64ECE01DF91CF911F910F910895F0
:109E1000CF93DF93A091562BB091572B109719F049
:109E2000ED016C9605C0C091522BD091532B299611
:109E30008091512B86FF22C010929B1640E0EEE7E6
:109E4000F6E116C08081918114962D913C91159771
:109E50008217930759F482819381009739F04093D8
:109E60009B16998388831B821A8206C034964F5FA3
:109E7000443040F340939B160E94134D8881998192
:109E8000009731F04A815B81609148260E94582DED
:109E9000DF91CF9108950F931F93CF93DF9380911C
:109EA0005A26863009F074C08091492690914A263E
:109EB00025E08030920709F06BC0C4E9D2E0D0936E
:109EC0004A26C093492602E00093532614E91093D2
:109ED000542610927626109275260E943D53809546
:109EE0009095909376268093752610925C2610921A
:109EF0005B260E942C538095909590935C268093CE
:109F00005B260E941E4DD0934A26C093492600939B
:109F10005326109354269091542B8091552BE92F62
:109F2000F82FDF01A459BD4F8CE692E00D9001920D
:109F30000197E1F789E696E26CE672E00E94E95249
:109F400080914D268093692680914E2680936A26C3
:109F500080914F2680936B268091502680936C26AB
:109F600010927626109275260E943D53809590950A
:109F7000909376268093752610925C2610925B262D
:109F80000E942C538095909590935C2680935B263D
:109F90000E941E4DDF91CF911F910F910895FC01FA
:109FA00020E030E080E0A8E111C0419198E0542F1A
:109FB0005827B52FB17050FD8A278695B13009F426
:109FC00080684695915099F72F5F3F4F26173707C6
:109FD00061F708951F920F920FB60F920BB60F9272
:109FE00011242F933F934F935F936F937F938F939E
:109FF0009F93AF93BF93EF93FF93809194009091C1
:10A000009500909335268093342681E08093262610
:10A0100080917100807D809371000E941E4C809120
:10A0200026268823E9F18091940090919500209153
:10A0300034263091352682179307A0F48091FA25B3
:10A040009091FB25A091FC25B091FD258C57914E58
:10A05000AF4FBF4F8093FA259093FB25A093FC252B
:10A06000B093FD258091940090919500821B930BF5
:10A07000A0E0B0E04091FA255091FB256091FC25CD
:10A080007091FD25840F951FA61FB71F8093FA2599
:10A090009093FB25A093FC25B093FD2510922626D6
:10A0A000FF91EF91BF91AF919F918F917F916F91B0
:10A0B0005F914F913F912F910F900BBE0F900FBE6C
:10A0C0000F901F9018959FB7F894E1E7F0E080811A
:10A0D000807D808388B38F6288BB10929000E1E915
:10A0E000F0E010821092920010929500109294006D
:10A0F0008081856080839FBF08952FB7F8949093E7
:10A1000099008093980088B38F6288BBE1E7F0E004
:10A110008081826080832FBF0895CF93DF93FC01FD
:10A12000DB0185E0EB0119928A95E9F7858190E0E2
:10A1300083709070009711F082E08C93878190E09B
:10A1400083709070009721F082E012968C931297A2
:10A15000858190E083709070009799F0878190E0FE
:10A1600083709070009769F0238934898185928586
:10A170002817390731F481E0848312961C921297D4
:10A1800001C01482C581C370C250C23028F4D0E02F
:10A19000C450DA4F888101C080E011968C931197EA
:10A1A000E781E370E250E23028F4F0E0E450FA4F47
:10A1B000808101C080E013968C931397DF91CF913B
:10A1C0000895CF93DF9300D000D00F92CDB7DEB7C4
:10A1D000BE016F5F7F4F0E948D5089819A81890FE8
:10A1E0008D5F9B81890F9C81890F9D81890F0F90C5
:10A1F0000F900F900F900F90DF91CF910895DF9205
:10A20000EF92FF920F931F93CF93DF9300D000D074
:10A2100000D0CDB7DEB78C017B01BE016F5F7F4FF1
:10A220004E830E948D5079816A81AB81BC81872FDA
:10A2300090E00396860F911D8A0F911D8B0F911D43
:10A240002D81820F911D4E8150E0481759070CF463
:10A2500098C0F801218130E02170307083E0220F36
:10A26000331F8A95E1F7828190E08170907034E02D
:10A27000880F991F3A95E1F7822B90819770892B6F
:10A28000438150E04170507095E0440F551F9A95FE
:10A29000E1F7842B448150E04170507026E0440F78
:10A2A000551F2A95E1F7842BF7018083F80125815A
:10A2B00030E023703070220F331F220F331F86814E
:10A2C00090E08370907054E0880F991F5A95E1F7E1
:10A2D000822B97819295990F990F907C982BF7017B
:10A2E0009183F8018085F7018283723051F4F8017F
:10A2F0008185F7018383F8018285F701848355E026
:10A3000001C053E040E080E090E09801260F311D4D
:10A3100009C0F901E80FF91FD384F701E70FF11D18
:10A32000D0824F5F742F750F0197461791F7972FC3
:10A33000A23089F49701270F311DF8018389F901B3
:10A340008083872F8F5F9701280F311DF801848943
:10A35000F90180839E5F40E020E030E00B0F111D8B
:10A3600009C0F801E20FF31F5589F701E80FF11D4D
:10A3700050834F5F842F890F215030404B1789F74E
:10A3800001C080E026960FB6F894DEBF0FBECDBFA9
:10A39000DF91CF911F910F91FF90EF90DF90089583
:10A3A000BF92CF92DF92EF92FF920F931F93CF93C2
:10A3B000DF937C01B62EEA0182E0861708F0AEC07A
:10A3C000F7018081D82ED294D694D69463E0D62219
:10A3D000F1E0DF22F7019181292F26952695237040
:10A3E000C92EC294C694C69473E0C722382F377022
:10A3F0003883382F36953695369531703983382F16
:10A40000329531703A838295869581708B83DC8298
:10A410002D83892F829583708E83CF828281888756
:10A42000222369F13381948180E0830F911D9A8703
:10A430008987223079F4CA010B9668EB74E00E9498
:10A44000032BF70186818B8785818C878701095FC4
:10A450001F4F20C087010B5F1F4F2330D9F4F70136
:10A460003D96DA0180E092911B969C931B978F5F3B
:10A4700011968830C1F78701035F1F4F0BC087011A
:10A480000D5F1F4FCA010B9668EB74E00E94032B0F
:10A490001A861986CC2089F1DD2059F4F801208133
:10A4A000918180E0820F911D9C8B8B8B0E5F1F4FE3
:10A4B00004C089859A859C8B8B8BF2E0CF1671F452
:10A4C000CE01459668EB74E00E94032BF801818170
:10A4D0008D8B80818E8B0E5F1F4F17C0F3E0CF16E0
:10A4E000A1F4085F1F4FD801FE0180E09E91958B7B
:10A4F0008F5F31968830D1F708C0CE01459668EB62
:10A5000074E00E94032B1C8A1B8A802F8E199B2DBE
:10A51000981B9FA71EA70DA7B81608F480E0DF912F
:10A52000CF911F910F91FF90EF90DF90CF90BF9050
:10A5300008959C0141505040460F571FFB010EC02B
:10A54000B081A0E08181BD01680F711D260F371F0A
:10A550002617370710F42F5F3F4F3296E417F507A1
:10A5600078F3E417F50749F4908180E0280F391F4C
:10A570002817390710F42F5F3F4FC9010895CF9373
:10A58000DF93C0915426D0E064973091532620E0A9
:10A59000C20FD31F9E01280F311DC9016DE576E260
:10A5A00048E050E00E94995265E676E2AE010E94D2
:10A5B0009952009721F098278927982702C08FEF9A
:10A5C0009FEFDF91CF9108959093A3168093A216E9
:10A5D0000895FC014381460F40935026872F992709
:10A5E0002281280F20934F26A181A0934E265081CF
:10A5F00050934D2630E02817390748F48A2F8F5F93
:10A6000080934E26882319F45F5F50934D26842F44
:10A6100090E070708617970798F480914F268F5FAF
:10A6200080934F26882361F480914E268F5F80931C
:10A630004E26882329F480914D268F5F80934D26E6
:10A6400008959C01AB0180E090E0B9010E9499520D
:10A65000982789279827089580E090E061E576E2C1
:10A6600044E150E00E949952009721F098278927F1
:10A67000982708958FEF9FEF089586E00E94BF52BC
:10A68000089581E10E94BF52089580E0E82FF0E034
:10A69000EE0FFF1FE852F44D118210828F5F84305D
:10A6A000A8F380E0E82FF0E035E0EE0FFF1F3A95C9
:10A6B000E1F7E85AF44D118E8F5F843098F380E013
:10A6C00094E09093A6168093A51640E08DE090E06C
:10A6D000242F30E0289FF001299FF00D389FF00DC6
:10A6E0001124E251F44D158214824F5F4A3080F3F9
:10A6F0004093A4160895CF93DF93EC012091A51603
:10A700003091A6162F5F3F4F8DE72030380710F0AD
:10A7100020E030E1522F432FA0E012C0EA2FF0E0FA
:10A72000B5E0EE0FFF1FBA95E1F7E85AF44D818DC1
:10A73000882329F0848195818417950719F3AF5FE9
:10A74000A43061F73093A6162093A5161092A41694
:10A7500080E0E0E0F0E01EC0A82FB0E055E0AA0FD6
:10A76000BB1F5A95E1F7A85AB44D59969C91599739
:10A77000992321F48093A416FD0110C0973049F469
:10A78000309731F05A962C915A97928D921708F47F
:10A79000FD018F5F843000F38093A416309799F108
:10A7A00082E0818F8091A71684878091A816858783
:10A7B0008091A91686878091AA16878788ED94E0F4
:10A7C000938B828B958B848B81E090E0918B808B37
:10A7D000138E81E0828F83E0808F168A80E1878BE1
:10A7E0008091A5169091A61698278927982795837A
:10A7F00084837783668388819981AA81BB818083E2
:10A800009183A283B383CF01DF91CF9108950F93FA
:10A810001F93CF93DF93EC018B012091A51630910C
:10A82000A6166DE070E02F5F3F4F8DE720303807B0
:10A8300010F020E030E1522F432FA0E011C08A2F0A
:10A8400090E0869FF001879FF00D969FF00D1124F8
:10A85000E251F44D84819581AF5F8417950719F318
:10A86000AA3069F73093A6162093A51640E02DE094
:10A8700030E018C0542F5F5F842F90E0829FF0017A
:10A88000839FF00D929FF00D1124E251F44D8481CD
:10A890009581009731F44093A4169F01309749F4B5
:10A8A00024C0452F4A3030F34093A41620E030E016
:10A8B0001CC08091A5169091A616982789279827E5
:10A8C0009583848317830683209729F4108211824D
:10A8D0001282138208C088819981AA81BB818083FA
:10A8E0009183A283B38380E48087C901DF91CF91F4
:10A8F0001F910F91089540E013C0E42FF0E0542F12
:10A900005F5FEE0FFF1FE852F44D20813181281761
:10A91000390729F44093A416118210820895452F17
:10A92000443058F34093A416089540E013C0E42F38
:10A93000F0E0542F5F5FEE0FFF1FE852F44D2081CF
:10A9400031812115310529F44093A4169183808328
:10A950000895452F443058F34093A4160895AF92BC
:10A96000BF92CF92DF92EF92FF920F931F93CF93FC
:10A97000DF93C091562BD091572B843009F4F1C14D
:10A9800029E736E23093552B2093542B30934C26F5
:10A9900020934B26833071F4898D90E08F709070F6
:10A9A0008330910509F074C088899989009709F06E
:10A9B00031C78DC0823009F08EC08091AA168F5F9A
:10A9C0008093AA16882399F48091A9168F5F8093AB
:10A9D000A916882361F48091A8168F5F8093A8162A
:10A9E000882329F48091A7168F5F8093A716109271
:10A9F0004A26109249261092ED2B1092EC2B898D4D
:10AA0000873011F0853041F48A8D8F5F8A8F8431D1
:10AA100009F000C7198EFEC6882309F4FBC62889F1
:10AA200039892115310509F44EC09A8D292F2150FD
:10AA30002A8F992309F0EEC69B8D983031F0282F8C
:10AA40002150223048F4953039F4198E80E88093F3
:10AA5000512B0E94084F94C5953048F423E030E014
:10AA6000092E02C0220F331F0A94E2F701C020E32F
:10AA70002A8F9F5F9B8F90E08F709070833091053D
:10AA8000E1F0843091054CF48130910509F469C3FB
:10AA90008230910509F0BEC60DC08630910509F4DB
:10AAA0007EC58830910509F47AC58430910509F096
:10AAB000B1C675C51092722657C384E08093512B9E
:10AAC0000E94084F92C58F70833009F0A3C688E0BA
:10AAD0008093512B4AC5853019F5E091522BF091A6
:10AAE000532B84819581009709F494C61092572BBB
:10AAF0001092562B2C5030403093552B2093542BD2
:10AB000030934C2620934B261092ED2B1092EC2B79
:10AB100010924A261092492688E08093512B1FC13B
:10AB200080915126853409F075C61091532600E0B6
:10AB300080915426080F111D8091492690914A2634
:10AB40008017910708F466C610934A260093492699
:10AB50008091572690E08F739070009709F05AC645
:10AB600080915826882309F055C64091E82B5091D2
:10AB7000E92BA090FE05B090FF054A155B0559F43E
:10AB80008091EA2B9091EB2B2091000630910106E9
:10AB900082179307A1F08091612690916226841715
:10ABA000950709F037C6209163263091642680917D
:10ABB000EA2B9091EB2B2817390709F02BC60E943E
:10ABC0002C532FEF8F3F920709F024C680915A260D
:10ABD000863009F42EC18131D1F1813009F01AC6D5
:10ABE00080916526883009F015C6109265268091FF
:10ABF0006726909168262FEF873F920710F00996FD
:10AC000001C008969093682680936726E1E5F6E2F6
:10AC100080915D2690915E26A0915F26B09160267E
:10AC20008093612690936226A0936326B093642656
:10AC30008091E82B9091E92BA091EA2BB091EB2B1E
:10AC400084879587A687B78780E48087C0C50C5125
:10AC5000104010934A26009349268DE696E2909381
:10AC6000552B8093542B80916B2690916C260097E6
:10AC700039F00E9441532FEF8F3F920709F0CAC568
:10AC800040916726509168264115510509F4C2C5C7
:10AC90008EEE9BE29093532B8093522B609165260E
:10ACA00070916626A0910006B0910106C09102063F
:10ACB000D09103060091040610910506E0905D26F0
:10ACC000F0905E26C0905F26D09060262EC08481D2
:10ACD0009581009721F14817590709F586819781D9
:10ACE000009719F068177907D1F4208131812A156E
:10ACF0003B0529F4828193818A179B07F9F02C1771
:10AD00003D0729F48281938180179107B9F0E216FB
:10AD1000F30629F482819381C816D90679F0CF0110
:10AD20000D969093532B8093522BE091522BF091E0
:10AD3000532B8CE2E037F80750F26CC51092572B7A
:10AD40001092562B82E08093512B8DE696E29093E1
:10AD50004C2680934B261092ED2B1092EC2B0E94E8
:10AD6000084F8091EC2B9091ED2B009709F452C580
:10AD70009C01245E3F4F30934A262093492630930E
:10AD8000532620935426E091522BF091532B20858B
:10AD90002093592621E120935A260896982789273F
:10ADA000982790936A268093692610926C261092B9
:10ADB0006B26848195819093662680936526868193
:10ADC000978190936826809367268091E82B9091D5
:10ADD000E92BA091EA2BB091EB2B80935D26909309
:10ADE0005E26A0935F26B093602680819181A28128
:10ADF000B3818093612690936226A0936326B093DB
:10AE0000642689E796E29093552B8093542B0E94F9
:10AE100041538095909590936C2680936B26009774
:10AE200009F0D5C48FEF9FEF90936C2680936B262B
:10AE3000CEC40E943D532FEF8F3F920709F0EAC422
:10AE400020916726309168262115310509F4E2C466
:10AE500040916526509166264115510509F4DAC4E2
:10AE6000E0915D26F0915E26A0915F26B09160266C
:10AE7000C8E5DBE2698D6623A9F08C819D812817E6
:10AE8000390781F48E819F814817590759F48881C9
:10AE90009981E817F90731F48A819B81A817B907CE
:10AEA00009F47AC1A0968BE2C83BD80719F310F3D6
:10AEB000809172268F738230B9F43093AC16209350
:10AEC000AB1640E00DC0E42FF0E0EE0FFF1FE8529C
:10AED000F44D808191814F5F2817390709F47DC0B7
:10AEE000443088F34093A4168091722682FD92C468
:10AEF00084E18093722688E290E090934A268093C2
:10AF0000492680E58093712680916C269091702669
:10AF100090936C2630916B2690916F2690936B26C0
:10AF200030936F2620916A2690916E2690936A2620
:10AF300020936E26909169269093A41640916D26D9
:10AF40004093692690936D268F5F809370268823A7
:10AF500079F4832F8F5F80936F26882349F4822FA3
:10AF60008F5F80936E26882319F49F5F90936D26E0
:10AF700080916526909166269093AC168093AB16CF
:10AF800020916726309168263093662620936526A7
:10AF9000909368268093672680915D2690915E2627
:10AFA000A0915F26B09160268093612690936226DF
:10AFB000A0936326B09364268091E82B9091E92BAF
:10AFC000A091EA2BB091EB2B80935D2690935E26A7
:10AFD000A0935F26B0936026DFC31092A41680E092
:10AFE000C0E0D0E022C0E82FF0E075E0EE0FFF1FD8
:10AFF0007A95E1F7E85AF44D918D992321F48093E5
:10B00000A416EF0116C0973079F4209721F0228D15
:10B010009A8D921748F4C82FD0E065E0CC0FDD1F61
:10B020006A95E1F7C85AD44D8F5F8430E0F280937F
:10B03000A416209709F4EEC3D093572BC093562B38
:10B0400083E08A8F888F1E8A84E08F8B1B8E80918D
:10B050006726909168269D838C83809165269091C8
:10B0600066269F838E8380915D2690915E26A091B7
:10B070005F26B091602688839983AA83BB8381E091
:10B08000898F8091A7168C878091A8168D878091D3
:10B09000A9168E878091AA168F8781E090E0998B00
:10B0A000888B80916C268B8780916B268A87809114
:10B0B0006A26898780916926888781E090E00E94CE
:10B0C000465D80917126282F30E0207F3070213539
:10B0D00031050CF446C082958F7090E00597880F7B
:10B0E000991F880F991F3091AD1620E031C0EF5A9B
:10B0F000F94D30A5332329F42093A4161092AD16F0
:10B1000030C0313011F42F5F23C03230E9F441A553
:10B110004430D1F42093A4163093AD1692A580E06C
:10B1200023A530E0282B392B3093AC162093AB1697
:10B13000C90124E0893D920710F088ED94E09B8BD3
:10B140008A8B9D8B8C8B0DC041A5442331F0240F3D
:10B15000E22FF0E0E817F90754F22093A416309399
:10B16000AD1680E180937226809172268260809372
:10B17000722682E08093792684E080937A268093F9
:10B180007B2688ED80937C268CE290E090934A2683
:10B190008093492680E6ADC2D093572BC093562B9F
:10B1A0001092512B4091722650E042FF03C0198E3D
:10B1B00080E248C28091712682958F70880F880F37
:10B1C0008093A4169801281B3109245130403093F4
:10B1D0004A2620934926862F90E08F709070823007
:10B1E000910539F4CA018F7390708231910551F441
:10B1F00029C08130910531F4CA018F73907082307B
:10B20000910501F12115310529F4CA01837090706F
:10B210000097C1F0909169268885981709F05FC260
:10B2200090916A268985981709F059C290916B26EA
:10B230008A85981709F053C290916C268B859817D0
:10B2400009F04DC244FF4AC06889798961157105CA
:10B2500009F444C0CE010C960E94E95230916D264B
:10B2600080914D263817D1F520916E2680914E267B
:10B270002817A1F590916F2680914F26981771F5A8
:10B280008091702640915026841741F53C872D8788
:10B290009E878F878B8D8823D1F42E89888D9A8DF8
:10B2A000891B922F969596959695891B280F2E8B24
:10B2B00087FD81959F89392F36953695931B980F79
:10B2C0009F8B822F869586958695890F888F81E042
:10B2D0008093512B888D8A8F198A188A498D50E066
:10B2E000CA018F7090708430910509F4B0C1853027
:10B2F000910564F482309105C9F1833091050CF019
:10B30000B6C08130910509F085C211C08630910523
:10B3100009F4DDC1863091050CF4B9C1873091057F
:10B3200009F4DDC18830910509F074C285C18091AE
:10B33000512B80FF14C083E0898F80E48093512BD0
:10B34000198A188A8091492690914A26009709F413
:10B3500008C122E42093512B0E94465D02C18091D6
:10B3600072268F73823009F055C2FBCE8091512B2B
:10B3700080FF72C0809172268F73823109F06CC099
:10B3800080917126282F30E0207F307021353105E3
:10B390000CF446C082958F7090E00597880F991F36
:10B3A000880F991F3091AD1620E031C0EF5AF94D4A
:10B3B00030A5332329F42093A4161092AD1630C083
:10B3C000313011F42F5F23C03230E9F441A544300D
:10B3D000D1F42093A4163093AD1692A580E023A556
:10B3E00030E0282B392B3093AC162093AB16C901D3
:10B3F00024E0893D920710F088ED94E09B8B8A8BC6
:10B400009D8B8C8B0DC041A5442331F0240FE22F7E
:10B41000F0E0E817F90754F22093A4163093AD1624
:10B4200083E0898F80916926888780916A26898741
:10B4300080916B268A8780916C268B8781E090E0D3
:10B440000E94465D82E48093512B198A188A1092DB
:10B450004A261092492685C080E28093512B0E9493
:10B46000084FE091562BF091572B118E3DCD8091D6
:10B47000722680FF25C044FD23C0888999890097E2
:10B4800009F0C8C18091492690914A2601960E94F0
:10B49000465D2091512B822F80618093512B8091AA
:10B4A000492690914A26009719F022612093512B4A
:10B4B0000E94084F81E090E0998B888B88E06DC0F6
:10B4C00085FF1CC09091772680E02091782630E09F
:10B4D000282B392B8091542B9091552B820F931F41
:10B4E0009093552B8093542B8091492690914A2616
:10B4F000821B930B90934A2680934926809149267C
:10B5000090914A26009749F044FD07C02091512BA5
:10B5100022602093512B0E94465D9091732680E01B
:10B5200020917426820F911D9093AC168093AB16D8
:10B530002C893D892817390710F0009721F43093A2
:10B54000AC162093AB168091AB169091AC169B8BEA
:10B550008A8B8091512B90E083709070009709F452
:10B5600059C11092ED2B1092EC2B0E94084F2091A4
:10B57000512B25FF07C01092ED2B1092EC2B198E4A
:10B5800084E1AEC024FF0DC01092ED2B1092EC2B85
:10B5900081E090E0998B888B84E0898F1B8E81E11C
:10B5A0009FC08091EC2B9091ED2B0097E9F020FF4C
:10B5B00002C0198A188A288939892115310581F430
:10B5C0002A893B892817390720F43093ED2B2093E3
:10B5D000EC2B8091EC2B9091ED2B998B888B04C0F8
:10B5E0003093ED2B2093EC2B1B8E80914B2690916A
:10B5F0004C269093552B8093542B8091EC2B90915B
:10B60000ED2B009759F088899989009739F0889631
:10B6100090934A268093492688E10BC08091512B54
:10B6200081FFF8C088E290E090934A2680934926F3
:10B6300080E1809372265CC08091512B80FFEAC02C
:10B64000198E80E18093512B0E94084FE3C08091B6
:10B65000492690914A26009711F00E94465D9091EC
:10B6600072268091512B90FF0BC080FF06C087E0AF
:10B67000898F1A8E198A188A19C086E0898F16C098
:10B6800080FF1EC085E0898F198A188AC3C0809107
:10B69000492690914A26009711F00E94465D8091BC
:10B6A000722680FF0DC087E0898F1A8E81E090E0BE
:10B6B0000E94465D80E18093512B0E94084F0FC08D
:10B6C0008091492690914A26009749F4A3C0809121
:10B6D000512B80FF9FC087E0898F1A8E9BC080E12D
:10B6E0008093722688E290E090934A2680934926C0
:10B6F00080E580937126888580936D268985809367
:10B700006E268A8580936F268B85809370268C8524
:10B71000809369268D8580936A268E8580936B261B
:10B720008F8580936C2686E080935A268C819D813C
:10B7300090936626809365268E819F8190936826DC
:10B74000809367268091E82B9091E92BA091EA2BBA
:10B75000B091EB2B80935D2690935E26A0935F269D
:10B76000B093602688819981AA81BB8180936126EC
:10B7700090936226A0936326B0936426898D84FFFC
:10B7800005C0109274261092732606C084E0809340
:10B79000732688ED8093742680E4809359268091E7
:10B7A000492690914A2690935326809354261092CE
:10B7B00078261092772610927626109275260E948F
:10B7C0003D5380959095909376268093752685E4D9
:10B7D0008093512610925226109258261092572686
:10B7E0008091A2169091A31601969093A316809330
:10B7F000A216909355268093562610925C2610929E
:10B800005B260E942C538095909590935C268093A4
:10B810005B2604C010924A26109249261092512BA2
:10B82000DF91CF911F910F91FF90EF90DF90CF901C
:10B83000BF90AF90089598278927982708950F9370
:10B840001F93DC01CB011A2F0B2F20E030E098274B
:10B8500089279827A0E0B0E0DC0199278827082BEA
:10B86000192B2A2B3B2BB801C9011F910F91089569
:10B87000FC0120914B2630914C2681E59BE2821BF6
:10B88000930BAB01861797070CF4AC011416150641
:10B890005CF44093EC2B5093ED2BE217F30721F06F
:10B8A000C901BF010E9451660895CF92DF92EF92C5
:10B8B000FF920F93CF93DF93CDB7DEB760970FB6AC
:10B8C000F894DEBF0FBECDBF002309F45AC029870C
:10B8D0003A874B875C876D877E878F87988B80E25E
:10B8E000801B49855A856B857C851816B4F01982B2
:10B8F0001A821B821C82992787FD909590958195CD
:10B900009F4F04C0440F551F661F771F8A95D2F7BB
:10B910004D835E836F8378872CC06A017B01002E84
:10B9200004C0CC0CDD1CEE1CFF1C0A94D2F7C982AB
:10B93000DA82EB82FC826A017B0104C0F694E79410
:10B94000D794C7948A95D2F7D701C6014D855E85F5
:10B950006F85788904C0440F551F661F771F0A95AD
:10B96000D2F7842B952BA62BB72B8D839E83AF8389
:10B97000B88729813A814B815C816D817E818F817D
:10B98000988560960FB6F894DEBF0FBECDBFDF91ED
:10B99000CF910F91FF90EF90DF90CF900895A0E1AD
:10B9A000B0E0E5EDFCE50C946A6329873A874B87A4
:10B9B0005C876D877E878F87988BA982BA82CB82BE
:10B9C000DC82ED82FE820F8318874D855E856F8550
:10B9D00078898D819E81AF81B885481759076A079C
:10B9E0007B07C8F084179507A607B70790F049852D
:10B9F0005A856B857C8589819A81AB81BC8148178A
:10BA000059076A077B0738F084179507A607B70719
:10BA100020F482E003C080E001C081E06096EAE0AB
:10BA20000C94866380E880936100109261000E940C
:10BA30003D390E94C52C0E949C3D8091F823909135
:10BA4000F923009729F001979093F9238093F82325
:10BA5000C090FA23D090FB23E090FC23F090FD23CC
:10BA60000E94413CDC01CB01C816D906EA06FB0660
:10BA700001F30E94413CDC01CB018093FA239093B7
:10BA8000FB23A093FC23B093FD23D3CFBC01809173
:10BA9000562B9091572B08960E94E952E091562B15
:10BAA000F091572B80914D26808780914E2681877B
:10BAB00080914F26828780915026838708952F9208
:10BAC0003F924F925F926F927F928F929F92AF922E
:10BAD000BF92CF92DF92EF92FF920F931F93CF937B
:10BAE000DF93CDB7DEB765970FB6F894DEBF0FBE14
:10BAF000CDBF4C017F876E87FC0117821682838140
:10BB000081FD04C076C34C855D8504C01E01089488
:10BB1000211C311CF4019381EE85FF8593FD8591F5
:10BB200093FF8191FF87EE87882309F45EC38532F6
:10BB300041F493FD859193FF8191FF87EE878532D4
:10BB400059F490E0B4014C8B5D8B0E94A4664C8943
:10BB50005D895D874C87D7CFFF24DD2410E010324C
:10BB6000B0F48B3269F08C3228F4803251F0833299
:10BB700071F40BC08D3239F0803349F411602CC060
:10BB80001260146029C0186027C0106125C017FD1D
:10BB90002EC0282F20532A3098F416FF08C08F2D6E
:10BBA000880FF82EFF0CFF0CF80EF20E15C08D2D2D
:10BBB000880FD82EDD0CDD0CD80ED20E10620CC012
:10BBC0008E3221F416FD11C3106406C08C3611F4B8
:10BBD000106802C0883659F4EE85FF8593FD859183
:10BBE00093FF8191FF87EE87882309F0B8CF982FC4
:10BBF0009554933018F41061805E06C0982F9556C6
:10BC0000933008F0A2C11F7E16FD02C0E6E0FE2EB2
:10BC10001F73853611F4106406C0863611F410685F
:10BC200002C0F110FA9417FF07C0FBE3FF1548F0BC
:10BC3000EF2CE39427E00DC027E02F1530F02F2DD7
:10BC400007C027E07CE3E72E04C027E067E0F62E7C
:10BC5000EE24CA0104969D878C87FA016081718168
:10BC600082819381A1010E2D0E9461655C01C980D2
:10BC70002C2D30E0398B288BC0FE03C0388933FF70
:10BC800006C011FD06C012FF06C000E205C00DE2AD
:10BC900003C00BE201C000E0888999898C70907024
:10BCA000009709F43CC0002311F084E001C083E058
:10BCB0008D1558F4D81A13FD09C080E290E0B40144
:10BCC0000E94A466DA94C9F701C0DD24002329F09C
:10BCD000802F90E0B4010E94A466888983FD05C08E
:10BCE0003AE6E32E3CE0F32E11C026E6E22E2CE0ED
:10BCF000F22E0CC00115110509F0805290E0B4013C
:10BD00000E94A4660894E11CF11C04C0012F10E0FD
:10BD100000711070F7018491882361F763C217FFE7
:10BD20000EC0EA0CF889F4FF04C08A81813309F45B
:10BD3000EA941E144CF528E02E1548F12CC016FD8F
:10BD40002AC08F2D90E08A159B0544F03CEFA31686
:10BD50003FEFB3061CF0106801C0FA94FF2049F0D1
:10BD6000E2E0F0E0EC0FFD1FEF0DF11D808180336C
:10BD7000A1F317FF10C0EF2CE3948F2D90E0A816CD
:10BD8000B90644F4FA1807C0EE24E39404C098E01E
:10BD9000E92E01C0FF2417FF07C01A141B043CF44E
:10BDA00095012F5F3F4F05C025E030E002C021E044
:10BDB00030E0002311F02F5F3F4FFF2029F08F2D3F
:10BDC00090E00196280F391F8D2D90E02817390734
:10BDD00014F4D21A01C0DD24612E7724C3018970C6
:10BDE0009070009749F406C080E290E0B4010E9490
:10BDF000A466DA94DD20C1F7002329F0802F90E0BB
:10BE0000B4010E94A46663FC09C006C080E390E010
:10BE1000B4010E94A466DA94DD20C1F717FF48C080
:10BE20008501B7FE02C000E010E0442455249501CE
:10BE30002E1931093B8B2A8B3501601A710A620C6D
:10BE4000731C6F2D70E0EE24FF24E61AF70A3FEF13
:10BE50000F3F130729F48EE290E0B4010E94A4661C
:10BE6000A016B10654F02A893B89201731072CF41B
:10BE7000F301E40DF51D818101C080E30150104004
:10BE80000894411C511C0E151F052CF090E0B401C4
:10BE90000E94A466DCCF0A151B0541F49A819633F3
:10BEA00020F4953319F4388934FF81E390E049C0D8
:10BEB0008A81813311F09FEEC92290E0B4010E9483
:10BEC000A466FF2089F08EE290E0B4010E94A4668F
:10BED00012E0F101E10FF11D1F5F808190E0B401DC
:10BEE0000E94A466FA94A9F764FE03C085E490E07A
:10BEF00002C085E690E0B4010E94A466B7FC05C0CC
:10BF0000A114B10441F4C4FE06C0B094A194B108D8
:10BF1000B3948DE201C08BE290E0B4010E94A4666C
:10BF200080E305C08F5FE6EFFFEFAE0EBF1EFAE0C5
:10BF3000AF16B104BCF790E0B4010E94A466C5013D
:10BF4000C096B4010E94A4664DC1833631F0833798
:10BF500089F0833509F059C022C09A012E5F3F4F06
:10BF60003D872C87FA018081898381E0E82EF12CBE
:10BF7000510113C09A012E5F3F4F3D872C87FA0174
:10BF8000A080B18016FF03C06F2D70E002C06FEF7C
:10BF90007FEFC5010E946A667C011F7714C09A0179
:10BFA0002E5F3F4F3D872C87FA01A080B18016FF9E
:10BFB00003C06F2D70E002C06FEF7FEFC5010E94DC
:10BFC00041667C01106813FD1CC006C080E290E051
:10BFD000B4010E94A466DA948D2D90E0E816F9066B
:10BFE000A8F30FC0F50117FD859117FF81915F013F
:10BFF00090E0B4010E94A466D110DA940894E1089C
:10C00000F108E114F10471F7EDC0843611F08936BE
:10C0100071F59A0117FF0AC02C5F3F4F3D872C87AF
:10C02000FA0180819181A281B3810BC02E5F3F4FC5
:10C030003D872C87FA0180819181AA2797FDA095E1
:10C04000BA2F012F0F76B7FF08C0B095A095909535
:10C0500081959F4FAF4FBF4F0068BC01CD01A1013B
:10C060002AE030E00E94AC67E82EE21841C0853734
:10C0700021F41F7E2AE030E020C0197F8F36A9F01E
:10C08000803720F4883509F0B0C00BC0803721F02C
:10C09000883709F0AAC001C0106114FF09C01460FC
:10C0A00007C014FF08C0166006C028E030E005C0D5
:10C0B00020E130E002C020E132E0CA0117FF09C0F0
:10C0C00004969D878C87FA016081718182819381BA
:10C0D00008C002969D878C87FA016081718180E09B
:10C0E00090E0A1010E94AC67E82EE218012F0F77C3
:10C0F00006FF09C00E7FEF1430F404FF06C002FDF6
:10C1000004C00F7E02C01E2D01C01F2D802F90E0A5
:10C1100004FF0CC0FE01EE0DF11D2081203311F44F
:10C12000097E09C002FF06C01E5F05C086789070B8
:10C13000009709F01F5FA02EBB2403FD12C000FF73
:10C140000DC0FE2C1D1550F4FD0CF11A1D2D06C05E
:10C1500080E290E0B4010E94A4661F5F1D15C0F349
:10C1600004C01D1510F4D11A01C0DD24A4FE0FC0B7
:10C1700080E390E0B4010E94A466A2FE1FC0A1FE6D
:10C1800003C088E590E010C088E790E00DC0C501CD
:10C1900086789070009791F0A1FC02C080E201C007
:10C1A0008BE207FD8DE290E0B4010E94A46606C018
:10C1B00080E390E0B4010E94A466FA94EF14C0F307
:10C1C000EA94F101EE0DF11D808190E0B4010E942E
:10C1D000A466EE20A9F706C080E290E0B4010E94B8
:10C1E000A466DA94DD20C1F78ECCF40186819781B4
:10C1F00002C08FEF9FEF65960FB6F894DEBF0FBEBB
:10C20000CDBFDF91CF911F910F91FF90EF90DF9005
:10C21000CF90BF90AF909F908F907F906F905F90E6
:10C220004F903F902F9008955058BB27AA270ED0CB
:10C2300044C135D130F03AD120F031F49F3F11F4B0
:10C240001EF42AC10EF4E095E7FB20C1E92F46D188
:10C2500080F3BA17620773078407950718F071F423
:10C260009EF55EC10EF4E0950B2EBA2FA02D0B01AA
:10C27000B90190010C01CA01A0011124FF27591B2B
:10C2800099F0593F50F4503E68F11A16F040A22F31
:10C29000232F342F4427585FF3CF469537952795A2
:10C2A000A795F0405395C9F77EF41F16BA0B620BA1
:10C2B000730B840BBAF09150A1F0FF0FBB1F661FE8
:10C2C000771F881FC2F70EC0BA0F621F731F841F2B
:10C2D00048F4879577956795B795F7959E3F08F051
:10C2E000B3CF9395880F08F09927EE0F9795879510
:10C2F0000895A8D008F481E008950CD0DEC0D6D00F
:10C3000040F0CDD030F021F45F3F19F0BFC05111A3
:10C3100008C1C2C0E3D098F39923C9F35523B1F300
:10C32000951B550BBB27AA2762177307840738F0A4
:10C330009F5F5F4F220F331F441FAA1FA9F333D003
:10C340000E2E3AF0E0E830D091505040E695001CB7
:10C35000CAF729D0FE2F27D0660F771F881FBB1F73
:10C36000261737074807AB07B0E809F0BB0B802D4D
:10C37000BF01FF2793585F4F2AF09E3F510568F099
:10C3800085C0CFC05F3FECF3983EDCF38695779590
:10C390006795B795F7959F5FC9F7880F911D96959B
:10C3A000879597F90895E1E0660F771F881FBB1FF7
:10C3B000621773078407BA0720F0621B730B840BA4
:10C3C000BA0BEE1F88F7E0950895E89409C097FB33
:10C3D0003EF490958095709561957F4F8F4F9F4F5C
:10C3E0009923A9F0F92F96E9BB279395F6958795A0
:10C3F00077956795B795F111F8CFFAF4BB0F11F463
:10C4000060FF1BC06F5F7F4F8F4F9F4F16C0882309
:10C4100011F096E911C0772321F09EE8872F762F3F
:10C4200005C0662371F096E8862F70E060E02AF080
:10C430009A95660F771F881FDAF7880F969587956C
:10C4400097F90895990F0008550FAA0BE0E8FEEF41
:10C4500016161706E807F907C0F012161306E407C8
:10C46000F50798F0621B730B840B950B39F40A26C1
:10C4700061F0232B242B252B21F408950A2609F49F
:10C48000A140A6958FEF811D811D089597F99F67A3
:10C4900080E870E060E008959FEF80EC089500244C
:10C4A0000A941616170618060906089500240A9419
:10C4B00012161306140605060895092E0394000C9F
:10C4C00011F4882352F0BB0F40F4BF2B11F460FF2E
:10C4D00004C06F5F7F4F8F4F9F4F089557FD905857
:10C4E000440F551F59F05F3F71F04795880F97FB38
:10C4F000991F61F09F3F79F08795089512161306F2
:10C500001406551FF2CF4695F1DF08C01616170620
:10C510001806991FF1CF8695710561050894089555
:10C52000E894BB2766277727CB0197F908950BD0AE
:10C53000C4CFB5DF28F0BADF18F0952309F0A6CFF5
:10C54000ABCF1124EECFCADFA0F3959FD1F3950FA7
:10C5500050E0551F629FF001729FBB27F00DB11D87
:10C56000639FAA27F00DB11DAA1F649F6627B00D17
:10C57000A11D661F829F2227B00DA11D621F739F00
:10C58000B00DA11D621F839FA00D611D221F749F0E
:10C590003327A00D611D231F849F600D211D822F55
:10C5A000762F6A2F11249F5750408AF0E1F088239C
:10C5B0004AF0EE0FFF1FBB1F661F771F881F9150A9
:10C5C0005040A9F79E3F510570F060CFAACF5F3F62
:10C5D000ECF3983EDCF3869577956795B795F795DC
:10C5E000E7959F5FC1F7FE2B880F911D9695879564
:10C5F00097F90895629FD001739FF001829FE00D2B
:10C60000F11D649FE00DF11D929FF00D839FF00DD1
:10C61000749FF00D659FF00D9927729FB00DE11D7D
:10C62000F91F639FB00DE11DF91FBD01CF0111245A
:10C630000895AA1BBB1B51E107C0AA1FBB1FA61769
:10C64000B70710F0A61BB70B881F991F5A95A9F7BB
:10C6500080959095BC01CD01089597FB092E072682
:10C660000AD077FD04D0E5DF06D000201AF47095DB
:10C6700061957F4F0895F6F7909581959F4F0895A6
:10C68000A1E21A2EAA1BBB1BFD010DC0AA1FBB1FD6
:10C69000EE1FFF1FA217B307E407F50720F0A21B48
:10C6A000B30BE40BF50B661F771F881F991F1A94B5
:10C6B00069F760957095809590959B01AC01BD01DF
:10C6C000CF0108952F923F924F925F926F927F9287
:10C6D0008F929F92AF92BF92CF92DF92EF92FF9292
:10C6E0000F931F93CF93DF93CDB7DEB7CA1BDB0B3E
:10C6F0000FB6F894DEBF0FBECDBF09942A883988E3
:10C7000048885F846E847D848C849B84AA84B984E9
:10C71000C884DF80EE80FD800C811B81AA81B981F5
:10C72000CE0FD11D0FB6F894DEBF0FBECDBFED0109
:10C7300008958F929F92AF92BF92CF92DF92EF9225
:10C74000FF92CF93DF93EC0188819981AA81BB810D
:10C750000097A105B10521F484E299EDABE5B7E0BE
:10C76000BC01CD012DE133EF41E050E00E94DF69D3
:10C7700049015A0127EA31E440E050E00E94FA62A0
:10C780006B017C01C501B4012CEE34EF4FEF5FEF7C
:10C790000E94FA62DC01CB01C80ED91EEA1EFB1E04
:10C7A000F7FE08C08FEF9FEFAFEFBFE7C80ED91EAF
:10C7B000EA1EFB1EC882D982EA82FB82C6019F77ED
:10C7C000DF91CF91FF90EF90DF90CF90BF90AF902F
:10C7D0009F908F9008950E949963089586E096E057
:10C7E0000E9499630895A0E0B0E0809306069093BC
:10C7F0000706A0930806B093090608953F924F924A
:10C800005F926F927F928F929F92AF92BF92CF92E0
:10C81000DF92EF92FF920F931F93CF93DF9300D09D
:10C8200000D0CDB7DEB72B017A016115710529F073
:10C83000DB018C9311969C931197E114F10439F06C
:10C840009701225030402332310508F0FCC06C01C2
:10C8500086010894C11CD11CF80130803601832D5B
:10C8600090E00E943966009799F7FDE23F1661F467
:10C87000D80111963C90119792E0692E712C600EB0
:10C88000711ECC24C3940BC0BBE23B1639F4F801F3
:10C89000318082E0682E712C600E711ECC24E11470
:10C8A000F10421F0F0E1EF16F104F9F480E3381619
:10C8B00091F4D3018C91883711F0883561F4F3013C
:10C8C000318082E090E0680E791E92E0C92AB0E1E2
:10C8D000EB2EF12C0AC0E114F10439F4A0E33A166E
:10C8E000D1F0AAE0EA2EF12C30C0BAE0EB16F10448
:10C8F00061F1E0E1EE16F10429F0F8E0EF16F10441
:10C90000B1F409C0FFEF8F2EFFEF9F2EFFEFAF2E88
:10C91000FFE0BF2E22C078E0E72EF12CEFEF8E2E45
:10C92000EFEF9E2EEFEFAE2EEFE1BE2E16C0970179
:10C93000442737FD4095542F6FEF7FEF8FEF9FEF28
:10C940000E94406349015A0108C069E9862E69E9DD
:10C95000962E69E9A62E69E1B62E40E000E010E0CF
:10C9600020E030E0C701AA2797FDA095BA2F898360
:10C970009A83AB83BC8350EDD52ED30C99E09D15E3
:10C9800070F4832D81548A3118F499ECD92E06C0A5
:10C99000832D81568A3168F589EAD82ED30C8D2DE6
:10C9A00090E08E159F052CF54F3FF9F0801691060B
:10C9B000A206B306B8F0C901B80129813A814B81BA
:10C9C0005C810E94FA628B019C018D2D90E0A0E0B9
:10C9D000B0E0080F191F2A1F3B1F081719072A0765
:10C9E0003B0710F44FEF01C041E0D3013D903D0102
:10C9F000C2CF4114510489F0442339F008946108EE
:10CA00007108F2017182608208C0C1FE06C0C301D4
:10CA10000297D20111969C938E93C0FE07C0309569
:10CA20002095109501951F4F2F4F3F4F47FF0FC087
:10CA300082E290E09093772C8093762C0FEF1FEF9B
:10CA40002FEF3FEF04C000E010E020E030E0B8013D
:10CA5000C9010F900F900F900F90DF91CF911F9110
:10CA60000F91FF90EF90DF90CF90BF90AF909F908D
:10CA70008F907F906F905F904F903F9008956627C2
:10CA800077270C944568FC0188279927E894219121
:10CA90002032E9F3293010F02E30C8F32B3241F068
:10CAA0002D3239F4689404C00E949C66820F911D57
:10CAB000219120532A30C0F31EF4909581959F4F09
:10CAC0000895283008F027E03327DA01990F311D47
:10CAD00087FD916000966105710539F432602E5F23
:10CAE0003D9330E32A95E1F708959F3F30F0803879
:10CAF0007105610509F03C5F3C5F3D93913008F0A2
:10CB00008068911DDF93CF931F930F93FF92EF9255
:10CB1000192F987F9695E92F96959695E90FFF27FF
:10CB2000E853F34F99273327EE24FF24A701E701A9
:10CB300005900894079428F4360FE71EF81E491F45
:10CB4000511D660F771F881F991F0694A1F7059046
:10CB5000079428F4E70EF81E491F561FC11D770FD2
:10CB6000881F991F661F0694A1F70590079428F463
:10CB7000F80E491F561FC71FD11D880F991F661F2A
:10CB8000771F0694A1F70590079420F4490F561FCC
:10CB9000C71FD81F990F661F771F881F0694A9F714
:10CBA00084911095177041F0D695C7955795479584
:10CBB000F794E7941A95C1F7EEE6FCE068941590B7
:10CBC000159135916591959105907FE27395E118E6
:10CBD000F10A430B560BC90BD009C0F7E10CF11E4B
:10CBE000431F561FC91FD01D7EF4703311F48A9560
:10CBF000E6CFE894015030F0080F0AF4002702173E
:10CC000008F4202F2395022F7A3328F079E37D93BF
:10CC10002A95E9F710C07D932A9589F60694979591
:10CC20006795379517951794E118F10A430B560B42
:10CC3000C90BD00998F023957E9173957A3308F04B
:10CC400070E37C932013B8F77E9170617D9330F090
:10CC5000839571E37D9370E32A95E1F71124EF90BA
:10CC6000FF900F911F91CF91DF91992787FD9095AC
:10CC70000895911189C3803219F089508550D0F7F9
:10CC80000895FC010590615070400110D8F780951F
:10CC900090958E0F9F1F08954EEA56E10E9475668B
:10CCA0000895FB01DC0102C001900D9241505040FB
:10CCB000D8F70895DC0101C06D9341505040E0F772
:10CCC0000895FB01DC018D91019080190110D9F3C9
:10CCD000990B0895FC016150704001900110D8F744
:10CCE000809590958E0F9F1F0895FA01A191B081B4
:10CCF000009719F41097E1F0CD01DC01CD010D9002
:10CD0000002011F4C00113C0FB012191222319F06E
:10CD10002015D9F7F3CFFB012191201519F41E92AC
:10CD2000119606C02223C1F70D900020A1F7D00173
:10CD3000FA01A193B08308957AE0979F902D879F81
:10CD4000802D910D112408950F931F93CF93DF939E
:10CD50008C01EB018B8181FF1BC082FF0DC02E81F6
:10CD60003F818C819D812817390764F4E881F9811E
:10CD70000193F983E88306C0E885F985802F09953A
:10CD8000009731F48E819F8101969F838E8302C02C
:10CD90000FEF1FEFC801DF91CF911F910F91089501
:10CDA000CF93DF93CDB7DEB7FE01359661917191D8
:10CDB0008091722C9091732CAF010E945F5DDF9186
:10CDC000CF910895CF93DF93CDB7DEB7FE013596AF
:10CDD000619171918091722C9091732CDC0113966A
:10CDE0002C911397286013962C93AF010E945F5DDE
:10CDF000E091722CF091732C2381277F2383DF91A4
:10CE0000CF9108956091722C7091732C0E94A4664A
:10CE100008950F931F93CF93DF938C01E091722CB1
:10CE2000F091732C838181FF1AC0C0E0D0E005C06F
:10CE30000995009711F0CFEFDFEFF80181918F0195
:10CE40006091722C7091732CDB011896ED91FC911E
:10CE50001997882369F78AE00995009711F0CFEFB9
:10CE6000DFEFCE01DF91CF911F910F9108950F93C6
:10CE70001F93CF93DF93CDB7DEB72E970FB6F894FD
:10CE8000DEBF0FBECDBF0D891E898F89988D26E02C
:10CE90002C831A83098397FF02C080E090E80197F2
:10CEA0009E838D83AE01455E5F4FCE010196698DF5
:10CEB0007A8D0E945F5D4D815E8157FD0AC02F8192
:10CEC0003885421753070CF49A01020F131FF8011B
:10CED00010822E960FB6F894DEBF0FBECDBFDF9145
:10CEE000CF911F910F9108950F931F93CF93DF93CD
:10CEF000CDB7DEB72E970FB6F894DEBF0FBECDBF0D
:10CF00008C0186E08C831A83098377FF02C060E07E
:10CF100070E8615070407E836D83CE010196BA0146
:10CF2000A9010E945F5D4D815E8157FD0AC02F817E
:10CF30003885421753070CF49A01020F131FF801AA
:10CF400010822E960FB6F894DEBF0FBECDBFDF91D4
:10CF5000CF911F910F910895FA01AA27283051F11E
:10CF6000203181F1E8946F936E7F6E5F7F4F8F4F1A
:10CF70009F4FAF4FB1E03ED0B4E03CD0670F781F79
:10CF8000891F9A1FA11D680F791F8A1F911DA11D5E
:10CF90006A0F711D811D911DA11D20D009F4689497
:10CFA0003F912AE0269F11243019305D3193DEF63F
:10CFB000CF010895462F4770405D4193B3E00FD0F5
:10CFC000C9F7F6CF462F4F70405D4A3318F0495DE0
:10CFD00031FD4052419302D0A9F7EACFB4E0A695C3
:10CFE0009795879577956795BA95C9F700976105E5
:10CFF000710508959B01AC010A2E0694579547953B
:10D0000037952795BA95C9F7620F731F841F951F2F
:10D01000A01D0895DC01CB01FC01F999FECF06C0EB
:10D02000F2BDE1BDF89A319600B40D9241505040E6
:10D03000B8F70895F999FECF92BD81BDF89A992766
:10D0400080B50895A8E1B0E042E050E00C940C688F
:10D05000DC01CB0103C02D910E9433684150504048
:10D06000D0F70895262FF999FECF1FBA92BD81BD42
:10D0700020BD0FB6F894FA9AF99A0FBE019608955A
:10D080000E943268272F0C9433686F927F928F92A0
:10D090009F92AF92BF92CF92DF92EF92FF920F9347
:10D0A0001F93CF93DF935B016115710521F0DB01C5
:10D0B0008C9311969C937C01E7010894E11CF11C70
:10D0C00008816701802F90E00E9439660097A1F7E0
:10D0D0000D3241F4098142E0C42ED12CCC0EDD1E6C
:10D0E00011E009C00B3231F4098132E0C32ED12C9A
:10D0F000CC0EDD1E10E0E6012197CE0168E67DE052
:10D1000043E050E00E94C7690097D1F4E6012296FF
:10D11000CE016BE67DE045E050E00E94C7690097D4
:10D1200011F4E6012796A114B10419F0F501D18399
:10D13000C08330E020E090E8112309F40DC107C15D
:10D14000CE0160E77DE043E050E00E94C7690097B0
:10D1500059F4A114B10409F4FCC0C6010296D5012A
:10D1600011969C938E93F5C040E050E060E070E033
:10D170008824992400530A3090F51260212F30E062
:10D18000C9018870907012FF06C0009769F5089475
:10D19000811C911C29C0009719F0089481089108FE
:10D1A000DB01CA01D2E0880F991FAA1FBB1FDA95C5
:10D1B000D1F7480F591F6A1F7B1F440F551F661F69
:10D1C000771F400F511D611D711D4839B9E95B077B
:10D1D000B9E96B07B9E17B0738F0146005C00E3F71
:10D1E00039F413FD43C01860F60101916F01C2CFFD
:10D1F000053311F00531D1F5D601EC91ED3211F482
:10D20000106108C0EB3229F0C601019621E030E040
:10D2100008C0D6011196EC911197C601029622E042
:10D2200030E0E053EA3020F06C01C21AD30A1EC08D
:10D23000DC0120E030E0FCE020383F075CF4C9016D
:10D24000880F991F880F991F280F391F220F331F2E
:10D250002E0F311DED91E0536D01EA3060F314FFA4
:10D2600003C0309521953F4F820E931EC12FD0E011
:10D2700011FF08C0A114B10429F0C6010197D5011E
:10D280008D939C93CB01BA010E94E5616B017C01F7
:10D29000CE01837090708330910521F4F7FAF094F9
:10D2A000F7F8F094C701B60120E030E040E050E02C
:10D2B0000E947961882309F445C097FE07C09094C5
:10D2C000819491089394CFE9DDE002C0C7E8DDE0E6
:10D2D00098EE692E9FEF792E6C0E7D1E20E2A22E15
:10D2E000B12C0FC0FE010591159125913491C70114
:10D2F000B601A90198010E9497626B017C018A180E
:10D300009B088A149B0474F72497B594A794C615B8
:10D31000D705B9F7C601D7012A2F220F2B2F221FBD
:10D320002F3F51F0BC01CD0120E030E040E050E063
:10D330000E947961882331F482E290E09093772C07
:10D340008093762C3C2D2D2D9E2D8F2D06C08FEF9A
:10D3500004C030E020E090EC8FE7B901AC01872FEA
:10D36000922FA52FB42FBC01CD01DF91CF911F913A
:10D370000F91FF90EF90DF90CF90BF90AF909F9074
:10D380008F907F906F900895992788270895FB01CB
:10D39000DC014150504088F08D9181341CF08B3578
:10D3A0000CF4805E659161341CF06B350CF4605EAA
:10D3B000861B611171F3990B0895881BFCCF97FBB5
:10D3C000092E05260ED057FD04D05AD90AD0001CCC
:10D3D00038F450954095309521953F4F4F4F5F4F12
:10D3E0000895F6F790958095709561957F4F8F4FD2
:08D3F0009F4F0895F894FFCF50
:10D3F800263A202573205B414444523D252D642E56
:10D40800252D64205345513D252D64205253534901
:10D418003D252D75204C51493D252D7520445250F0
:10D428003D252D642E253032645D0A0054696D65F2
:10D438006F757420414444523D252D642E252D647A
:10D44800205345513D252D6420525353493D252DE8
:10D4580075204C51493D252D750A00284578745092
:10D4680077722900007374617475733D30782530C4
:10D4780032780A2000312E30204669726D77617249
:10D4880065205665722E20332E3220323031322DEF
:10D4980031302D303900656570726F6D006F6E0028
:10D4A8006F666600666F7263655F69646C650064C9
:10D4B800656570004F6E00613100726573657400B8
:10D4C800613200765F696E0031003200330034004B
:10D4D8006175746F00666C75736800414444523D11
:10D4E800252D642E252D64205345513D252D64207E
:10D4F800525353493D252D75204C51493D252D75D5
:10D508000A00707772733D25730A007472696D00A2
:10D5180043683D252D642054785077723D252D644D
:10D528000A004572726F72205458204C656E6774F9
:10D53800683D25640A0049443D00253032780020C2
:10D5480050533D25640020543D252D362E3266006B
:10D558002054313D252D362E32660020545F4D4330
:10D56800553D252D352E31660020565F4D43553DDE
:10D57800252D342E3266002050303D252D6C580064
:10D588002050305F543D252D372E33660020503112
:10D598003D252D6C58002050315F543D252D372EE8
:10D5A8003366002055503D252D6C58002052483DCB
:10D5B800252D342E31660020565F494E3D252D35E8
:10D5C8002E32660020565F41313D252D352E3266BC
:10D5D8000020565F41323D252D352E326600263A11
:10D5E8002025730A00545820706B74206C656E20D7
:10D5F8003D2025640A0025303258006C656E3D25B3
:10D60800640A0075045F0447042B040000536C652A
:10D6180065702070726F636573730000001D04F9F4
:10D628000D0000000062726F6164636173742070A2
:10D63800726F636573730000003504B12400000045
:10D6480000737464696E2070726F63657373000091
:10D658000051040B0D00000000636D642070726FB0
:10D66800636573730000006904F823000000000A72
:10D67800003C00130A6162636465666768696A6BE7
:10D688006C6D6E6F7020090D0095041A22FFCC3B5B
:10D6980022FFCC3BED478A3C010010001D004000F2
:10D6A800380678060E0700000000302B242B1810CF
:10D6B800000000004576656E742074696D6572001F
:10D6C8000000C404182F000000004374696D6572DF
:10D6D8002070726F63657373000000DA044E3000C7
:10D6E800000000020306070A0B0E0F436F6E7469F1
:10D6F8006B6920322E3500C600C500C400C100C2C7
:10D7080000000000CE00CD00CC00C900CA00000017
:10D718000000000002000000000C3D000000005264
:10D7280046323330206472697665720000002F0536
:10D73800BC41000000001940563F0B424D43AC402D
:10D74800AF3FBA3DB43DA43E953F00010101010140
:10D75800010101010101010101010052696D65002A
:10D768006B05BE44894461646174612E6E756D20D9
:10D77800776179206F75742074686572653A202521
:10D78800640A00F745F6450048244956470080C01A
:10D79800E0F0F8FCFEFF6E756C6C6D616300A60529
:10D7A800D049B549BB49C149C749CD497369637374
:10D7B8006C6F776D616300BC05E14A454ADA49D16F
:10D7C80049EB4AD749BA00080037103F1035000224
:10D7D800000F1611165443502F495020737461637B
:10D7E8006B000000E505284D00000000020800005D
:0AD7F8000000FFFFFFFF010000002A
:00000001FF
